:020000021000EC
:10000000B8270120B14F01005BDE07009D4F0100C2
:100010009D4F01009D4F01009D4F01009D4F01002C
:10002000000000000000000000000000E94F010097
:100030009D4F010000000000355201009D4F01005E
:10004000F9520100F9520100F9520100F952010080
:10005000F9520100F9520100F9520100F952010070
:10006000F9520100F9520100F9520100F952010060
:10007000F9520100F9520100F9520100F952010050
:10026000F9520100F9520100014E0300F952010058
:10027000F9520100F9520100F9520100F95201004E
:10028000F9520100F9520100F9520100F95201003E
:10029000F9520100F9520100F9520100F95201002E
:1002A000F9520100F9520100F9520100F95201001E
:1004800081F0004102E000BF83F0004330B54FEA45
:1004900041044FEA430594EA050F08BF90EA020FB2
:1004A0001FBF54EA000C55EA020C7FEA645C7FEA45
:1004B000655C00F0E2804FEA5454D4EB5555B8BF68
:1004C0006D420CDD2C4480EA020281EA030382EAD9
:1004D000000083EA010180EA020281EA0303362D6B
:1004E00088BF30BD11F0004F4FEA01314FF4801C3E
:1004F0004CEA113102D0404261EB410113F0004F50
:100500004FEA03334CEA133302D0524263EB430306
:1005100094EA050F00F0A780A4F10104D5F1200EA4
:100520000DDB02FA0EFC22FA05F2801841F10001FF
:1005300003FA0EF2801843FA05F359410EE0A5F1D3
:1005400020050EF1200E012A03FA0EFC28BF4CF004
:10055000020C43FA05F3C01851EBE37101F00045BA
:1005600007D54FF0000EDCF1000C7EEB00006EEBC7
:100570000101B1F5801F1BD3B1F5001F0CD3490851
:100580005FEA30004FEA3C0C04F101044FEA4452A8
:1005900012F5800F80F09A80BCF1004F08BF5FEA2F
:1005A000500C50F1000041EB045141EA050130BD0F
:1005B0005FEA4C0C404141EB0101013C28BFB1F521
:1005C000801FE9D291F0000F04BF01460020B1FA6C
:1005D00081F308BF2033A3F10B03B3F120020CDA3F
:1005E0000C3208DD02F1140CC2F10C0201FA0CF01D
:1005F00021FA02F10CE002F11402D8BFC2F1200C82
:1006000001FA02F120FA0CFCDCBF41EA0C01904037
:10061000E41AA2BF01EB0451294330BD6FEA040480
:100620001F3C1CDA0C340EDC04F11404C4F120026B
:1006300020FA04F001FA02F340EA030021FA04F37D
:1006400045EA030130BDC4F10C04C4F1200220FAD4
:1006500002F001FA04F340EA0300294630BD21FA12
:1006600004F0294630BD94F0000F83F4801306BFD8
:1006700081F480110134013D4EE77FEA645C18BFCC
:100680007FEA655C29D094EA050F08BF90EA020F63
:1006900005D054EA000C04BF1946104630BD91EA5B
:1006A000030F1EBF0021002030BD5FEA545C05D15E
:1006B0004000494128BF41F0004130BD14F580049D
:1006C0003CBF01F5801130BD01F0004545F0FE4111
:1006D00041F470014FF0000030BD7FEA645C1ABF46
:1006E000194610467FEA655C1CBF0B46024650EA7D
:1006F000013406BF52EA033591EA030F41F40021A9
:1007000030BD00BF90F0000F04BF0021704730B52E
:100710004FF4806404F132044FF000054FF0000103
:1007200050E700BF90F0000F04BF0021704730B5C4
:100730004FF4806404F1320410F0004548BF404299
:100740004FF000013EE700BF42004FEAE2014FEAEE
:1007500031014FEA02701FBF12F07F4393F07F4FC9
:1007600081F06051704732F07F4208BF704793F0CC
:100770007F4F04BF41F40021704730B54FF46074DF
:1007800001F0004521F000411CE700BF50EA0102E2
:1007900008BF704730B54FF000050AE050EA01028B
:1007A00008BF704730B511F0004502D5404261EBFB
:1007B00041014FF4806404F132045FEA915C3FF43C
:1007C000D8AE4FF003025FEADC0C18BF03325FEAD9
:1007D000DC0C18BF033202EBDC02C2F1200300FA8A
:1007E00003FC20FA02F001FA03FE40EA0E0021FAAF
:1007F00002F11444BDE600BF70B54FF0FF0C4CF49D
:10080000E06C1CEA11541DBF1CEA135594EA0C0F4E
:1008100095EA0C0F00F0DEF82C4481EA030621EA89
:100820004C5123EA4C5350EA013518BF52EA0335C4
:1008300041F4801143F4801338D0A0FB02CE4FF076
:100840000005E1FB02E506F00042E0FB03E54FF0A6
:100850000006E1FB03569CF0000F18BF4EF0010E9E
:10086000A4F1FF04B6F5007F64F5407404D25FEA9A
:100870004E0E6D4146EB060642EAC62141EA55514D
:100880004FEAC52040EA5E504FEACE2EB4F1FD0C8F
:1008900088BFBCF5E06F1ED8BEF1004F08BF5FEA0D
:1008A000500E50F1000041EB045170BD06F00046BF
:1008B00046EA010140EA020081EA0301B4EB5C046C
:1008C000C2BFD4EB0C0541EA045170BD41F4801164
:1008D0004FF0000E013C00F3AB8014F1360FDEBF89
:1008E000002001F0004170BDC4F10004203C35DA65
:1008F0000C341BDC04F11404C4F1200500FA05F3E8
:1009000020FA04F001FA05F240EA020001F0004288
:1009100021F0004110EBD37021FA04F642EB0601FE
:100920005EEA430E08BF20EAD37070BDC4F10C0428
:10093000C4F1200500FA04F320FA05F001FA04F2EC
:1009400040EA020001F0004110EBD37041F10001D8
:100950005EEA430E08BF20EAD37070BDC4F12005E3
:1009600000FA05F24EEA020E20FA04F301FA05F24B
:1009700043EA020321FA04F001F0004121FA04F2F3
:1009800020EA020000EBD3705EEA430E08BF20EAC3
:10099000D37070BD94F0000F0FD101F000464000FD
:1009A00041EB010111F4801F08BF013CF7D041EA7F
:1009B000060195F0000F18BF704703F00046520083
:1009C00043EB030313F4801F08BF013DF7D043EA54
:1009D0000603704794EA0C0F0CEA135518BF95EA0A
:1009E0000C0F0CD050EA410618BF52EA4306D1D191
:1009F00081EA030101F000414FF0000070BD50EAB0
:100A0000410606BF1046194652EA430619D094EA39
:100A10000C0F02D150EA013613D195EA0C0F05D123
:100A200052EA03361CBF104619460AD181EA030177
:100A300001F0004141F0FE4141F470014FF000002F
:100A400070BD41F0FE4141F4780170BD70B54FF0CA
:100A5000FF0C4CF4E06C1CEA11541DBF1CEA13554A
:100A600094EA0C0F95EA0C0F00F0A7F8A4EB05042C
:100A700081EA030E52EA03354FEA013100F0888023
:100A80004FEA03334FF0805545EA131343EA1263EC
:100A90004FEA022245EA111545EA10654FEA0026A1
:100AA0000EF000419D4208BF964244F1FD0404F55A
:100AB000407402D25B084FEA3202B61A65EB0305B6
:100AC0005B084FEA32024FF480104FF4002CB6EB73
:100AD000020E75EB030E22BFB61A754640EA0C00F3
:100AE0005B084FEA3202B6EB020E75EB030E22BF33
:100AF000B61A754640EA5C005B084FEA3202B6EB74
:100B0000020E75EB030E22BFB61A754640EA9C0032
:100B10005B084FEA3202B6EB020E75EB030E22BF02
:100B2000B61A754640EADC0055EA060E18D04FEAC0
:100B3000051545EA16754FEA06164FEAC30343EA60
:100B400052734FEAC2025FEA1C1CC0D111F4801F2D
:100B50000BD141EA00014FF000004FF0004CB6E726
:100B600011F4801F04BF01430020B4F1FD0C88BFC5
:100B7000BCF5E06F3FF6AFAEB5EB030C04BFB6EBD0
:100B8000020C5FEA500C50F1000041EB045170BDC3
:100B90000EF0004E4EEA113114EB5C04C2BFD4EBF0
:100BA0000C0541EA045170BD41F480114FF0000E74
:100BB000013C90E645EA060E8DE60CEA135594EAF0
:100BC0000C0F08BF95EA0C0F3FF43BAF94EA0C0FF3
:100BD0000AD150EA01347FF434AF95EA0C0F7FF468
:100BE00025AF104619462CE795EA0C0F06D152EABC
:100BF00003353FF4FDAE1046194622E750EA4106A0
:100C000018BF52EA43067FF4C5AE50EA41047FF4B0
:100C10000DAF52EA43057FF4EBAE12E74FF0FF3C15
:100C200006E000BF4FF0010C02E000BF4FF0010CE6
:100C30004DF804CD4FEA410C7FEA6C5C4FEA430C5F
:100C400018BF7FEA6C5C1BD001B050EA410C0CBFAE
:100C500052EA430C91EA030F02BF90EA020F002010
:100C6000704710F1000F91EA030F58BF994208BF77
:100C700090422CBFD8176FEAE37040F00100704734
:100C80004FEA410C7FEA6C5C02D150EA013C07D18B
:100C90004FEA430C7FEA6C5CD6D152EA033CD3D0D6
:100CA0005DF8040B704700BF8446104662468C46D0
:100CB0001946634600E000BF01B5FFF7B7FF002803
:100CC00048BF10F1000F01BD4DF808EDFFF7F4FF2C
:100CD0000CBF012000205DF808FB00BF4DF808EDB7
:100CE000FFF7EAFF34BF012000205DF808FB00BFDA
:100CF0004DF808EDFFF7E0FF94BF012000205DF8FC
:100D000008FB00BF4DF808EDFFF7CEFF94BF0120B0
:100D100000205DF808FB00BF4DF808EDFFF7C4FFA9
:100D200034BF012000205DF808FB00BF4FEA4102FC
:100D300012F5001215D211D56FF47873B3EB62522D
:100D400012D94FEAC12343F0004343EA505311F054
:100D5000004F23FA02F018BF404270474FF00000E6
:100D6000704750EA013005D111F0004008BF6FF024
:100D7000004070474FF00000704700BF4FEA41024B
:100D8000B2F1E04324BFB3F5001CDCF1FE5C0DD9E9
:100D900001F0004C4FEAC0024CEA5070B2F1004F33
:100DA00040EB830008BF20F00100704711F0804F36
:100DB00021D113F13872BCBF01F00040704741F4FB
:100DC00080114FEA5252C2F11802C2F1200C10FAFF
:100DD0000CF320FA02F018BF40F001004FEAC123E3
:100DE0004FEAD32303FA0CFC40EA0C0023FA02F387
:100DF0004FEA4303CCE77FEA625307D150EA01335D
:100E00001EBF4FF0FE4040F44000704701F000402C
:100E100040F0FE4040F40000704700BF7BB972B95B
:100E20000029BEBF00204FF0004106E008BF0028A7
:100E30001CBF6FF000414FF0FF3000F057B8ADF12C
:100E4000080C6DE904CE002909DB002B1ADB00F049
:100E500069F8DDF804E0DDE9022304B070474042A0
:100E600061EB4101002B1BDB00F05CF8DDF804E0D6
:100E7000DDE9022304B0404261EB4101524263EBE1
:100E800043037047524263EB430300F04BF8DDF835
:100E900004E0DDE9022304B0404261EB4101704708
:100EA000524263EB430300F03DF8DDF804E0DDE976
:100EB000022304B0524263EB4303704753B94AB96B
:100EC000002908BF00281CBF4FF0FF314FF0FF3052
:100ED00000F00CB8ADF1080C6DE904CE00F022F87A
:100EE000DDF804E0DDE9022304B07047704700BF7D
:100EF00010F8012B11F8013B012A28BF9A42F7D0C4
:100F0000D01A7047034611F8012B03F8012B002A71
:100F1000F9D17047034613F8012B002AFBD1181AA8
:100F2000013870472DE9F0478C468E46089E1546DD
:100F300004461946002B40F0D080724547D9B2FADA
:100F400082F74FB1C7F120030EFA07FCBD40BC4049
:100F500020FA03F343EA0C0C4FEA154EA8B2230C17
:100F6000BCFBFEF80EFB18CC08FB00F943EA0C436F
:100F7000994528D9EB1808F1FF3204D2994502D9D6
:100F8000A8F102022B44A3EB0903A4B2B3FBFEFCBD
:100F90000EFB1C330CFB00F044EA0344A04214D9BE
:100FA0002C190CF1FF3304D2A04202D9ACF1020398
:100FB0002C44241A43EA02401EB1FC400023346052
:100FC0007360BDE8F0874246DDE76346F1E7002A3B
:100FD00079D0B2FA82F3002B3FD01946C1F1200339
:100FE00002FA01F500FA01F42EFA03F20EFA01FEFC
:100FF00020FA03F3AFB243EA0E034FEA154EB2FBF9
:10100000FEFC0EFB1C201A0C0CFB07F842EA004207
:1010100090455AD9AA180CF1FF3004D2904502D954
:10102000ACF102002A44A2EB08029BB2B2FBFEFC28
:101030000EFB1C220CFB07F743EA02439F4246D9F2
:10104000EB180CF1FF3204D29F4202D9ACF102023C
:101050002B44DB1B42EA004202E0AEEB020301221A
:101060004FEA154EAFB2200CB3FBFEFC0EFB1C3357
:101070000CFB07F840EA034398452AD9EB180CF11A
:10108000FF3004D2984502D9ACF102002B44A3EB07
:101090000803A4B2B3FBFEFC0EFB1C330CFB07F7EA
:1010A00044EA0344A74216D92C190CF1FF3304D2A9
:1010B000A74202D9ACF102032C44E41B43EA0040EE
:1010C0000F46114678E71F2188E76046ABE7624686
:1010D000BFE76046DBE76346EFE7734506D916B91D
:1010E000002108466DE7C6E9000EF9E7B3FA83F779
:1010F00087B9734501D3824207D8841A6EEB030384
:1011000001209C461EB900215BE73846FAE7C6E994
:10111000004CF8E7C7F1200CBB4000FA07F422FAB4
:101120000CF520FA0CF1BA401D432EFA0CF30EFA1E
:1011300007FE4FEA154941EA0E011FFA85FEB3FB8F
:10114000F9F809FB18300B0C08FB0EFA43EA0043D0
:101150009A4540D9EB1808F1FF3004D29A4502D9DC
:10116000A8F102002B44A3EB0A0389B2B3FBF9F800
:1011700009FB183308FB0EFE41EA03418E452CD9CA
:10118000691808F1FF3304D28E4502D9A8F1020391
:10119000294443EA0040A1EB0E01A0FB029841451F
:1011A000CE46434602D306D14C4504D20138B9EBB2
:1011B000020E68EB0503002EA5D0B4EB0E0261EB26
:1011C000030101FA0CFC22FA07F3F9404CEA03038D
:1011D000C6E9003197E74046C5E74346D9E7000036
:1011E0000022F0B5114640F6034085B007F01EFE20
:1011F0000446002856D107F091F8214641F2030039
:1012000003AA07F013FE044600284BD1039A274D8A
:10121000D16805F12C03D1F80100D1F8051003C302
:10122000104604F031FC214641F2010003AA07F008
:10123000FDFD0446002835D10398C3685A7885F827
:1012400023205A88EA841A7985F82420B3F80720E5
:101250002A85B3F805306B8504F016FC214641F26F
:10126000020003AA07F0E2FD0446D8B9039F05F186
:101270003406FA68531C41323446186859680833FA
:1012800003C493422646F7D1384604F0FDFB95F897
:101290003030580610D40121054A06486DF0BCFCD8
:1012A0006FF01204204605B0F0BD00BF30000020F2
:1012B000D0DD0A001CF80900002142F2030003AA55
:1012C00007F0B4FD04460028ECD1039AC04BD16866
:1012D000D1F80100D1F8051003C3104604F0D4FB87
:1012E000214642F2020003AA07F0A0FD04460028AE
:1012F000D8D1039EF468B4F801309AB292B1E27882
:1013000082B1A5F8BC30E378032B06D0032202217A
:101310000092B048B04A6CF09FFAE278AF481146AC
:1013200072F004FA304604F0AFFB002142F23A00BA
:1013300003AA07F07BFD0446002840F020810398B3
:10134000C368B3F80130A5F8D83004F09DFB95F8D8
:10135000306016F0200619D14FF0FF304FF0FF310A
:1013600007F092FB0446002800F0768102210C3041
:101370006CF077FE0123214603704670324640F63A
:101380006D4007F053FD044600288BD195F850308E
:101390001A0713D5002142F21C0003AA07F046FDEC
:1013A000044600287FF47EAF0398C368D3F8012079
:1013B000D3F80530C5E9262304F066FB95F8903094
:1013C0009B0626D50DF10A0102A807F0D9FD0446B7
:1013D00000287FF467AF4FF0FF304FF0FF3107F088
:1013E00053FB0646002800F0378104210C306CF0D6
:1013F00038FEBDF8083022460380BDF80A30314679
:10140000438042F2240007F011FD044600287FF4D7
:1014100049AF95F890305F0610D5002142F22A00BE
:1014200003AA07F003FD044600287FF43BAF0398AE
:10143000C3685B7885F8DA3004F026FB4FF0FF30A4
:101440004FF0FF3107F020FB0446002800F0048134
:1014500008210C306CF005FE95F8901002466048AB
:1014600011F0020F5F4B08BF034695F891008E06FE
:1014700048BF43F0400310F0090F18BF43F4006366
:1014800001F0010143EA011000216DF0E9FB214662
:10149000002242F2010007F0C9FC044600287FF454
:1014A00001AF95F83030B5F8BC10980673D4C9B9BF
:1014B00041F2050003AA07F0B9FC044600287FF4B6
:1014C000F1AEB5F8BC30039C4BB9E368B3F801202A
:1014D000A5F8BC209A884148114672F027F92046A9
:1014E00004F0D2FA4FF0FF304FF0FF3107F0CCFAA2
:1014F0000446002800F0B08008210C306CF0B1FDEB
:1015000095F890300246D90747BF2FA1D1E90001D5
:101510004FF0005134486DF0A3FB2146002240F605
:10152000014007F083FC044600287FF4BBAE01466F
:1015300003AA4FF6014007F079FC0446002834D096
:101540002A4A022123486DF067FBEB79002B74D106
:101550006DF01FFE044600287FF4A4AE0BF054FB90
:10156000044600287FF49EAEEB79002B3FF49AAE40
:1015700008211F486DF059FB07F08AFB92E6411DD8
:101580007FF490AE02211B4A12486DF045FB1F23E9
:10159000A5F8D830DBE60029A4D10121164A0D4870
:1015A0006DF03AFB6FF004047CE6039804F06CFAEB
:1015B00021464FF6024003AA07F038FC0446F8B172
:1015C0000E4ABEE7AFF30080908800020080002042
:1015D000C00000201CF80900F4DD0A00F000002023
:1015E0000E1207002E12070010880002BADE0A0051
:1015F000B80000203ADE0A0097DE0A00DEDE0A00AC
:101600000398C368B3F80130A5F8753004F03CFACC
:1016100095F875305A0798D521464FF6034003AA2E
:1016200007F004FC08B11A4A8BE70398C3685B789B
:1016300085F8743004F028FA87E72E78002E87D1D9
:1016400095F875309B061FD54FF0FF304FF0FF31F6
:1016500007F01AFA044610B96FF0680422E6062172
:101660000C306CF0FEFCD5F8013021460360094BCC
:1016700032469B8883804FF6064007F0D7FB04462E
:1016800000283FF465AF0DE66FF085040AE600BF61
:1016900007DF0A00310000204FF0FF329FED0A7B88
:1016A0000D4B00211A6000200C4B002283ED007BC3
:1016B0009FED077B0A4BC3E900010A490A4B81ED04
:1016C000007B1A6014F0AEBFFFFFFFFFFF1F00009A
:1016D0001F000000000000005C510020B00100204D
:1016E000182B0020A8010020545100200000000009
:1016F0002DE9F047044640F2712690F85E3090F8EC
:10170000382023F00103C3F3800060F386128CB00D
:1017100004F1460184F85E3084F8382013F008FDA7
:10172000B4F84C300022A3FB0663636D484D23657B
:1017300003F5D673B34228BF33464649A4EB0505EB
:10174000A1FB051594F83810C5F3871501F0790150
:10175000DFF81091C4E90222227032BF6360666034
:10176000226584F8381005EB4502246149F82230DF
:1017700013F08AFC63694FEA450A00F5D677002B1F
:101780004BD00DF12C089121AA4409EB8A034FF0AC
:1017900000094FF0020A0993CDF820800694B4F8AE
:1017A0004C302D4A2D480792A3FB000201FB032178
:1017B0002B4BCDF80C9005936368CDF82CA00493C7
:1017C00021A3D3E90023FFF779FB104619464FF414
:1017D0007A720023FFF772FB0535EDB20321CDE9E4
:1017E00001603B462A464846CDF8009013F0D2FAF5
:1017F000414614F0ADFA60B994F85E3043EA0A034A
:1018000084F85E3018F0BEF9B8B100200CB0BDE825
:10181000F0870C200CB0BDE8F0870DF12C08CDE965
:101820000A330320434661680AAA21F0D5FF002845
:10183000A9D1DDE90A371F44A5E7504622F0D8FDBB
:10184000E3E700BFAFF3008000CA9A3B000000004E
:10185000502B0020ABAAAAAAA9510200002AE784B3
:10186000C5BD0200B054002070B50D46044600F11D
:101870008F06334600223B3105F12B0029F0BAFADE
:1018800000229FED2D7BD4F89B30D4F89710C4F83C
:10189000BC30D4F8AC30D4F89300C4F8CD3094F810
:1018A000C830D4F88FC043F0010384F8C83094F8EE
:1018B000A730C4F8B810D4F8A81062F30003C4F835
:1018C000B400C4F8C9102046294684ED307BC4F822
:1018D000B0C084F89F2084F8A02084F8A12084F868
:1018E000A22084F8A32084F8A42084F8A52084F8FA
:1018F000A62084F8A7301DF0B9FF0646B8B1301D08
:101900001FF0B8FBF37931466B7320461DF0C4FF1E
:1019100020461FF0C3F840F206636B8194F88E30C6
:1019200023F0180343F0180384F88E3070BD00DEF6
:10193000E5E700BFAFF300800000000000000000FA
:1019400070B504460D461DF089FF10B90623AB7231
:1019500070BD04F18F063346002205F13B0105F10D
:101960002B0029F047FA00229FED2B7BD4F89B3007
:10197000D4F89710C4F8BC30D4F8AC30D4F8930045
:10198000C4F8CD3094F8C830D4F88FC062F30003A7
:1019900084F8C83094F8A730C4F8B810D4F8A81068
:1019A00043F00103C4F8B400C4F8C9102046294626
:1019B00084ED307BC4F8B0C084F89F2084F8A02068
:1019C00084F8A12084F8A22084F8A32084F8A4201D
:1019D00084F8A52084F8A62084F8A7301DF046FFDF
:1019E0000646A8B1301D1FF03BFBF37931466B73FF
:1019F00020461DF051FF204620F024FD4FF4C16326
:101A00006B8194F88E3043F0080384F88E3070BDFB
:101A100000DEE7E7AFF300800000000000000000F8
:101A20002DE9F04F984685B000F15803C0E9163310
:101A3000129B0026838104239FED257B073222F031
:101A4000070A0374119B01EB0A090F4680ED087B1E
:101A50004946C0E9066686608373C6730446DDF8AE
:101A600038B003F051F8109BC51D25F00705C4F8E8
:101A70008850C4E9207A02930F9BA9EB0505CDE9B4
:101A800000B32A4643463946204603F037FB0F9BF6
:101A9000C4E91B8B6367109B6665A367EFF3118234
:101AA000202383F31288BFF36F8F0B4B596A5C625C
:101AB000E16782F31188BFF36F8F9B680BB1D3F896
:101AC0008C302846C4F88C3005B0BDE8F08F00BFDC
:101AD000000000000000000044640020000000003E
:101AE00030B5144617A3D3E9002385B0FFF796F964
:101AF000054601A9284649F097FB9DF807309DF857
:101B000006201B0443EA42539DF808200C4943EA8F
:101B1000C2239DF8092025F0010543EA42139DF8F0
:101B20000A20A5FB010143EA5203BDF80420A2F2FA
:101B3000BC7243EA4263236005B030BDAFF300805E
:101B400000CA9A3B00CA9A3B000000000000000057
:101B50002DE9F0412DED028B90F8A5300446B0EE52
:101B6000408A86B01BB9F7EE007A37EEC08AD4F807
:101B700084202F4B9A4213D118EE100AFEF7E4FD91
:101B800029A3D3E90023FFF7C7F8011E18BF0121DD
:101B900004F1840034F02EF984ED268A012005E05A
:101BA000B4F89C30B3F5807F05D1002006B0BDECC1
:101BB000028BBDE8F08104F1500840464EF062FB14
:101BC0000028F2D0DFED1B7A68EE277AFCEEE77A88
:101BD000CDED037A94F8806094F89C209DF80C3049
:101BE000276E206D6EB18DF8153002238DF814200C
:101BF00000210122009305ABB84740467DF06BF908
:101C0000CAE7012531468DF813208DF814302A4695
:101C10000DF113030095B847009532462946276E0B
:101C2000206D05ABE8E700BFAE47E17A14AEEF3FA9
:101C3000807B0A0000007F432DE9F04F044685B009
:101C400008466160062190461D469DF838709DF853
:101C50003CB043F009F8A060067C16F0010602D003
:101C60007D4837F0E3FD9DF8403005FB08F084F82F
:101C70002A309DF844307D3084F828307E2390FB54
:101C8000F3F0C0010430C4E904852773606278F082
:101C900029F90DF1080A0622C4E907066F49204612
:101CA000A66183F0EEFA022251462046ADF8088084
:101CB00083F0E7FA022251462046ADF8085083F03F
:101CC000E0FAF623032269462046ADF800308DF88D
:101CD000026083F0D6FA7B1EDBB2082B05D840F2F7
:101CE0005515DD4015F0010501D15D48B9E7052F17
:101CF00009D0072F06D0032F73D1012384F8293090
:101D0000002502E02E4684F82960002646F34F1095
:101D1000C0EB0020FEF706FD0022524BFEF7B6FB9B
:101D20000022514BFEF792FEFFF700F85FFA80F8B1
:101D3000C6F38200C0EB0020FEF7F4FC00224B4B00
:101D4000FEF7A4FB00224A4BFEF780FEFEF7EEFFF3
:101D5000C7B206F00300C0EB0020FEF7E3FC002250
:101D6000404BFEF793FB00223F4BFEF76FFEFEF762
:101D7000DDFFC0B2002D5ED08DF808008DF809801F
:101D80008DF80A70032251462046013683F079FA15
:101D9000802EBBD1BBF1000F1AD0364D01A92A8885
:101DA000AB782046ADF8042003228B7083F069FAEB
:101DB0000B222046304983F064FAD5F80300EB7912
:101DC00002900522514620468AF8043083F059FAE1
:101DD000204683F044FAA06983F065FA05B0BDE8B7
:101DE000F08F092F84F829608AD10FF25C09D9E9B4
:101DF0000089354616A7D7E900672846FEF792FC0A
:101E000042464B46FEF742FB32463B46FEF71EFE7D
:101E1000FEF78CFFC0B28DF808008DF809008DF830
:101E20000A00032251462046FF3583F02AFAB5F511
:101E3000FF4FE2D1AEE78DF808808DF809708DF87C
:101E40000A009FE7AFF300800000000000C04F4091
:101E50000000000000C05F40D4570B008B3A0B001D
:101E6000F84E0B000000F83F0000084000000C4056
:101E700000001C40B2FA0900923A0B00000000007A
:101E800010EE103A33F0004210B52DED028B06D162
:101E90000120BDEC028BBDE8104069F043BC002B73
:101EA00005DABDEC028BBDE8104069F049BCB3F126
:101EB000FF4F06DB30EE008AB0EE480ABDEC028B25
:101EC00010BDB3F5000F6049BBBFDFED607A6FF066
:101ED0001802002260EE277AB8BF17EE903AF7EEAC
:101EE000007ADC15C3F316037F3C1944144401F453
:101EF000000282F07E5204EBD15403F10F011A4329
:101F000007EE102A524A0A4037EE678AB2BBB5EE96
:101F1000408AF1EE10FA0FD1002C00F08C8007EE11
:101F2000904A9FED4C0A9FED4C7AF8EEE77A27EE47
:101F3000808A07EE878ABFE741A1D1E90001FEF759
:101F40001DFFB6EE007A07EE900A07EEC87A68EE3B
:101F5000087A27EE277A14B938EE478AACE707EEFD
:101F6000904ADFED3C6AF8EEE77A07EEE67A37EE64
:101F7000488A9FED397A17EE878A9DE7F0EE007A5E
:101F80009FED365ADFED364A364A78EE277A1A4404
:101F9000C3F5571388EE276A07EE904A03F52273BC
:101FA0001343F8EEE76ADFED307A002B66EE065A4F
:101FB00025EEA57A07EE275ADFED2C7A45EE077A53
:101FC0009FED2B5A07EE875ADFED2A7A47EE274A14
:101FD000DFED297A44EE877A67EE877A45EE257A37
:101FE0001ADDB6EE007A28EE077A27EE087A77EE49
:101FF000877A67EE867A14B937EE677AACE79FED99
:10200000156A46EE867A37EE677A37EE488ADFED54
:10201000127A16EEA78A4FE778EE677A67EE867A2D
:1020200014B938EE678A47E79FED0A7A46EEC77A19
:1020300037EEC88AEBE79FED118A3DE7AFF30080EA
:10204000555555555555D53F20FB4A000000004CCD
:10205000F0FF7F00D1F717378071313F25333A3ECB
:10206000298E633E305CCFFF9788173E2549923E0C
:10207000ABAA2A3F4FD01C3ECDCCCC3E0000000086
:10208000F8B510EE904A10EE103A34F000472DEDFE
:10209000048BB0EE609A0DD183F480035B0013F5DE
:1020A000000F40F2AA8230EE098AB0EE480ABDEC79
:1020B000048BF8BD23F000411846B1F1FF4F02D860
:1020C000B7F1FF4F08D9B3F17E5FECD184F48004FF
:1020D000640014F5000FE4E7002B25DAB7F1974F01
:1020E00080F09482B7F17E5F39D3FA15C2F196027F
:1020F00047FA02F505FA02F2BA4229D105F00105C4
:10210000C5F10205B7F17E5F2AD1002C80F27B82F7
:10211000B5EE400AF1EE10FA1CD1D80FBDEC048BDD
:10212000BDE8F84069F0FEBAB7F1FF4F10D1B1F148
:102130007E5F00F0628205D9002CDFEDD17A29FEA6
:10214000278AB2E7002C80F25B82B1EE498AACE7C5
:102150000025D7E7B7EE007A87EE008AA5E70025CD
:10216000B4F1804F0A4640F05782B1F1BF4F0CD214
:10217000B1F1D05F02D920EE008A96E7B0EEC08AB6
:1021800059BB012D00FE088A8FE723F04046B0EED0
:10219000C08AB6F17E5F17D1002CBCBFB7EE007AC3
:1021A00087EE088A002B80DAA1F17E51294305D100
:1021B000BDEC048BBDE8F84069F0C2BA012D7FF494
:1021C00074AFB1EE488A70E739B9002CD9DA002B28
:1021D000A4D06B1E58425841A0E7DE0F013E55EADD
:1021E0000600E5D0B7F19A4F71D9A64B994208D8AD
:1021F000002C0BDA0020BDEC048BBDE8F84069F040
:1022000083BAA14B994208D9002CF3DC0020BDEC25
:10221000048BBDE8F84069F069BAB7EE007ADFEDEB
:102220009B7ADFED9B9A38EE478A93A1D1E90001B2
:1022300068EE278AFEF7A2FDB5EE007A07EE900A57
:10224000DFED946A68EE299A48EE477AB6EE007A96
:1022500007EEC87A68EE087A27EE277AF0EE687AF9
:1022600047EE667A39EEA77A17EE103A6FF30B0352
:1022700007EE103A77EE699A77EEE97A013DF7EECC
:10228000006ABFEE008A6FF30B04354367EE890ADC
:1022900008FE268A06EE904A39EE666A67EE267ACE
:1022A00046EE070A30EEA77A17EE101A002921F041
:1022B000004340F31381B3F1864F40F2CC80B5EE7A
:1022C000C08AF1EE10FA4CBF0120002093E713F012
:1022D000FF4F05BF9FED707A6FF01701002168EE88
:1022E000077A08BF17EE902AD315C2F316027F3B78
:1022F00042F07E500B4469498A4206DD68498A42B1
:1023000040F3A7800133A0F500000021654A06EEE6
:10231000100AF7EE006A02EB8102D2ED005A75EE68
:10232000867A36EE657AC6EEA74A27EE245A15EE6F
:10233000102A6FF30B0206EE902A5B4A02EA600253
:1023400042F0005202F5800202EB415207EE902A61
:1023500006EEE77A77EEE57ADFED545A36EE676AF5
:1023600065EE057A06EE667A9FED516A47EE865A6B
:102370009FED506A27EE247A66EEA64A05EEA76A1C
:10238000DFED4D5A46EE275A9FED4C6A05EEA76ADF
:10239000DFED4B5A46EE275A36EE856A67EEA77A8E
:1023A00026EE076A05EEA76AF0EE085A74EEA57AE3
:1023B00077EE867A17EE902A6FF30B0207EE902ADB
:1023C00077EEE55A27EE277A66EEA76A75EEE45AAD
:1023D00036EE656A06EE057A9FED3A6A76EE877A02
:1023E00017EE902A6FF30B0207EE902A364A77EE2B
:1023F000E66A02EB810227EE866A37EE667ADFED47
:10240000336A67EEA67ADFED326A47EE267A92EDFE
:10241000007A77EE877A07EE103A2E4BF8EEC76A0D
:1024200003EB810336EE277AD3ED005A37EE257A97
:1024300037EE267A17EE103A6FF30B0307EE103AD9
:1024400077EE666A76EEE56A76EEC66A77EEE67A4B
:1024500014E701215AE755D1DFED1F6A37EE677A9D
:1024600070EEA66AF4EEC76AF1EE10FA3FF727AFF6
:1024700086234BE0AFF30080E13D55555555D53FE0
:1024800000000000F3FF7F3F0700803F70A5EC369F
:1024900000AAB83F3BAAB83F0000804B71C41C00A3
:1024A000D6B35D008CBC0A0000F0FFDF55326C3EF5
:1024B00042F1533E05A38B3EABAAAA3EB76DDB3E6D
:1024C0009A99193F0040763F7CBC0A00C623F6B8B3
:1024D0004F38763F84BC0A003CAA3833534A9342B3
:1024E00007D9B5EEC08AF1EE10FA4CBF01200020EA
:1024F0008DE607D137EE677AB4EEE07AF1EE10FAA6
:10250000B6DBEEE7B3F17C5F72D9DB157E3B4FF4AF
:102510000000474A002940FA03F00844C0F3C753BB
:10252000A3F17F0342FA03F2C3F1170302EA0002A8
:10253000C0F3160040F4000007EE102A40FA03F042
:1025400077EEC77AB8BF404237EEA07ADFED396A3E
:10255000DFED395AB7EE000A9FED386A17EE103AF0
:102560006FF30B0307EE103A77EE677A67EE266A91
:1025700070EEE70ADFED327A27EE277ADFED317A67
:1025800000EEA77A76EE877A77EEE66A37EE667A1D
:1025900067EEA76A07EE877A16EEA56ADFED2A5A7C
:1025A00046EE265A9FED296A15EEA66ADFED285AF7
:1025B00046EE265AB0EE676A05EEE66AF0EE006A6D
:1025C00067EE865A36EE666AC5EE866A36EEC77ADA
:1025D00077EE677A30EE670A10EE103A03EBC053DD
:1025E000B3F5000F06DA68F005FF20EE088A5CE517
:1025F0000020A9E700EE103AF7E7B7EE008A54E5AD
:102600009FED148A51E5B0EE408A4EE5B7F1FF4FD9
:102610003FF48DAD0A460225B4F17C5F7FF4B5AD81
:10262000002BFFF6B2ADB1EEC08A3EE500001643C6
:10263000000080FF0072313F4CBB31330EEADD35C4
:102640008CBEBF351872313F55B38A38610B363BAB
:10265000ABAA2A3E0000000010EE103AB3F1FF4F83
:1026600010B52DED048BB0EE408A06DB30EE008A0B
:10267000B0EE480ABDEC048B10BD774A934276DC7D
:1026800023F00042B2F17E5F13D3FFEE007AB4EE86
:10269000670AF1EE10FA06D10120BDEC048BBDE80B
:1026A000104069F03FB8BDEC048BBDE8104069F004
:1026B00047B8B2F1645F0FD2B2F14A5F24BF20EE97
:1026C000007AF6EE007ABDEC048B28BF07EE670AAD
:1026D000BDE8104068F048BE604A134493424ED8AB
:1026E000F7EE007A38EE277A17EE103ADC157F3CC9
:1026F000002CD5BF77EE677A37EE488A78EE677A96
:1027000077EEC87A87EE879AC3F31603544A93424A
:10271000CCBF43F07C5243F07E52F7EE007AC8BF44
:10272000C3F5000307EE102AC4BF01349B1037EE37
:10273000678AF6EE008A68EE288A68EE888A002B9F
:1027400044D1B5EE408AF1EE10FA1DD1002C7AD0BA
:1027500007EE904AB0EE498A9FED427AF8EEE77AAA
:1027600007EE878A9FED407A07EE878A80E7B3F10C
:10277000B44FB5DBDC159FED3D9A7F3CC4E70123E8
:1027800000249FED3A9AD4E731A1D1E90001FEF788
:10279000F5FAB7EE007A07EE900A07EEC87A27EE50
:1027A000287A14B938EE478A62E707EE904ADFEDDF
:1027B0002D6AF8EEE77A07EEA69A37EE497A37EEF9
:1027C000488A9FED297A17EE878A51E7F0EE007A62
:1027D0009FED276A9FED277A78EE277AC8EE276A61
:1027E00066EEA67A07EE867A9FED236A07EE276AE1
:1027F0009FED227A06EE277A9FED216A07EE276A7F
:102800009FED207A06EE277A9FED1F6A07EE276A72
:10281000B0EE687A06EE277A27EE267A24B978EEAB
:10282000C78A38EE688A23E707EE904ADFED0D6A23
:10283000F8EEE77A07EEA69A39EE079A78EEC98A9B
:1028400038EEC88ABDE79FED098A11E7AFF3008033
:10285000555555555555E53FD613D43EE0096A41C7
:10286000F6043500D1F717378071313F00000000C2
:102870009788173E4FD01C3E25333A3E298E633E43
:102880002549923ECDCCCC3EABAA2A3F2DE9F84F4C
:102890000B1F884602F00701A3EB00090B3103F080
:1028A00007030B444FEAD906D40829F0070904EBC3
:1028B000D30481448368B9F802B09C4228BF1C4607
:1028C0001BF0010B054600AF16D1EA4688B06A46F8
:1028D0004A4BCDE90538032342F8103F4FF4C2516B
:1028E0005B46474801F0F0F9D5468BF31188BFF3FA
:1028F0006F8F0423184602DF3146284669F01BFB20
:10290000304435F83030C01A864217D0EA4688B0D5
:102910006A463C4BCDE90538032342F8103F0023BB
:102920004FF4C251364801F0CFF90023D54683F366
:102930001188BFF36F8F0423184602DF3146284603
:1029400069F0F9FA8442824622D026D234442846DD
:10295000224669F095FBB9F80230214643F00103A5
:10296000A9F80230284669F0E6FA261805EBC603F6
:102970005B88DB0708D43146284669F025FB3246E0
:102980002146284669F065FB2146284669F0D8FAB9
:1029900001221046BD46BDE8F88F06EB000805EBA6
:1029A000C802528812F0010225D14146284669F03A
:1029B000C2FA50448442ECD8284669F005FB4146EF
:1029C000284669F0B8FAA4EB0A0A824507D22846DD
:1029D000321969F055FB1146284669F0B1FA4246B2
:1029E0003146284669F035FBB9F8023043F001035F
:1029F000A9F80230CCE70022CBE700BFE0C60A000E
:102A0000ECF8090004C70A002DE9F84F8A4600AF28
:102A1000002974D004680E1F361BF50826F007063F
:102A200004EB0608B8F802B01BF0010B16D1E9461A
:102A300088B06A46334BCDE90531032342F8103F95
:102A40004FF4C2515B46304801F03EF9CD468BF35E
:102A50001188BFF36F8F0423184602DF29462046F2
:102A600069F069FA284434F83030C01A854217D02A
:102A7000E94688B06A46254BCDE9053A032342F87A
:102A8000103F00234FF4C2511F4801F01DF90023ED
:102A9000CD4683F31188BFF36F8F0423184602DFFE
:102AA000B8F80230294623F00103A8F80230204686
:102AB00069F041FA05EB000804EBC8035B88DA070C
:102AC00008D44146204669F07FFA4246294620460E
:102AD00069F0BFFAA65BAE1B04EBC6035B88DB079D
:102AE00009D43146204669F06FFA2A46314620461D
:102AF00069F0AFFA35462946204669F021FABD460D
:102B0000BDE8F88F2DC70A00ECF8090004C70A00D9
:102B100008B5024869F0F1FD002008BD5AC70A0057
:102B20000E4A0346904202D30D4A904211D30D4AF9
:102B300022B1934202D30C4A93420AD30B4A52B1B8
:102B40000B48834234BF01200020934238BF00204D
:102B50007047012070471046704700BF2CF40900F1
:102B6000B4710B0000000000000000000000000035
:102B7000000000002DE9F04F9BB000AF04468B46EB
:102B8000D7F890A0FA637B6349B9037846788078D8
:102B900000EB830020445E4522D8A0EB040B0AF032
:102BA000010394F80280FB62E378B8F1000F0CBFD8
:102BB0004FF000090AF001093B6313B11AF0020F4C
:102BC00017D1B9F1000F14D1FB6B1BB15946204648
:102BD0007A6B98475D4628466C37BD46BDE8F08F56
:102BE000451C2846FEF796F9013028440BF1010BED
:102BF000D1E7CAF3C003FB612378BB629B00BB61D2
:102C000063683B62BB6A04EB8301FB6B002B7DD1E5
:102C10005D468844B9F1000F1DD08B469946A94EF8
:102C20001BF8013B54F82300002808BF3046FEF78C
:102C300071F9D7F8943001304BB1D7F898304B4543
:102C400082BFD7F8943023F8190009F10109C34570
:102C50000544E5D1D8461AF0050F0CBF4FF0020B22
:102C60004FF0010B00260AF00203FB633B6B9E4210
:102C7000B1D298F8013008F1020854F823A0504668
:102C8000FFF74EFFFA69034602B3B86318F8021C57
:102C9000386A69F011FDBB6BC0B1EA468AB06A467A
:102CA000894B05933B6ACDE906314FF40073ADF8CB
:102CB0002030864B42F8103F00234FF412518448D5
:102CC00001F002F8D546023D0136CFE723B1FB6A99
:102CD0002BB9A5EB0B05F7E7FB6B002BF4D079487C
:102CE000BAF1000F18BF5046FEF714F9D7F8943028
:102CF00053B1D7F8983099453FBFD7F89420431C7B
:102D000022F8193009F101090544DDE7B9F1000F96
:102D10006DD04346102B28BF10230026BB6397F8C5
:102D2000389007F14800BA6B79628CF0A7F8796A9D
:102D300000227A620AF0020201EB08033A610AF00B
:102D400004027B61FA6002337A6A396B8A4267D384
:102D50006378F96A1AF0020F7B624B4418BF0022B5
:102D6000DBB208BF7208002940F0A9801AF0040FF6
:102D700014BF314600216370A170E27020467A6B67
:102D8000B969FB6B9847051EFFF625AFBB6A314654
:102D900023707B6A7A6B63703B6B84F80280E3700C
:102DA00007F15800FB6B9847061EC0F2C5803A6BCE
:102DB000BB69386B03EB4203ABEB0301D7E90D238F
:102DC000C91A7B6903EB4000FB6B98470028C0F2EF
:102DD000B5804FF000082E44351807F1480AC84561
:102DE00078D300217A6B0846FB6B9847F3E6B8F17D
:102DF000000F0CD01AF0040F0ED04346102B28BF42
:102E00001023BB6397F8386007F158008BE74646FC
:102E1000C146C7F838808BE74E46C7F8388087E749
:102E200013F8015C13F8021C54F82500BB60FFF78F
:102E300077FE0246F869BB6838B1386AC7E90132E3
:102E400069F03AFCD7E90132F0B912B3FA6A72B10B
:102E5000B9F10F0F18D809F1280107F1400009F165
:102E60000102014401F8205C5FFA82F90CE0FA6883
:102E700052B10F2E08D806F1280107F14000721C4C
:102E80000E1806F8105CD6B27A6A023301327A6202
:102E90005AE73A69002ADBD10F2EF5D806F128004F
:102EA00007F1400C6044721C00F8101C07F1680127
:102EB000023651FA82F2F6B202F8105CE4E7002121
:102EC00059E700BF88C70A008FC70A000400000145
:102ED00074F8090018F80A3054F823B087F847301E
:102EE000D7F8943033B3D7F89830984522D2D7F832
:102EF000943033F8186001217A6BFB6B07F14700BF
:102F0000984700281ADB0E4B0544BBF1000F08BFA1
:102F10009B4626B95846FDF7FDFF461CB6B2314622
:102F200058467A6BFB6B9847002807DB054408F18D
:102F3000010854E70026DEE735464CE605464AE63A
:102F400088C70A00014B1860704700BF4802002084
:102F5000044608B5EFF31183202383F31288BFF3EF
:102F60006F8F29F03BFC204602F064FE024869F0B6
:102F7000C4FB6AF093FFFCE743C80A002DE9F04761
:102F8000058B0446280717460CD501290CBF45F0D0
:102F9000100545F02005258387F31188BFF36F8F57
:102FA000BDE8F087022905F0070540F0948020462F
:102FB00069F0B5FE052864D801A353F820F000BFDE
:102FC000992F0100D7300100833001004530010006
:102FD0005F3001007130010001F007035A1F012A20
:102FE0001FD8002221F00701062BD4F8008089B2F7
:102FF000C4E9002209D1434603E0628B01326283B7
:103000001B68002BF9D141F002012046218369F0B1
:1030100086FE4FF0000900286DD041F02001218389
:1030200069E0042B0AD121F0070189B220462183EF
:1030300069F075FE10B141F0200121834FF00008C6
:10304000C14658E02369D3F80090238B23F007038F
:1030500043F006034FF00008238346464BE0236904
:10306000D3F80490238B23F0070343F00403F1E724
:103070002369D3F80890238B23F0070343F005035B
:10308000E8E74FF00008C146E7E7012243F00803F4
:10309000238387F31188BFF36F8F002A3BD1B8F1E8
:1030A000000F4AD1B9F1000F02D020462C49C84781
:1030B000EFF31187202383F31288BFF36F8F238BE5
:1030C00023F008039BB22383D9063FD523F01002D7
:1030D000228303F007056669218B002EBFF67CAFC3
:1030E00000239946D4F8008021F00701C4E9003399
:1030F00041F001012183238B03F0070AAA4502D086
:10310000A268002AC1D1B8F1000F02D1B9F1000FB5
:10311000DAD00022BAE7A1680029C0D00D680029E2
:10312000BDD03346524620464F68B8471DB12B6884
:1031300029461D46F3E72B46FAE7414633465246F9
:103140002046D8F8008069F016FEA8E79A067FF5B9
:1031500023AF23F02002228303F0070527E700BFF7
:10316000A3CD070037B504460821C06A6AF0B6F857
:1031700000234FF6FF72104DADF804306368ADF8D0
:1031800000208DF80620E26819182B401344181A05
:1031900060606846ADF8021069F0F4FF69462046A9
:1031A0006AF0BBF82046211D69F0C6FF63682B401A
:1031B000A36003B030BD00BF0000FFFF2DE9F7435F
:1031C0000F4681460821C06A6AF088F880463C684C
:1031D000124D241A3C6004EA0506B4421CD3A0B286
:1031E00010B903B0BDE8F08308236A46214648467B
:1031F00069F069FF0028F4D16946A0B26AF05AF874
:1032000038B1BDF80230BDF804202E4013441E44EE
:103210003C60A4EB0804E0E70020E2E70000FFFFC9
:103220002DE9F04704468AB000F11407384670F0E3
:1032300089F9A06A83681B699847E06248B9A84980
:10324000A8486AF033F86FF0150528460AB0BDE8C3
:10325000F087A06A83681B6998470368013B1F2BAE
:1032600001D9A149ECE7E368B3F5803F08D94FF4F1
:103270008032012100929B489C4A6AF0EDFAE2E715
:10328000A06A216807AA6EF0E1FC08B19849D7E767
:10329000E5682DB1089BB5FBF3F203FB12550DB1A8
:1032A0009449CDE7238A012B01D89349C8E7E36A03
:1032B000029593F805804FF0FF334FF0FF32384608
:1032C0002BF080FA0821E06A6AF008F8A946064661
:1032D000238A1FFA85FA534544D8238A4B4500F0C8
:1032E0000F8153450BD10299082342462046891B82
:1032F00069F0F7FE18B9204602A969F01DFF2046C3
:1033000002A9FFF75BFF0546002840F0FB80029909
:103310004FEA11494FEA09496160C4F80890A3686F
:103320008B420DD80823204603AA69F0CCFEB8B919
:1033300003AB13F8012B904532D101300828F8D1A6
:10334000636820466FF30F0302A9029369F0F4FE4D
:1033500042462046E368029969F0C3FE00283CDA41
:103360000546CFE0E1682B04891B13FA81F1424640
:1033700008232046029169F0B4FE78B1204602A9E4
:1033800069F0DAFE09F10109082342462046029954
:103390001FFA89F969F0A5FE00289ED0013597E74C
:1033A000A08803A969F086FF626810B9911B61606B
:1033B000B5E7BDF810A0BDF80E10E06AC4F808909B
:1033C000514469F08BFF48448242A060EED1BAF1CB
:1033D000000FEBD06FF01C0594E05DD04FF6FF7945
:1033E000636806EB0308E3681FFA88F29B1B9A42A6
:1033F000CDF808801CD34FF000086168B8F1000FC9
:1034000030D06FF30F012046029102A969F094FEBB
:103410002046029969F09DFE0028A1D1E368A288A8
:10342000A3EB46039A426DD1204669F093FF97E7DC
:1034300008234146204605AA69F045FE00288FD1A1
:1034400005A91FFA88F069F035FF30B1BDF81430D6
:103450004B4502D1BDF818300BB1B044C3E74FF073
:103460000108CAE7204669F074FE00287FF478AFAF
:103470006368224AE16813400B44A3EB4603636090
:10348000134041462046A36069F0E8FFC4E7E26AC2
:10349000A36812681344A360D4E901318B4208D9B0
:1034A000424620465B1A69F01CFE0028FFF658AF22
:1034B000EDD16168E36801EB46029A42AED10F4B51
:1034C000A06801EA03029042A8D0204669F041FEBC
:1034D00000287FF445AF6268084B1A40A2609DE760
:1034E0008BC80A009CF80900ADC80A00CAC80A00C7
:1034F000F3C80A000BC90A001FC90A000000FFFF39
:103500006FF02C0538462BF0CFF9002D7FF49DAEDF
:103510000123A37499E600BF2DE9F04F1E46837C7A
:1035200004468946904695B04BB96A496A4869F0A5
:10353000BDFE6FF00C05284615B0BDE8F08FC26ADD
:103540000821104669F0CAFEB1B20190104669F038
:10355000C5FEE368019A0746A3EB82038342C0F0ED
:10356000B6801EB1B8F1000F00F0B180D4F804A00D
:10357000CDF810A0204605AA04A969F025FF05464C
:103580000028D8D1BDF814304B4507D0DDF810A085
:1035900063685345EED1002E39D1CCE705A91FFA57
:1035A0008AF069F087FE0028F0D0BDF8183066B3C5
:1035B000B3422CD1B3464FEA1A43BDF816A01B0400
:1035C0009A44E36ACDF800801B685B4203F0200355
:1035D0000293029B51465B4528BF5B4620460CAADE
:1035E000039369F070FD00284DD1039B00981A46A3
:1035F0000CA98BF071FC50B9039B009ABBEB030B39
:103600001A449A440092E4D195E7002B93D0002FFE
:103610003CD1BA4604F1140B4FF0FF324FF0FF33A8
:1036200058462BF0CFF8238A9D424DD0D4E9013281
:103630000AEB02018B422ED39BB263B3FF2300211E
:10364000ADF81E200CA818228DF82230ADF81C9081
:10365000ADF820608BF038FC20460CA9CDE90E8631
:1036600069F046FE074648B907A869F08BFD204679
:1036700007A969F052FE074600B9374658462BF0B5
:1036800013F93D4657E7C2DC054654E7019B1F444A
:103690001FFA87FABEE72046FFF764FD3DB9ADF893
:1036A0002490CDF82880ADF82C608DF82E5020465F
:1036B00009A969F0D3FE07460028DFD19DF82E3016
:1036C0000135002BAFD0D8E76FF01B07D6E76FF0BE
:1036D000150530E777C80A009CF809002DE9FF4777
:1036E0001E46837C04460F469046BDF8309043B991
:1036F0002748284969F0DAFD6FF00C0004B0BDE8F6
:10370000F0870821C06A69F0E9FDE368A3EB400394
:10371000B3423AD34FF0000A65680195204602AAE9
:1037200001A969F051FE0028E8D1BDF80830BB427C
:1037300006D102A9A8B269F0BDFD50441FFA80FA73
:10374000019B62689A4219D0CA4515D9BDF80C3060
:10375000C3B1CA4516D3BDF80A10B3426FF30F05C3
:1037600028BF334642462046294469F0ACFC002875
:10377000C4D1BDF80C00C1E71D46CFE7BDF8083045
:10378000BB42E3D06FF00100B8E76FF01500B5E77A
:103790009CF8090077C80A002DE9F047044607465F
:1037A0004FF00109DFF84C8094FAA4F5B5FA85F5DD
:1037B00009FA05F32E0108EB05156FEA030A24EA5E
:1037C00003042B7B63B158F806301B696BB9464480
:1037D000736802222846196807EA0A0769F0B9FFE8
:1037E000002CE1D13846BDE8F087284698470028EC
:1037F000F6D1ECE784F9090010B5002288B00E4933
:103800000E4870F09BFA002200230024CDE9062325
:103810000E234FF44072CDE90334CDE90144084B47
:103820000849009408482BF01FFC0849064870F02E
:10383000E0F8204608B010BD51380100A820002053
:10384000713B0100688E0020C01B002049C90A009E
:1038500001482BF0AFB800BF641600202DE9F047F7
:10386000804621480F4669F058FF0646002833D0AD
:1038700000252846BDE8F087237B83B12368DB68F9
:103880000BB120469847636883F8069023681B694C
:10389000D3B9636802222046196869F05AFF0136DD
:1038A00010345445E8D3B8F1000FE2D0002DDFD03A
:1038B0002846FFF771FF0546002FF7D0002140F2A0
:1038C000391070F098F9F1E7204698470028E0D0C9
:1038D00009FA06F31D43E2E705464FF00109034CE0
:1038E000DFF80CA0DDE700BF5836002084F909009E
:1038F00094F90900014B53F820007047ACFD090012
:1039000008B5034608462BB1044A136000F04CFC8E
:10391000002008BD6FF01500FBE700BF4C0200203F
:1039200010B5044C237813B903482BF043F8012356
:10393000237010BDD68700206416002010B5044601
:10394000094869F0EAFE3CB1084BD3E8EF1F0139A2
:10395000C3E8E21F002AF8D105482CF0A7F9BDE81A
:10396000104004482BF026B8503600205436002072
:10397000A8200020641600200022044BD3E8EF0F9B
:10398000C3E8E12F0029F9D1704700BF503600206D
:1039900070B5FFF7F1FF0546074C084EB44200D35F
:1039A00070BD63685B792BB123685B6813B12946EE
:1039B000204698471034F1E784F9090094F909008A
:1039C00010B5044C0449204668F0B2FF034B1C605C
:1039D00010BD00BF1415002098FD090048360020D6
:1039E00000230D4A10B513700C4A0D4913600D4A9F
:1039F0000D481360FFF784FFFFF7E2FF0B4B0C4904
:103A000018468B4200D310BD1A1A5C68121101329D
:103A100022711033F5E700BFD78700205036002011
:103A200040420F005436002017D7070084F90900E0
:103A300094F90900014647F612220023014868F074
:103A400098BF00BF14150020014869F02EB800BFD0
:103A500014150020024B0146186869F081B800BFB8
:103A600048360020014869F0B6B800BF14150020A0
:103A7000F8B5284B1B78002B4AD0FFF7E5FF04462A
:103A8000002842D1244B254D1B68002B19DD70F016
:103A90000DF94FF47A76A0FB060747F612220023B1
:103AA00006FB0171FDF70AFAD5E90032C01A40F2AF
:103AB000E93361EB0201984271F1000101D3FFF794
:103AC00067FFD5E9003213F57A7342F10002C5E9C8
:103AD0000032ECB1BDE8F840FFF7C4BF6B685B791A
:103AE00023B12B68214628461B6898471035B542FC
:103AF000F4D32046FFF7AEFF094BD3E8EF1F01399F
:103B0000C3E8E21F002ABDD0F7E7064D064EEEE7F8
:103B10000020F8BDD687002050360020A0200020CD
:103B20005436002084F9090094F9090070B50D4D50
:103B3000297861B90120FFF791FE0B4C0B4EB4427E
:103B400006D3FFF795FF0028FBD101232B7070BD32
:103B500063685B791BB1236820469B6898471034E3
:103B6000EDE700BFD787002084F9090094F9090028
:103B700000212DE9F8430846FFF770FE044648B3DC
:103B800040F21B684FF0000901F0C8FB1A4B1B4ABA
:103B90001B58136033B11A4B1B68092B02DD1948FF
:103BA0002AF008FF0025184F44B12046FFF7F4FD26
:103BB000044618B94FF0FF384FF0FF39FFF758FFB0
:103BC000064628B9B5B90F4842464B462AF02EFFA3
:103BD0003546E9E74FF0FF384FF0FF39D4E72B685F
:103BE0009B691BB100222846114698471035BD42FB
:103BF000F5D3E8E7054DFAE7080000004C36002051
:103C0000543600206416002094F9090084F9090054
:103C100013B5184869F081FD174B1B7873B1EFF3AA
:103C20001184202383F31288BFF36F8FFFF720FFE7
:103C300084F31188BFF36F8F02B010BD0F4B1B6868
:103C4000002BF9D050B9002200230D48CDE9002304
:103C500047F6122200232CF003F8EDE70928EBD1F8
:103C600007482CF023F8074802B0BDE810402AF0BE
:103C7000A1BE00BF54360020D78700204C3600205C
:103C8000A82000206416002010B5064B04461B68CF
:103C900098472146A060044868F0E8FEBDE810405F
:103CA000FFF7B6BF4C02002014150020044A054B54
:103CB0009B1AB1EBD30F34BF52F83100002070478C
:103CC000B4F7090084F909002DE9F04F8FB0C1F372
:103CD0004A2604AF0D469046B8607B600C0D002E5E
:103CE00061D04FF000090A234FF0040B07F1140ACA
:103CF000FE60C7E90799C7F824900093CDF808B093
:103D0000CDF804A007F11C034A464046F968FEF7C7
:103D100031FFB0F5006F03461CD36C468AB0D8F86B
:103D2000041004AB24481A46C3E9050140F2FF71B0
:103D3000D9614FF400711984204B42F8103F4FF4C1
:103D400012514B461E48FFF7BFFFA5462C37BD4614
:103D5000BDE8F08FC0F30A0604F11700184420F004
:103D6000070080083B60FFF765FE66F353250446B5
:103D700080B13B6800F11001C7E908390A23F961F5
:103D8000CDE901AB009340460E4AF96807F11C03E8
:103D9000FEF7F0FE66F353252A4620467B68B96895
:103DA00069F0F7FCD2E704F1170020F00700800863
:103DB000FFF740FE0446EDE75EC90A00040000017B
:103DC000B4F8090065D707002DE9F04F87B0054624
:103DD000DDE9106BDDE9127A884614469946BFB1D9
:103DE00010213B465A460020CDF800A0CDF814A083
:103DF00068F089FAB0F5006F01460BD340F2FF730B
:103E00000221184A184807B0BDE8F04F69F01ABD02
:103E10003946384604F0070305F00704E40044EA95
:103E2000831444EA402444EA065406F11700084487
:103E300020F0070080080391FFF7FCFD054640B124
:103E40003FB13B465A460399CDF800A0103068F0C8
:103E50005AFA4B4622464146284607B0BDE8F04F85
:103E600069F097BC9DC90A00B4F80900406820B108
:103E7000034BC01A40F3CF0070474FF0FF3070473C
:103E8000B4F709000EB403B503AB53F8042B014695
:103E90000448019301F076FC02B05DF804EB03B036
:103EA000704700BFA7D80700CA0605D48B064CBFD1
:103EB00002490349FFF7E6BF704700BF56050B00F4
:103EC000B7010B002DE9F04F8BB099469DF8588053
:103ED000179B044607930D46DDE918A31A9F069227
:103EE0000593B8F1000F00F0BC80834B07F0020B84
:103EF00013F80830089307F48073099369F027FCDE
:103F0000024600287AD020467C49FFF7BBFF0646D0
:103F1000BBF1000F08D017F0440F71D12A4620469C
:103F20007749FFF7AFFF064407F0010353B1754B24
:103F3000204653F82820744B7449002A08BF1A46BB
:103F4000FFF7A0FF07F48073002B07F0080318BFEA
:103F50004FF00009002B7FD06D4B204653F82820EE
:103F60006C49FFF78FFF0546069B2BB11A4620468A
:103F70006949FFF787FF0544B9F1000F0DD0089B91
:103F8000002B6CD06549664BB8F1040F18BF194679
:103F90004A462046FFF776FF054462483544079BB2
:103FA0001BB12246604968F056FB059B002B00F0D0
:103FB0008E80059B3946102B28BF1023204699463A
:103FC0000026FFF771FFB54252DC0026334620463B
:103FD0001AF803205549FFF755FF0136102E4DD032
:103FE000710703D120465249FFF74CFF4E45334637
:103FF000EDD320464F49FFF745FFEEE7064687E73A
:104000004D4B186800288ED04C4B4FF47A7B1B68C0
:104010004FF03C0CB5FBF3F5B5FBF0F14FF46163E9
:1040200000FB11550BFB05F5B1FBF3F2B5FBF0FE00
:1040300003FB121100FB1E55B1FBFCF30BFB05F556
:10404000B5FBF0F50CFB131120460091CDE901E51D
:104050003B49FFF717FF66E707F0080584E730499B
:1040600096E7B9F1010F45460CBF2E48354896E753
:1040700020462F49FFF706FF0136A4E70026204619
:104080003149FFF7FFFE33461AF803202046A2F11C
:1040900020035F2B28BF2E222C49FFF7F3FE0136A9
:1040A000102E0DD0720703D120462149FFF7EAFEFA
:1040B000B1453346E8D820461D49FFF7E3FEEEE759
:1040C000059BCA44B3EB090305937FF472AFB8F1C3
:1040D000000F0AD0FB0704D520460B4A0B49FFF717
:1040E000D1FE39462046FFF7DFFE20460BB0BDE883
:1040F000F04F69F0CBBB00BF163C0B00E3C90A00D0
:10410000E7C90A00BCFD0900D5C90A007A050B0001
:10411000D0FD09000DCA0A0013CA0A00DAC90A0054
:10412000DEC90A00A7D807008557010017CA0A0090
:10413000453B0B00433B0B00603600205C36002003
:10414000F1C90A00D5D807001DCA0A0093050B0063
:1041500042F20F7373B58B4228BF0B4605680446C5
:10416000052168460D4A63F0C1FF0646636828468C
:104170000B225B680A4969F07BFB6368324669463B
:1041800028465B6869F074FB63681B2228465B68FD
:10419000044969F06DFB02B070BD00BF7B3A0B00B3
:1041A0000A3C0B00EE3B0B0000210123064A904223
:1041B00006D8064A01B901231360054B1860704701
:1041C000012140085B00F2E740420F005C3600200E
:1041D00060360020F8B50D460446064F4618B44236
:1041E00001D12846F8BD14F8011BBB6801485B6883
:1041F0009847F4E770F50900014B03600020704711
:1042000018FE09002DE9F34205460E4600244FF042
:104210001409084B084F1B680193019BA34202DC61
:1042200002B0BDE8F0823868314609FB0400A847B7
:104230000134F2E718FE09005802002070B5104B57
:104240000D461C68B4B10F4B196800238B4202DB8A
:104250006FF0010070BD224612F8146B864202D046
:1042600014460133F2E7E0686FF02DF828B1002022
:104270002C60EFE76FF00C00ECE76FF01200E9E75D
:104280005802002018FE090010B5436888B0029358
:1042900083680C46CDE9033200230A68C068CDE983
:1042A0000623054901AA05936DF0EDFC079808B9AE
:1042B000059B236008B010BD67DA070010B54FF406
:1042C0002814DFF820C086B0CDE904C40824029485
:1042D00004AC0194BDF8204000946CF02DFB06B0B6
:1042E00010BD00BF180028002DE9F8430646FCF772
:1042F00011FE0546EFF31188202383F31288BFF3E4
:104300006F8F114B1C68D3F804909C4208BF0024A7
:1043100034B988F31188BFF36F8F2046BDE8F88366
:10432000A7683846FCF7F6FDA84206D12A4639466A
:1043300030468AF0EEFD0028EBD04C4501D02468D1
:10434000E6E70024E5E700BF740200202DE9F04114
:104350000E461546FFF7C8FF044628B3C3681BB3D3
:104360005F690FB3062E07D0072E20D02A463146AC
:104370003B46BDE8F0411847838A3BB92A4631469F
:10438000B84750B9A38A0133A38206E04FF6FF7203
:10439000934204D00133A3820020BDE8F0810121C3
:1043A000114A124869F045FA6FF01500F5E745B17A
:1043B0002A7832B10022828231462A465B699847C8
:1043C000EAE7A38A012B08D12A4607212046B847ED
:1043D0000028E2D1A38A013BD6E70BB1013BDAE723
:1043E0000221034ADDE700BF69CA0A0084F8090018
:1043F0008BCA0A002DE9F0410C4B05461C680E469D
:1044000017467CB100F06AF963682046D3F8108043
:1044100032463B462946C047044600F069F920462B
:10442000BDE8F0816FF00104F9E700BF903600208D
:1044300000230360044B5A6812B9C3E900007047B7
:1044400010605860704700BF94360020014B186020
:10445000704700BF90360020002330B585B0CDE90D
:1044600002330546019000F039F9094B1C6844B944
:10447000284600F0D5F8044600F03AF9204605B089
:1044800030BD636820461B6801A998472468EEE7A1
:10449000943600201FB5CDE90101039200F01EF90A
:1044A000074B1C6824B900F023F9204604B010BD66
:1044B000636820461B6801A998472468F2E700BF9B
:1044C000943600200022024BC3E90022704700BF4F
:1044D000943600200022024BC3E90022FFF7F2BF0E
:1044E0009C3600202DE9F74307460C4609B100230E
:1044F0000B6000261E4DDFF880904D450FD31D4BFD
:104500001D6885B355F8188C3846414601AA183DF8
:1045100069F08FFB10B3D6B914BB2E461EE0D5F858
:1045200000803846414601AA69F083FB50B116B9B4
:1045300054B92E4606E000224046316869F079FB06
:104540000028F5D11835D8E7019B2360F1E7002258
:104550004046316869F06DFB0028DDD1AD69D0E7D8
:10456000019B2360D9E7304603B0BDE8F08300BF6C
:1045700094F909009C36002024FA09002DE9F0473F
:1045800084B002AFD7F8289004460D4616469846E8
:104590007860B9F1000F07D0D9F8001031BBD9F815
:1045A00004A0BAF1000F28D12046391DFFF79AFF69
:1045B00008B3D0F80C904346324629467868C8477D
:1045C000C8B16D468AB002AA124BD061C2E9053467
:1045D0004FF400731384104B42F8103F00234FF444
:1045E00011510E48FFF770FBAD4604E03A1D69F02B
:1045F00020FB0028D3D1002007E0D9F8083032464C
:104600000093294643467868D0470837BD46BDE841
:10461000F08700BFAECA0A0004000001F4F80900E8
:104620002DE9F04780464FF000470026DFF8A490C0
:10463000DFF8A4A03D46264C4C450DD3DAF80040E7
:10464000002C40D0183CB8F1000F24D1226952BB95
:10465000A469F5E72F46EDE7B8F1000F03D1226911
:104660004AB91834E8E700224146206869F0E1FAC7
:104670000028F4D1F5E76368BB4206DDAF4202D003
:10468000AB42A8BF2B461D46EBE7EAD19047002E70
:1046900008BF0646E5E700224146206869F0C9FAEE
:1046A0000028D3D1D4E76368BB4206DDAF4202D015
:1046B000AB42A8BF2B461D46CAE7C9D19047002E82
:1046C00008BF0646C4E7AF42C4D13046BDE8F08714
:1046D00094F9090024FA09009C3600204FF0FF32BB
:1046E0004FF0FF3301482AF06DB800BFF0150020ED
:1046F00001482AF0D9B800BFF015002038B5094D9F
:10470000FFF7ECFF2B785BB9FFF7E4FE00F06AF8E7
:10471000044608B901232B70FFF7EAFF204638BD95
:104720000024F9E7D98700202DE9F04306460F461B
:10473000048F99B00134A4B200F10808651EADB22F
:10474000B5F5004F4AD04A23294605AA404668F0ED
:10475000C9FF04F57F543F34A4B2814621460123AA
:1047600040460DF10B0268F0BDFFB9F1000F0146A4
:1047700010DC002810DC338FAB4209D132466B1EAF
:1047800022F8383F4FF4004102234046FEF7C4FEB2
:104790002C46D3E7002808DC2946404668F09EFFF7
:1047A0002146404668F09AFFE5E7B9F1490FEFD896
:1047B00009F160030DEB03090023094A09F84C3C99
:1047C00005A8009703ABCDF80C80ADF81040FFF7BB
:1047D000D5FE0028DCD019B0BDE8F0830020FAE750
:1047E000A3DC07007FB50123694603200193FFF78F
:1047F00025FD044668BB032002AA01A969F055F90A
:10480000044610B110F10C0F23D10399B1F5803F8C
:1048100024D200231846009A9468084484421BD38B
:104820000133B3F5807FF8D10E4D69612B83536856
:104830002846AB60D368EB6369F0CBFA044640B915
:10484000094E28466E60FFF7F3FD28466E60FFF7BD
:10485000FDFD204604B070BD9BB2E5E76FF020047B
:10486000F7E700BFA4360020F8FE09002DE9F04F5D
:104870008BB09146D0F808A01E4600AFDAF8103091
:1048800080460D469847B9F1000F05DA2B4A012101
:104890002B4868F0CEFF0AE0036846EA09045A1E76
:1048A00014400BD00121274A254868F0CBFF6FF058
:1048B000150528462C37BD46BDE8F08FDAF80CB058
:1048C000BBF1000F06D0294633464A464046D8473A
:1048D0000546EEE7202B01D91B4AD8E729462022BE
:1048E00007F108008AF0F0FA2546A642E1D9331B09
:1048F000202B28BF202309EB040BDAF8045059467B
:10490000404607F108027B60A847051E7B6812DA63
:104910006C4688B06A460D4BCDF81CB0CDE9053821
:10492000042342F8103F00234FF401510448FFF7DD
:10493000CBF9A546BDE71C44D7E700BFD3CA0A00A0
:104940008CF80900F0CA0A0022CB0A0048CB0A0002
:1049500080B505460E46174698462AF0A5FE034642
:1049600000F0DCFC0446DFF81890424649F80030BD
:1049700039463046A84754F8090000F045FC00BF0E
:104980000800000008B50348034A0021121A69F024
:104990005CFA08BD80180020688E0020074808B522
:1049A000074A0849121A69F052FABDE80840064859
:1049B000064A0749121A69F04ABA00BF00000020EF
:1049C00074180020B4710B000000002000000020CB
:1049D000B4710B002DE9F84F80460C4600AF00295A
:1049E0006AD0D1E90012E9468AB0A3686D464FF05B
:1049F000050A6E463948CDE90723CDE9050146F899
:104A000010AF002332464FF421513548FFF75CF9CF
:104A1000D4E90312CD466369AD463248C5E90723A0
:104A2000C5E90501C5F810A0002332464FF4215115
:104A30002B48FFF749F9CD46E36901212A4A284866
:104A400068F000FF0121294A254868F0F2FE264659
:104A500000254FF00A0ADFF8A4B0E946D6E908C0FD
:104A6000D6E90A138EB06A46CDF81CC005F1010CD8
:104A7000CDE908C0A81CCDE90A01E91CCDE905B5BE
:104A8000CDE90C1342F810AF002345F24001144861
:104A90000435FFF719F9102DCD4606F11006DCD1CB
:104AA000236E0121124A0E4868F0CCFEA369012151
:104AB000104A0B4868F0C6FEB8F1010F07D1EFF3BA
:104AC00005830D4A41460648103B68F0BBFE21466F
:104AD000404629F0A7FBBD46BDE8F88F6FCB0A0022
:104AE000E4F809009ECB0A00CDCB0A00DCCB0A001B
:104AF00059CC0A0068CC0A0096CC0A0016CC0A00F1
:104B000030BFFFF7FDBF00BF2DE9F04105460B4E5A
:104B1000DFF83080324606EB0807CC1B20460849F8
:104B20008AF0ACF9A01942460021083C8AF0CCF981
:104B3000C5F8904007F10800BDE8F08100000000D2
:104B400024FA09000800000010B5244C2449254827
:104B500069F08AF9A36A99013ED52248224969F091
:104B600083F91E20A36ADA0104D51E481F4969F0A3
:104B70007BF91F20194CA36ADB0204D519481C4994
:104B800069F072F90220A36A1C0304D5154819497B
:104B900069F06AF92120114CA36A590304D5114820
:104BA000154969F061F92220A36A9A0304D50D48DA
:104BB000124969F059F92320084CA36ADB0304D594
:104BC00008480F4969F050F92420A36A6FEA0343AB
:104BD0006FEA1343A36210BD1D20C3E700ED00E0A0
:104BE000A9CC0A00E4F80900C1CC0A00D4CC0A0020
:104BF000EECC0A0018CD0A0036CD0A005BCD0A00C3
:104C000075CD0A0070B506460D46294C29492A483B
:104C100069F02AF9A36ADB0647D52748274969F0D6
:104C200023F91120A36A1C0704D52348244969F0FD
:104C30001BF912201E4CA36A990712D521491E4860
:104C400069F012F9636BA26A120609D501211E4AA6
:104C5000194868F0F7FD1EB1A36A23F08003A36230
:104C60001320134CA36ADE0704D51348174969F0D3
:104C7000FBF81420A36A9C0604D50F48144969F078
:104C8000F3F815200A4B9A6AD10658BF9A6A9A6AB5
:104C9000920642BF5A6A22F400525A629A6A42F05D
:104CA000FF029A6200232B7070BD1020BAE700BF8C
:104CB00000ED00E0A0CD0A00E4F80900B6CD0A003E
:104CC000E9CD0A00FCCD0A0014CE0A002ACE0A0063
:104CD00049CE0A0070B506460D46284C2849294899
:104CE00069F0C2F8A36AD9043CD52648264969F080
:104CF000BBF81720A36A1A0504D52248234969F096
:104D0000B3F818201D4CA36A9B0512D51D482049F5
:104D100069F0AAF8A36BA26A100409D501211D4A03
:104D2000184868F08FFD1EB1A36A23F40043A36204
:104D30001920124CA36A590504D51248164969F086
:104D400093F81A20A36ADA050ED50E48134969F0C4
:104D50008BF81B20094A936A43F47F439362002334
:104D60002B7070BD1620C5E7A36A9B04F2D50548D9
:104D70000B4969F079F81C20ECE700BF00ED00E07A
:104D800078CE0A00E4F809008ECE0A00E9CD0A00C8
:104D90009FCE0A00B8CE0A00CDCE0A00E8CE0A00A7
:104DA00049CE0A00F0B59DB0664B0546586800260E
:104DB00000AFC0F3080386F31188BFF36F8F02F0D2
:104DC0007F44B4F17F4F07D102F00C04082C0ED1C0
:104DD0005D495E4869F048F85D495C4869F044F80F
:104DE00000210846FFF7F6FD7437BD46F0BD1407F5
:104DF0004CBF0D460126002DEED00022FA71DA1EBE
:104E0000092A7ED8DFE802F0057578717D7D7D7D09
:104E10007D7B50494D4869F027F80023494CFB71D0
:104E2000E36A9A0705D54C49484869F01DF8002403
:104E30002DE0E36A002B01DA4849F5E7E36A5B00FD
:104E4000F5D54749414869F00FF86369AA6943F409
:104E500080736361BFF34F8FBFF36F8F32F8023CF3
:104E6000626922F480726261BFF34F8FBFF36F8F6C
:104E700003F47F42B2F55F4F21D1DBB2022B1ED18A
:104E80002B680121374A314868F0DCFC2C68FB793B
:104E9000002BA9D16822294607F1080089F0EEFF0E
:104EA0007B6A002E4AD0C3F3080222B96FEA53236B
:104EB0006FEA43237B62204607F1080192E7214B0A
:104EC0009A6AD2B222B10120F91DFFF79BFE0EE0D3
:104ED0009A6A12F47F4F04D00120F91DFFF7FAFE01
:104EE00005E09B6AB3F5803FA1D3FFF72DFE044692
:104EF000CDE70020F91DE8E70020F91DEEE71A498B
:104F000092E71A4A6C4610F4F87F8AB0184918BF25
:104F100011466A46103B07934FF400731548ADF8ED
:104F20002030154BCDE9050142F8103F00234FF426
:104F300011510648FEF7C8FEA54678E76FF308034F
:104F4000B8E700BF00ED00E02ECF0A00E4F809004A
:104F500059CF0A0095CF0A00ACCF0A00CDCF0A0086
:104F6000DBCF0A00FACF0A0016D00A0015CF0A00DC
:104F700000CF0A003AD00A0004000001064B5A692B
:104F800042F010025A615A6942F480625A615A69C9
:104F900022F008025A61704700ED00E0EFF308804C
:104FA000EFF3098101B57246FFF7FCFE01BD00BFBA
:104FB0000B4880F3088827F0A7FC202080F3118895
:104FC00008484FF40061401880F30988EFF314801B
:104FD0000221084380F31488BFF36F8F00F068F854
:104FE000B827012098BF00201EF0040F0CBFEFF37C
:104FF0000880EFF30980816911F8021C0229FFD0B3
:1050000001B5724668F025FF01BD00BF0028ACBFA6
:1050100000F16040064B4FEA4111C9B2ABBF00F549
:10502000614000F00F0080F800131954704700BF72
:1050300014ED00E000B2002807DB01234109034A18
:1050400000F01F00834042F82130704700E100E08B
:1050500000B200280CDB01220649430900F01F00C2
:105060008240203341F82320BFF34F8FBFF36F8F6F
:10507000704700BF00E100E0054B420953F82220D1
:10508000012300F01F0003FA00F01040704700BF3A
:1050900000E100E0044B054A23F07F039360BFF377
:1050A0004F8FBFF36F8F70470000010000ED00E0ED
:1050B00008B5FFF7EFFF104BD3F8882022F47002F9
:1050C000C3F88820D3F8882042F4A002C3F88820CF
:1050D0004FF04042C3F83422BFF34F8FBFF36F8FBE
:1050E0000023E1EE103AFFF74DFCFFF757FC00F00C
:1050F000F3F829F0C3F900BF00ED00E08189203A00
:1051000041F0020181814FF47D41C0F8DC10136051
:10511000009B08495360019B21F001019360029BB1
:105120009161D3604FF08073D36100230265C0F8B2
:105130009430704751490100104B9B6883421AD14B
:10514000EFF30580B8B9EFF31181202282F31288C2
:10515000BFF36F8F9A8922F002029A81EFF31483D2
:1051600023F0040383F31488BFF36F8F81F3118856
:10517000BFF36F8F70476FF01500704744640020D5
:105180000E461546002300B5E1EE103AEFF3148306
:1051900023F0040383F31488BFF36F8FBFF36F8F83
:1051A0000C4BD0F8902098600B4B1A60D0F88030F0
:1051B00083F30B882C4686F309880020034B98471D
:1051C0002046002100220023014C20478FDE0700EB
:1051D0005149010044640020E43600201022014BB4
:1051E0001A61704700ED00E0054B9A699B689A428E
:1051F0001FBF044A536843F080535360704700BF99
:105200004464002000ED00E0084B9B6883420BD112
:10521000EFF3058343B1064B5A6842F080525A605F
:105220005A6A22F400425A626EF0E8BB44640020DD
:1052300000ED00E025498A6882F8DDE04FF030009B
:105240001044EFF3098C80E8F01F1EF0100F03D11B
:1052500002F19C0080EC108A202080F31288BFF3BA
:105260006F8F1B4F4FF000668A698A603E60D2F8EC
:105270009000184C206092F9DDE0D2F894000023F1
:10528000C2F8943080F311881EF0100F03D0002371
:10529000E1EE103A03E002F19C0090EC108AEFF38B
:1052A000148323F0040383F31488BFF36F8F02F198
:1052B000300090E8F01F8CF3098802F1000004B57B
:1052C00068F0DEFDBDE80440704700004464002043
:1052D00004ED00E0E43600200023202040F20F120D
:1052E00010B5044CE1180133934281F80003F9D161
:1052F00010BD00BF00E100E008B5EFF30583064AEA
:10530000103B02EBC30152F8330049688847BDE8FF
:105310000840FFF769BF00BF840C00200148006807
:1053200070470000E43600201FB50121094B0A4AEE
:105330000A4800F00FF90023064A0393084B0121A5
:10534000019301A8D31A029300F00EF905B05DF89D
:1053500004FB00BF000004200000002014FF09002F
:10536000801800200A7A0B6810B562F304031C460B
:10537000CB68520923F01F0343EA4203044A43F077
:105380000103C2F89800C2F89C40C2F8A03010BDDA
:1053900000ED00E010B50A4BD3F89030C3F30723BB
:1053A000013B984208D901210346064A064868F0A5
:1053B00049FA6FF0150010BDFFF7D4FFFBE700BFFF
:1053C00000ED00E051D00A00CCF809002DE9F04FC3
:1053D0008946144606464FF000084F4D85B0C84533
:1053E00027DAD6F804A0BAF1000F44D0BAF11F0FA3
:1053F00017D91AF01F0F14D1D6F800B01BF01F0FE9
:105400000FD1584668F066FD07460AEB0B000138DD
:1054100068F060FD874210D06FF015073F4A3B46A9
:1054200001E043463E4A01213E4868F00BFA6FF026
:105430001504204605B0BDE8F08F17F1160FEDD02A
:10544000BC42EBDDC5F89870D5F89C10C5F8987093
:10545000D5F8A03021F01F0143F01F0BD6E9003230
:105460001A44994202F1FF3A1AD1D34507D1314685
:10547000F8B268F038FD08F101080C36AFE73146A4
:10548000C5F89870D5F89C30E0B263F30402C5F813
:105490009C2068F028FD10F1160FC8D0441CEAE7E4
:1054A000C5F89870D5F8A020013B23F01F0302F047
:1054B0001F021343D3453146E0B2C5F8A030E8D00F
:1054C00068F011FD10F1160FB1D0C5F89870D5F83D
:1054D0009C209DF808300BF1FF3B62F304038DF82C
:1054E0000830D5F8A0309DF808205B0863F3471218
:1054F0008DF80820D6E900321344009323F01F03EF
:105500005B44A3EB0A03013023F01F036946C0B2DA
:105510000393FFF73FFFBEE700ED00E09DD00A00D8
:1055200077D00A00CCF809000522044BC3F8942078
:10553000BFF34F8FBFF36F8F704700BF00ED00E0E8
:10554000BFF35F8F0022024BC3F89420704700BF67
:1055500000ED00E010B5034C2278FFF737FF207014
:1055600010BD00BFDA8700202DE9F74F294D8A468C
:1055700006464FF00008AB46274FD0451BDAD6F859
:105580000490B9F1000F3FD031680846019168F0EE
:10559000A1FC0199044609EB0100013868F09AFC6E
:1055A00084424FF014021D4B08D002FB08F36FF049
:1055B00015024BF8032003B0BDE8F08F14F1160F6D
:1055C0002C60F8D01978A142F5DD02FB08B0C7F8CD
:1055D0009840C7F89840D7F89C4000F10801007B3C
:1055E00064F304000871D7F8A0000C79400860F358
:1055F00047140C71D7F89C1021F01F016960D7F88F
:10560000A01021F01F01296108F1010814350C36A2
:10561000B3E700BFE836002000ED00E0DA870020A5
:10562000F0B55349534DD1F890302C68C3F307239C
:105630009C4287B000F299800020FFF781FF4E4B1B
:10564000C1F8C030844216D14C4D01A82C70FEF731
:10565000D3FD002607464A4CB74213D100202B78D1
:105660004349D1F89020C2F30722934277DBFFF73A
:105670005BFF002046E0696801EB0011FFF772FE56
:105680000130DFE70199300101EB0613DA682240AF
:10569000B2F1807F52D00AD8B2F5001F34D0B2F5F3
:1056A000800F3ED0B2F5801F12D00136D4E7B2F1A0
:1056B000006F43D0B2F1805FF7D15A689B680958F8
:1056C000013B22F01F00034423F01F03012032E0BE
:1056D0005A689B680958013B22F01F0003440120CF
:1056E000844623F01F0340EA4C10CDE902218DF8D7
:1056F000100002A928780593FFF74CFE00282ADA4B
:105700006FF0150007B0F0BD5A689B680958013B5F
:1057100022F01F0003444FF0020C012023F01F036E
:10572000E1E75A689B680958013B22F01F000344D7
:10573000022023F01F034FF0000CD4E75A689B6847
:105740000958013B22F01F0003444FF0030C0120D5
:1057500023F01F03C7E72B7801332B70A5E7C1F8AF
:105760009830C1F8A00001337BE74FF0FF30C9E764
:1057700000ED00E020FF0900AAFF4400DA870020C6
:105780000000F0FFF0B587B007460E461446002132
:10579000102268461D4689F097FB02238DF80230DF
:1057A000054B2A4621466846CDE90476019362F00E
:1057B0002FFE07B0F0BD00BF1FDF070008B5024B8A
:1057C0001B689847002008BDFC360020034B044AA4
:1057D0001860937843F0020393707047FC36002002
:1057E0007C02002008B5054866F087FF002383F39C
:1057F0001188BFF36F8F0423184602DFCFD00A0051
:1058000008B50649064821F00701C1F1005202F52A
:10581000802266F037FD002008BD00BF9B5B0120A1
:10582000003700204FF0FF324FF0FF33014828F0DF
:10583000C9BF00BF8C020020014829F035B800BF65
:105840008C02002038B50546FFF7ECFF2A460821F8
:10585000074866F06EFC044628B925B1FFF75EFDE7
:105860000C22044B1A50FFF7E7FF204638BD00BF5B
:10587000003700200C00000038B504460D46FFF745
:10588000D1FF21462B460822074866F0C3FC044698
:1058900028B925B1FFF742FD0C22044B1A50FFF73F
:1058A000CBFF204638BD00BF003700200C000000B1
:1058B00010B50446FFF7B6FF21460348FDF7A4F8EC
:1058C000BDE81040FFF7B8BF0037002070B5A0FB5F
:1058D000015434B92846FFF7B5FF064640B93046B3
:1058E00070BDFFF71BFD0C22044B00261A50F6E793
:1058F0002A46214689F0E8FAF1E700BF0C000000D3
:1059000070B541690446867A0A4D59B1437ADB077E
:1059100006D42C2303FB06535B6A1B689B689847DD
:10592000002363612C20214600FB0650BDE8704037
:105930006DF0D8BED01600202C22024B02FB0030A6
:10594000704700BFD01600202C21827A054B01FB46
:1059500002339A6A1B7F801A1B3323F00303B0FBC8
:10596000F3F07047D016002038B52C24827A064B0D
:1059700004FB02335B6AD3E901240C601568FFF76E
:10598000E3FF04FB005038BDD01600202DE9F043A2
:1059900085B00546684690461C4603916EF088F92E
:1059A000DDE90067EFF31189202383F31288BFF349
:1059B0006F8F6B8B002B41D02A8B9A4225D9002206
:1059C0000023284628F0C0FF0446F0B189F311886F
:1059D000BFF36F8F039B002B41D032463B46684696
:1059E0006EF08BF92C21A27A254B204601FB023365
:1059F0005B6A03A91B681D68DDE90023A847606195
:105A000070BB2046FFF77CFF24E0698B4B1E6B8345
:105A100089F31188BFF36F8F2B7F2A8BAC6A1B33FE
:105A200023F00303521A02FB0344154B154AEB1AE9
:105A30009B105343A3722B7FE372CBE789F311884A
:105A4000BFF36F8F23464246284628F07DFF044669
:105A50000028BFD10024204605B0BDE8F083636173
:105A6000012300252381039B29466382E27A656036
:105A700004F1180089F028FA63692582E360EAE7F7
:105A8000D0160020A38B2EBAF8B500242C260F4D7B
:105A900000B9F8BD476800F10802D2E8EF3F591E8F
:105AA000C2E8EC1FBCF1000FF7D1DBB2012BF0D143
:105AB000837AC46006FB035344601B6A13B19847A2
:105AC0003846E5E7FFF71CFFFAE700BFD0160020D5
:105AD0002DE9F84F06460D4617460446A34664686E
:105AE000002CFBD14FF02C09DFF878A0BBF8103068
:105AF000BBF81220DBF81410D21ADBF80C300BF1D3
:105B00000C005B1AD21AAA4228BF2A461FFA82F852
:105B10003946424668F0ABFAB5EB080544444744C1
:105B20001DD00C9B53B1DDE90A010D9A98478346BD
:105B3000A8B10146304668F065FAD7E7B07A09FBAC
:105B400000A0436A9B6843B1AB4228BF2B4619466D
:105B5000DDE90A23FFF71AFFE9E72946F8E72046BF
:105B6000BDE8F88FD016002008B5244A244B1A60EF
:105B700025F016FA4FF47A612248D0F82436C3F3A0
:105B80000802C3F309434B4382F480721E498832F2
:105B900001FB02334FF4FA215B00B3FBF1F201FB8E
:105BA00012331A49B3F57A3F28BF0132C1F80429EC
:105BB000D0F820364FF47A60C3F30802C3F30943E8
:105BC000434342F21C5082F4807202F2172200FB1F
:105BD00002334FF47A701B0AB3FBF0F200FB12336E
:105BE0000020B3F5FA7F4FF0010328BF0132C1F85E
:105BF0001C27C1F80009C1F8003608BD0020A10724
:105C00005409002000C0FF00F82A00800000125054
:105C100048B1054B054A1B68B3FBF2F35843044BEC
:105C200043F00103184770475409002040420F0019
:105C3000E0FA0900BFF34F8F0549064BCA6802F42A
:105C4000E0621343CB60BFF34F8F00BFFDE700BF9F
:105C500000ED00E00400FA05F7B506460D461446CF
:105C6000124F38466DF02FFBE0B1BB683146384625
:105C70001B68AAB29847002802DB002003B0F0BDE1
:105C8000002CFBD1AC42F8D22F1B042F28BF0427D5
:105C90006CF0EAFD3A46019001A9301989F0EEF85E
:105CA0003C44EFE76FF01200E8E700BF54F509004D
:105CB00038B50446806F68F08DF9054668F043F901
:105CC0002046294600F06EFF044638B10448012101
:105CD000044A67F0AEFD2846FFF7D6FE204638BDE1
:105CE00034F9090006D10A0038B5802104468069DC
:105CF0006BF088FE054678B10146204600F052FF61
:105D0000044638B106480121064A67F092FD28464C
:105D1000FFF7BAFE204638BD6FF00B04FAE700BF6C
:105D200034F9090025D10A0000232DE9F04F93B082
:105D300005930B7E044633F080060F4615460AD0C5
:105D40000121AD4AAD4867F074FD6FF0040630469E
:105D500013B0BDE8F08F82B10846FFF795FE7B7E59
:105D6000DA0704D49D07F2D53B7E002BEFD1204605
:105D700013B0BDE8F04FFFF79BBF4A7E00F1280942
:105D8000900705D5802B09D13846FFF77DFEDEE769
:105D9000910700F06584002B40F06284D3071ED584
:105DA0003B8A082B12D1FA68394613680020A36297
:105DB0005368C9F8043068F037F9059080B18F480E
:105DC00001218F4A67F035FD059805E08B480121D8
:105DD0008C4A67F02EFD3846FFF756FE1EE0059709
:105DE000FFF79CFA002394F82850874A15F0600FBB
:105DF0008350C5F341131CD0032B40F09C836FF0FC
:105E00008505FFF78BFA804B1B58002B00F0CD83E4
:105E1000002D00F0958305980028DDD1484668F0F4
:105E2000C0F90346A069002B00F05584802100F0E2
:105E30005BBC484668F0B5F994F82930002840F07A
:105E40002C81013B0A2BDAD801A252F823F000BFC3
:105E50008F5F0100FF5D010015600100FF5D010023
:105E60007D5E0100FF5D0100FF5D0100FF5D01003F
:105E7000E35E0100FF5D0100575F0100A069618DD5
:105E800003697F2993F88030B9D8A28D002AB6D152
:105E9000E28D002AB3D1EE06B1D194F83020022A67
:105EA00002D14FF0FF35ACE71D070BD5C9B268F042
:105EB000AEF9054648B1638D0121544A4F4867F059
:105EC000C1FC9EE7012384F8393094F83030012B6F
:105ED00005D1638D1BB984F83030002591E701238B
:105EE000F9E7204668F01FF9628D0146FF2A86D83F
:105EF000E38D002B83D194F82830D8067FF47FAF50
:105F000094F83030002BCCD092B9618D94F83830B1
:105F10008B42E2D02046C9B200F04CFD638D0546AD
:105F200068B1012100903A4A344867F095FC68E76F
:105F30002046D2B268F0FBF90028E6D1B1E7002B89
:105F400014BF02220122052184F8302020461A467F
:105F500068F02DFBC1E705F01F05012D7FF44FAF61
:105F6000E38D002B7FF44BAF628DFF2A3FF647AFE6
:105F7000A18DFF293FF643AF94F83030022B90D12A
:105F80002046D2B2C9B268F06BFA054639E7E38D14
:105F9000A68D002B7FF433AF94F83030002B80D0E7
:105FA000012B02D1002E7FF47CAF15F01F0515D018
:105FB000022D92D1B4F82A80B8F1000F8DD1F6B23B
:105FC0003146204600F056FE421C05463FF419AF0C
:105FD00042463146204668F0EAF812E7002E7FF488
:105FE00060AF638D012B7FF478AF94F86C3066F36B
:105FF000C30384F86C3070E748D10A0034F9090013
:1060000080D10A0069D10A000C000000A2D10A0068
:10601000C4D10A00A38DE28DDEB2002A7FF4EFAE78
:10602000628D022A11D105F01F0535434FEA132175
:106030007FF4E5AE0122A06968F0C9F800287FF47A
:10604000DEAE012384F8393047E794F83010002998
:106050003FF427AF012902D1002B7FF422AF15F0C6
:106060001F050FD0022D7FF438AF002A7FF435AF23
:106070003146204600F0DCFD431C05463FF4C1AE2E
:106080000122A6E7002B7FF40CAF012A7FF425AF95
:1060900094F86C3043F00803ABE70A2B63D8DFE8D1
:1060A00013F00B00620062006200620062003A00BE
:1060B0006200150262002A02E38D022B53D194F88C
:1060C0003030002B4FD0012BA18D01D100294AD1B6
:1060D00015F01F050ED0022D17D0002602212046F4
:1060E00068F03AFA054618B131460C3067F0D0FF37
:1060F0000595F2E6002936D194F86C309E0806F03A
:106100000206C3F300131E43E8E72046C9B268F055
:1061100043FA0646E2E7668DED064FEA1623F6B22D
:1061200007D0002320460AA90A9368F089F80A9D3F
:10613000DEE7013B0E2B16D8DFE813F00F0030002E
:106140009B0015001500970097001500150015001D
:1061500015001500150015003801204667F0E3FF13
:1061600018B1012818D00025C2E7266F002EFAD0FA
:10617000B4F82E8033782046984528BF984641468B
:1061800068F0EAF905460028B2D04246314605F1EA
:106190000C0067F06CFFABE7666FE7E7204667F03F
:1061A000C2FF751C01468046EAB2204668F099F8A5
:1061B000064630B901212B46BD4ABE4867F042FB76
:1061C000D1E7D0F804B0E18DBBF802302046994207
:1061D00028BF194668F0C0F905460028C3D0038AD5
:1061E000428A4169D21AC36800F10C0A5B1AD21ABA
:1061F0009BF8003059469A4228BF1A46504667F02D
:1062000036FFD6F80CB0BBF1000F09D1298AE38D17
:1062100099427FF66DAF5046C91A67F043FF67E7B2
:10622000DBF8040083681B6B13B9DBF800B0EAE706
:10623000414698470028F8D0061F56F8041F002949
:10624000F3D008780028F0D06A8A2B8AA2EB030CDE
:106250006A69EB689B1AACEB0302904294BF02465A
:1062600092B2504667F003FFE7E7204667F05BFF16
:1062700079E732460321204667F074FF8046002804
:106280003FF471AF67F088FFE58D98F81530C0B91D
:1062900098F814608DF82930AE428DF8286028BF38
:1062A0002E46D8F8103031461B882046ADF82A30EB
:1062B00068F052F9054600283FF455AF32460AA966
:1062C00065E74FF0000A7C4A8DF81130D8F80830A5
:1062D0008DF810A01A40794B9A4256D1102106A889
:1062E00025F002FD061E37DB0AAB102E984628BFAC
:1062F0001026734806AA564503F1020335D8B600A6
:106300000236F6B28DF81060AE4228BF2E46204607
:10631000314668F021F9054600283FF424AF022EEB
:10632000B34628BF4FF0020B5A46A6EB0B06C346F6
:1063300000F10C0A504604A967F099FE730808EBB7
:106340005602934528D1F0077FF5D2AE504618F893
:10635000031067F095FECBE658367FF404AF0121B9
:10636000584A544867F065FAFDE612F8011B0AF135
:10637000010A4FEA111C01F00F0110F80CC0415C3A
:1063800003F802CC03F8011CB5E798F81460D8F8BC
:1063900010808DF81060B7E750461BF8011BCDE95F
:1063A000022367F075FEDDE90223CAE7204667F0A5
:1063B000BAFE20B101287FF4D6AE636F00E0236FF0
:1063C000002B3FF4D0AE5B88B3F5007F7FF6CBAEF9
:1063D0003D4B04F14C060A9300238DF82C30E36CFE
:1063E0009E4208BF0023BDF82A2093B1597D0F2992
:1063F00008D1197D0A44ADF82A209DF82C200132DD
:106400008DF82C20226D9A4201D01B68EBE7BDF875
:106410002A20B4F82E802046904528BF9046414659
:1064200068F09AF8054600283FF49DAE9DF82820B4
:1064300000F10C0A424528BF424650460AA967F0BF
:1064400016FE9DF82830434594BFA8EB0308A8EB3F
:106450000808B8F1000F3FF44BAED4F84CB0B34588
:106460003FF446AEBBF1000F3FF442AE9BF815304F
:106470000F2B15D19BF814205046424528BF4246A9
:10648000DBF8101067F0F3FD9BF81430434594BF20
:10649000A8EB0308A8EB0808B8F1000F3FF428AEFA
:1064A000236D5B453FF424AEDBF800B0DAE700BFB4
:1064B000E7D10A0034F9090000FF020000030200DE
:1064C0001B3C0B000DD20A00050F050094F830307C
:1064D000002B3FF448AEE18D01297FF444AE94F8DF
:1064E0003860204668F038F8054600283FF400AED2
:1064F00031460C302DE705F01F05012D7FF433AE3A
:10650000204667F002FF00283FF42DAEA38D4268BD
:10651000FF2B3FF628AE12799A42FFF424AEDAB28E
:106520000F2A3FF620AEE18D01297FF41CAE2344F3
:1065300093F83A60D5E7204605A967F081FE24E587
:106540006DF0B4FB4FF47A76A0FB060C47F61222EE
:10655000002306FB01C1FAF7B1FC654BD3E8AF1F7E
:1065600041F28732461A9642624A39D9D3E8EF6F30
:106570008E4204D1C3E8EC0FBCF1000FF6D12FD14D
:10658000D2E8EF3FC2E8E15F0029F9D123B102214F
:10659000594A5A4867F056F90221594A574867F054
:1065A00048F9FEF7BBFE574B1D58002D7FF433AC66
:1065B0007B7EE28DD9071BD5484667F0F2FDB8B95E
:1065C000BAB12946A0696BF009FA01460590002886
:1065D0003FF424AC204613B0BDE8F04F00F0E2BA1F
:1065E000D2E8EF3F0133C2E8E13F0029D9D0F7E715
:1065F0003AB92046FFF778FB00287FF40FACFFF78D
:10660000B6BB484667F0CDFD059D18B92846FFF793
:106610003BFAEEE7002D3FF401AC2946204600F09E
:10662000C1FA10B12846FFF7D7BBA069036993F8F8
:10663000801011F004017FF49AAB6BF0E3F905468A
:1066400000283FF4EBAB0146204600F0ABFA0028EF
:106650003FF48DAB01212C4A284867F0EAF8E1E7C6
:1066600052077FF5DBAB002B3FF48EAB3846FFF7CC
:106670000BFA94F83930002B3FF469AB94F82930C9
:10668000052B0CD1618DA069C9B267F0C0FD05462C
:1066900028B1638D01211D4A184867F0D3F894F89A
:1066A0002930032B11D1638D022B0ED1A18D002235
:1066B0000E0A3146A06967F08AFD054628B101211E
:1066C0003346134A0D4867F0BDF800232E4684F880
:1066D0003930FFF73CBBE38D002B3FF4A7AB0599A6
:1066E000003918BF0121C9016BF0B5F8FFF73FBBB6
:1066F000103700200C3700202FD20A0034F909008F
:1067000043D20A000C0000006CD20A00A2D10A0099
:1067100090D20A0030B589B0002200230024CDE9D0
:1067200006236FF007034FF48062CDE90334CDE90F
:106730000144154B15490094154828F095FC15495E
:1067400013486DF056F9144B14498B4207D30020BF
:10675000134B14498B420CD3002009B030BD03F118
:106760001402D2E8EF0FC2E8E54F002DF9D118333B
:10677000EBE703F11402D2E8EF4FC2E8E50F002D7A
:10678000F9D11833E6E700BF0168010068910020E5
:10679000E0200020B7D20A005C1800207418002006
:1067A000741800207418002038B50D4667F0ADFD50
:1067B00030B90121BDE838400F4A104867F039B8B8
:1067C000C46804B938BD2B78032B05D0052B0ED037
:1067D000022B08D02468F4E7606883685B69002BAB
:1067E000F8D09847F6E7606883689B69F7E76068C8
:1067F0008368DB69F3E700BFBCD20A0044F90900F3
:106800002DE9FF4120274FF0FF334FF0FF3264485E
:1068100001A927F073FF039B1B69D3F89C40236AEF
:1068200093B1EFF3118287F31288BFF36F8F216A60
:1068300029B1606A0B688142236208BF636282F3F8
:106840001188BFF36F8FC9B99DF80430062BDAD0D9
:10685000072BD8D801A252F823F000BFA16801008D
:1068600095680100C9680100A7680100FD68010082
:10687000EB68010007680100916901000B7E20466A
:106880005D06D1F81E2002D1FFF74EFAC7E767F088
:1068900075FDC4E700220121204667F088FEB2E7BB
:1068A00000221146F8E794F86C3043F0040384F8B2
:1068B0006C3094F83030022B03D1204601A9FFF749
:1068C00073FF00220321E7E794F86C3023F0040300
:1068D00084F86C3094F83030022B03D1204601A9A3
:1068E000FFF762FF00220221D6E794F83030022B36
:1068F00089D1204601A9FFF757FF84E794F86C304F
:10690000A66923F0040384F86C30D6F80880336954
:10691000A033D3E8AF3F9A071ED53046D8F83C30B5
:106920009847D8F824300021304698470546D8F8D3
:1069300040303046984795B11A4A01211A4866F00E
:1069400078FF00220421204667F031FE002D3FF43D
:106950005AAF2A4607219FE74FF0FF35ECE729465B
:10696000204600F027F8054608B1104AE5E7A0697F
:106970006BF067F8831E5842584194F86C3084F8E5
:10698000305023F0680343EA401384F86C30D8E7B2
:106990000121074A044866F04CFF0621029A7BE772
:1069A00034160020EBD20A0044F9090019D30A007A
:1069B00045D30A002DE9F04105460E4667F0B3FBCA
:1069C00095F8383080463BB3284667F09EFC074672
:1069D000F8B10146284667F0F1FC10220446002178
:1069E00005F13A0088F070FA002385F83830FF6826
:1069F00047B98CB10121194A194866F01AFF20469F
:106A0000BDE8F081786883685B6A03B198473F68A6
:106A1000EEE76FF03C04EDE71EB985F8386000241E
:106A2000EDE732464146284667F05BFC074690B1E9
:106A30000246284667F0ECFC04460028DFD185F8C2
:106A40003860FC68002CEAD0606883681B6A03B178
:106A500098472468F6E76FF03C04D0E769D30A0052
:106A60002CF9090070B5012501F07F0311F0800FAA
:106A700018BF10339D4090F830300446022B06D0EA
:106A800001210C4A0C4866F0D4FE002070BD90F83D
:106A9000386067F048FB32460146204667F021FC2B
:106AA0000028F2D0C0680028EFD083681D42EDD1E5
:106AB0000068F8E790D30A003CF909002DE9F04F8F
:106AC00083B000AF7B6097F830304C680E463B6077
:106AD0008146904667F027FBA36801461B6B33B9DC
:106AE0006FF0150420460C37BD46BDE8F08F2046F8
:106AF00098470028F4D00024051F06F10C0A55F829
:106B0000041F09B10B782BB9002C14BF00246FF0BF
:106B10003C04E7E74B78042B0ED1002C3CD18B785A
:106B20007A689342EBD1CB783A689342E7D10B79FC
:106B3000002BD7D00124E2E7052BE0D1002CDED0DA
:106B4000B8F1010F91F802B009D0B8F1020FF1D1FC
:106B500052465946D9F8180067F0E8FC04E052465E
:106B6000D9F8180067F0C6FC04460028E2D06D464C
:106B70008AB06A46F368CDE907B30623074909904E
:106B8000CDE9051842F8103F00234FF44151044865
:106B9000FDF79AF8AD46A5E70024A3E7C0D30A00A5
:106BA00064F909002DE9F0410B7E0C4659060546B3
:106BB00037D16BB367F0BCFA40B11B4801211B4AC7
:106BC00066F037FE4FF0FF30BDE8F0812846D5F87B
:106BD0007080268AEF8D67F0A6FAF8B1421E534204
:106BE00053419B01228A9AB1BE42324628BF3A469F
:106BF000E98D91420CD9B2FBF3F103FB11223AB9B2
:106C000094F91830002BBEBF637E43F0080363760F
:106C10002146A869BDE8F0416AF079BE98F80730CE
:106C2000E0E76FF01500CFE75CF90900FCD30A003C
:106C300070B5064680690C466AF00DFE054638B10F
:106C400002212346094A0A4866F0FCFD284670BD29
:106C5000012214F0800F18BF24F08004736B18BF5A
:106C60001034A2401A437263F0E700BF10D40A0048
:106C70005CF9090070B5054680690E466AF016FE9B
:106C8000044638B102213346054A064866F0DAFD6B
:106C9000204670BD314605F1340067F01DFCF7E772
:106CA00027D40A005CF9090070B50646EFF311819C
:106CB000202383F31288BFF36F8F1B4D2A6881F363
:106CC0001188BFF36F8F526892F86C20D20705D4F9
:106CD000BDE870402022002328F042B9EFF3118272
:106CE00083F31288BFF36F8F2C682CB16968236817
:106CF0008C422B6008BF6B6082F31188BFF36F8FEB
:106D000044B1606804F10801C36998472146074807
:106D10006CF075FB2B6833B13046BDE87040002243
:106D2000002328F0E5B870BD14370020AC15002012
:106D300030B585B0CDE90012054600220023144885
:106D400003A927F041FC0246E8B9DDE90001039BF5
:106D50005D60083383E80300EFF31180202383F3A1
:106D60001288BFF36F8F039B1A600A4A516861B99A
:106D7000C2E9003380F31188BFF36F8F0022002334
:106D8000054828F0B5F805B030BD0B605360F1E759
:106D9000AC1500201437002000000020D3B50026D9
:106DA00000270446CDE90067054867F0D5F828B10B
:106DB000230658BF0023047658BF038202B0D0BD1B
:106DC000D81700202DE9F04383B000234FF00108CD
:106DD00005691C4C1C4E02AF28602B7785F82030CB
:106DE00005F12409B442234601D3002019E095F8A7
:106DF00020201034CAB16C4688B01B6802AA13491F
:106E0000C2E905134FF400739383114B42F8103F0E
:106E1000104800234FF4E251FCF756FF6FF00B00CF
:106E2000A5460437BD46BDE8F08385F8208054F8B8
:106E3000043C4846009354F8101C54E9032367F0BF
:106E40003AFDCFE7288A0B00288A0B0051D40A00AC
:106E50000300000174F909001FB5CDE90101039297
:106E60004FF0FF324FF0FF3301A903486CF02AFBCB
:106E7000002005B05DF804FB041600201FB50023B8
:106E80000190CDE902334FF0FF324FF0FF3301A9FB
:106E900002486CF017FB05B05DF804FB04160020F7
:106EA0002DE9F041036804461B6917465B680E46EE
:106EB00093F80B804046FFF771FFD4F87B2005461E
:106EC000D21B0146C4F87B20206867F04AFB88B1DA
:106ED0000B4A434601210B4866F0B4FC314620467C
:106EE00067F030FC2846FEF7CFFD2046BDE8F041B4
:106EF00067F0DCBBA37F0133A377BDE8F08100BF5F
:106F000068D40A0074F909002DE9F04105463027DC
:106F100003681B695B689E7CEB7F012B27D82B687D
:106F2000D3F8108098F8614007FB0484243420468D
:106F300067F0E7FCB0F5007F636A044628BF4FF4B2
:106F4000007424F03F0413B1B4FBF3F45C4398F8ED
:106F50001F205AB1041BB4F5007F28BF4FF4007402
:106F600024F03F0413B1B4FBF3F45C430CB9BDE867
:106F7000F081284667F029FB2246014680463046CC
:106F8000FFF70CFF04460146286867F0EAFA80B173
:106F900001213346094A0A4866F054FC2046FEF7B0
:106FA00073FD4146284667F0CDFBBDE8F04167F030
:106FB0007DBBEB7F0133EB77AEE700BF68D40A00FF
:106FC00074F909002DE9F04FB14F87B04FF0FF324F
:106FD0004FF0FF33AF4803A927F090FBDDF80C908A
:106FE000049DD9F81040002D40F08D80257704F1E4
:106FF000240694F820309D427FDB04F11803D3E887
:10700000EF2F22F00202C3E8E12F0029F7D1D3E8E5
:10701000EF1F21F00401C3E8E21F002AF7D104F1B9
:107020001803D3E8AF3FDB07D0D5237F022B00F056
:107030006981032B00F0628143BBDDF80CA0DAF814
:107040001050EB7F13BB6B68284693F8129067F0E3
:10705000BCFA4022014606464846FFF79FFE80469E
:107060000146504667F07DFA002800F04381012177
:107070004B46894A894866F0E5FB4046FEF704FD29
:107080003146284667F05EFB67F010FBA37F002BBC
:107090009CD1237F012B40F05A81302304F16306F9
:1070A00094F86150304694F8621003FB054500F0F7
:1070B0003FFA2435024631462369284600F056FA45
:1070C0000646C4F88400284667F011FC814628462D
:1070D00067F012FC8046284667F013FCE26D3044EE
:1070E000002A40F01881002840F01081284667F0FF
:1070F0002FFC003818BF012009E1304667F0EEFB95
:107100000135303675E7059AD9F804A02B7EF2B127
:10711000298A71326148009107BF614A0221012129
:10712000604A66F099FBD9F810202B7E5268917C5A
:10713000994240F0D780E37F013BE37720466969BD
:1071400067F000FB2946504667F023FA67E761685D
:10715000887C984240F09280237FEE68B5F810B0AA
:10716000002B48D1BBF11F0F41D13368BB423ED148
:10717000314604F1540306F11C0251F8040B91420C
:1071800043F8040BF9D10A881A808A7842219A7050
:10719000552384F87330532384F8743084F87630A0
:1071A000A36DE26DC4F877300023C4F8803094F802
:1071B0006030C4F87B209A0684F875100FD194F8DB
:1071C000612094F820309A4209D294F86230013B51
:1071D0000F2B04D8012384F87F302377A3E720689E
:1071E00067F007FA022384F87F300423F5E720468E
:1071F00067F05CFA97E7032B95D1302394F8618010
:1072000003FB0848D4F8803008F124085B44C4F834
:107210008030BBF1000F15D0404667F072FB88B19B
:1072200031465A46404667F07EFB064628B90221A1
:107230005B461D4A194866F005FBD4F87B309B1B62
:10724000C4F87B30D4F88020E36D9A420DD24046DA
:1072500067F057FB00287FF466AFD4F88020E36D19
:107260009A4202D2206867F0CAF9404667F070FB84
:10727000003818BF012084F87F00B6E7C97A994228
:107280007FF451AF237F052B10D122774BE700BF4E
:10729000555342430416002068D40A0074F90900CB
:1072A0008DD40A00B1D40A00D2D40A00022B7FF494
:1072B0003AAF2A8AD4F8803020681344C4F880306A
:1072C00094F8616067F026FA00287FF42CAFD4F8B8
:1072D0007B3013B1206867F08CF9302303FB064044
:1072E0002430C3E7D27A9A4202BFA37F03F1FF336F
:1072F000A37723E7EB7F0133EB77C7E62046FFF761
:1073000003FEC3E6204667F02DFABFE6022084F8AC
:107310007F0004231AE094F9601040B90029206826
:1073200002DA67F066F9E1E667F069F9DEE600295E
:1073300014DA904202D8B9F1000F06D1206867F044
:1073400058F9022384F87F30E3E702232377237F71
:10735000022B0ED1204667F005FA37E6904202D89C
:10736000B8F1000F03D1206867F049F9E9E703237A
:10737000ECE7032B03D12046FFF7C6FD26E6042BDE
:107380007FF424AEA37F2BB101211E4A1E4866F074
:1073900050FA1BE6236820461B695B6893F80B8054
:1073A00067F013F90546024604F1730304F17F0107
:1073B00053F8040B8B4242F8040BF9D11B78294691
:1073C000137040460D22FFF7E9FC0646014620688F
:1073D00067F0C7F878B10D4A434601210A4866F0C4
:1073E00031FA3046FEF750FB2946204667F0AAF9ED
:1073F00067F05CF9EAE5A37F0133A37705232377E0
:10740000E4E500BFF8D40A0074F9090068D40A0062
:10741000802938B50D46144621D083290DD019BBDB
:107420008023537183230320117193710023E07033
:1074300023706570A370043038BD022313710123DB
:107440005371002393710A23D37108224168A01855
:1074500087F071FD064B0E201B882382E6E7044B64
:1074600002201B889380E1E76FF08500E4E700BF0E
:10747000443B0B002DE9F0418769D0F82480BA42E3
:1074800028BF3A46B2FBF8F40646C26923460068B4
:1074900066F0B1FB0546C0B9B7FBF8F7A7420BD1C0
:1074A000002205213068FCF751FF28B101210A4A6A
:1074B0000A4866F0BEF90125F3692344F3613DB142
:1074C0000020074BB362BDE8F08100240125E7E707
:1074D000706A6043F7E700BF19D50A0074F9090024
:1074E0000203000C81420B4607B509D302210D4A65
:1074F0000D4866F0A7F96FF0150003B05DF804FBC6
:107500006AB101391144814201D28B4207D902216B
:10751000009305481346054A66F09EF9EBE7002004
:10752000EBE700BF30D50A0074F9090047D50A001F
:107530000C290346084616D11B78252B12D009D8F2
:10754000122B10D8084A42FA03F313F0010F08BFB8
:107550000620704703F0FD02282A03D05A2B08BFEB
:107560000A2070470A207047F6FFFBFF2DE9F04123
:10757000984690F82C3086B023F00C0380F82C301D
:107580000023C0E904338361062A04460F460B78C2
:1075900040F010810BBB4B795B0724D490F82C3062
:1075A0009F070DD402234FF468521946002584F832
:1075B000283084F829106285284606B0BDE8F0819D
:1075C00067F0FEF80028EDD1002319461A46EDE7D2
:1075D0000223052145F20232E8E7032B36D14E792A
:1075E00016F0040604D0022305214FF41052DDE703
:1075F00090F82C308DF8076043F0040380F82C30AD
:107600007023ADF8043090F829300D7903F00F03A2
:107610008DF806300A23122D28BF12258DF80B3065
:10762000438D2A465BBA404601A98DF808608DF863
:1076300009608DF80A600396ADF81030ADF812605D
:10764000ADF8146087F01AFCA662B5E71B2B00F0BA
:10765000898009D8122B1AD01A2B61D00121B24A85
:10766000B24866F0EFF8BEE71E2BF7D14B795E0704
:10767000B9D40B7913F0030300F09780012BA3D149
:1076800090F82C3043F0010380F82C309CE74B79C4
:107690005E07A8D490F82C3043F0040380F82C3017
:1076A0004A7812F002061FD1D5078B7822D5B1F89F
:1076B000035042461946FFF7ABFE6DBAADB28542A4
:1076C0000BDAB7F803506DBAADB200231A4684F84E
:1076D000283084F8296062856EE742462046B978F2
:1076E000FFF796FE051EF0DA022305264FF410522E
:1076F0000025ECE72BB102218D4A8C4866F0A2F8F8
:10770000F2E7B1F8035041466DBAADB267F08BF8BD
:10771000232DD6D94146204667F085F82425D4E7A5
:107720004D7915F004057FF45EAF90F82C3043F0EE
:10773000040380F82C308B783F2B0ED1CE78002EAE
:10774000D2D10D790323042D28BF042540462A46B3
:1077500001A9019387F092FBB7E7022305264FF4B6
:107760001052B4E74B7959073FF53DAF3B791A0901
:107770000CD19A070AD5DB0715D494F82C3003F006
:107780000303032B3FF424AF002305E094F82C20DF
:107790009707C2F34003F0D594F82C2063F341021D
:1077A00084F82C2010E70123F6E790F82C2063F3EF
:1077B0000002F5E70A2A7FF451AF2A2B1AD8222BB0
:1077C0007FF64CAFA3F12302072A3FF647AF01A192
:1077D00051F822F04B7801005D760100CD78010070
:1077E0005D7601005D760100357901005D7601006E
:1077F0008D7901005A2B7FF431AF4D7A15F00405D5
:107800007FF4F1AE90F82C3043F0040380F82C3074
:107810008B783F2B40F0DD80CE78002E40F0D98071
:107820004FF4C063CDE90136B1F8075040466DBA58
:10783000ADB2082D28BF082501A92A4687F01EFBF6
:107840003246334684F8282053E07B7A13F0040351
:107850007FF4C9AE01AEADF80430B370082390F8E0
:107860002C208DF8073042F0040280F82C2066F0BE
:10787000A7FF0028B5BF4FF0FF3302220322236A7F
:107880008DF80C20A8BF1BBA0293636A31461BBA5D
:107890008DF80D30C3F30722C3F307438DF80F3083
:1078A00094F82C308DF80E2043F0040384F82C302B
:1078B000B7F8075040466DBAADB20C2D28BF0C2565
:1078C0002A4687F0DBFA0023A36275E67E7A16F07B
:1078D00004067FF488AE90F82C3043F004039D0733
:1078E00080F82C3009D402264FF46853002584F820
:1078F000286084F8296063855EE666F061FF0028F1
:10790000F1D1236A03B1013B94F82C10626A1BBACF
:1079100012BA41F0040184F82C100825C8F8003090
:10792000C8F804200023E2E78ED50A0074F90900A4
:1079300071D50A007B7A58073FF555AE94F82C3084
:10794000D7F8026043F004039907B7F8075084F8AA
:107950002C307FF527AE204666F032FF00287FF4FA
:1079600021AE6DBA36BAADB22A463146206AFFF76B
:10797000B9FD20B1022305214FF4045216E6174B3E
:107980002361636AE6616B43A3611DE67B7A5A0754
:107990003FF529AE90F82C30D7F8026043F0080389
:1079A000B7F8075080F82C309B077FF5FBAD66F0E9
:1079B00007FF00287FF4F6AD6DBA36BAADB22A469D
:1079C0003146206AFFF78EFD0028D3D1044B636156
:1079D000D7E7022205264FF4105333E789E8070062
:1079E0007574010070B50B7892B006460C4607AD71
:1079F000032B31D8DFE803F0022A2C2E1949284640
:107A0000F9F780FA05956378174A0493A3781E2145
:107A10000393E3780AA80293237910AD0193637965
:107A20000093A37960F062FB32460AAB1C4603CC9C
:107A3000AC4210605160234602F10802F6D1206882
:107A400010603046A388938012B070BD0749D6E716
:107A50000749D4E70749D2E70A212846064A60F0D9
:107A600045FBCFE7A9D50A00C4D50A00A62B0B0019
:107A7000B0D50A00BAD50A0061F70A000E4B4029BA
:107A800028BF402170B51D460C4C4618B04203F18A
:107A9000020304D1002305F81130074870BD0278B5
:107AA0001209A25C03F8022C10F8012B02F00F025D
:107AB000A25C03F8012CE9E7DB870020463C0B00C1
:107AC00010B50024094B86B009480393CDE904445E
:107AD0006BF02EFF03AB00934FF440620A2305497D
:107AE000034827F09BF9204606B010BDEED50A00EA
:107AF000A0220020689B00200146014827F0CEB953
:107B0000A02200200146014827F0F8B9A022002059
:107B1000014601486BF0E1BEA02200202DE9F743A9
:107B200006468946174698463C4DD5E8AF3FDA07EA
:107B300022D548B901213A4A3A4865F07AFE6FF0F9
:107B4000010003B0BDE8F08301A966F096F80228B1
:107B500004462BD102463449304687F0BDF900284F
:107B6000EDD1D5E8AF3FC3F3C0061B0706D52F4ABA
:107B700021462C4865F05DFE0020E2E7A5F188046F
:107B8000072221464046B84706280AD80121284A3C
:107B9000244865F04EFE45F8886CE671C4F8036031
:107BA000EAE70723B0FBF3F0E071E5E7042818D11A
:107BB00002462049304687F08FF904460028BED19E
:107BC0001C22404605F1A001B847031E05DA012139
:107BD000194A144865F036FECEE72B4483F8A040DE
:107BE000CAE70A28ABD102461449304687F074F937
:107BF0000028A4D1B9F1020F07D00A480121104A88
:107C000065F017FE6FF015009BE74A46404605F108
:107C1000BE01B84700EAE07093E700BFB80000205B
:107C2000F7D50A0054F80900B7D50A0018D60A009B
:107C30003CD60A0027DC0A0061D60A0093D60A0067
:107C40009ED60A002DE9F04389B0DDF840909D7979
:107C50005E791F7993F803C093F802E093F80180EE
:107C60000C461B78B9F1000F15D0CDE90639CDE9E6
:107C700004E81346CDE9027CCDE900560D4A60F0D8
:107C800035FA002813DBA0422CBF6FF0150000204E
:107C900009B0BDE8F083CDE90583CDE903CE1346F5
:107CA000CDE90167044A009560F020FAE9E76FF03A
:107CB0001500EDE7D5D60A00F9D60A0010B5FCF795
:107CC0001DFD044628B101210346034A034865F01F
:107CD000B9FD204610BD00BF1AD70A0054F80900AC
:107CE00070B504461E4615468CB0AAB129B10A46A5
:107CF00002A8042164F087FF02A900912B462246C6
:107D0000242103A8FFF79EFF70B93146109A03A8FB
:107D1000FCF770FB0CB070BD03462421044A03A895
:107D200060F0E4F92328F0D96FF01500F2E700BF06
:107D30003FD70A0007B50B4B0B48DA79C2EBC202FA
:107D4000009200221146FFF7CBFF034638B1012114
:107D5000064A074803B05DF804EB65F073BD03B055
:107D60005DF804FB30000020B7D50A0045D70A00B3
:107D700054F8090030B5044615468DB09AB129B1C2
:107D80000A4602A8042164F03EFF02A900912B4696
:107D90002246242103A8FFF755FF60B903A865F028
:107DA00044FF0DB030BD03462421044A03A860F00F
:107DB0009DF92328F2D96FF01500F2E73FD70A00AA
:107DC00007B5009313460A4601460348FFF788FFAC
:107DD00003B05DF804FB00BFA0F40A000A460146A8
:107DE0000148FFF7C7BF00BFA0F40A0007B5009322
:107DF00013460A4601460348FFF772FF03B05DF8D9
:107E000004FB00BF9AF40A000A4601460148FFF746
:107E1000B1BF00BF9AF40A0007B5009313460A46A3
:107E200001460348FFF75CFF03B05DF804FB00BFA9
:107E3000CBF20A000A4601460148FFF79BBF00BF8C
:107E4000CBF20A0007B50022034600910348114611
:107E5000FFF746FF03B05DF804FB00BF92F40A0091
:107E600007B500220346009103481146FFF738FF8B
:107E700003B05DF804FB00BF27DC0A0007B5002251
:107E80000346009103481146FFF72AFF03B05DF84F
:107E900004FB00BF93D60A0008B5024826F0B8FFDD
:107EA000002008BD80040020F8B51E4DD5E8AF3F86
:107EB00013F0010F2F4632D095F8A040A5F18806A7
:107EC0003CB91C22184906F5947087F034F886F8FE
:107ED0004441F3798BB902F039F8044630B10121FD
:107EE000124A134865F0A5FC2046F8BDF37923B982
:107EF00002F03CF804460028F1D1D5E8AF3F5A071C
:107F000001D400F0C5FED7E8EF3F23F40062C7E8D4
:107F1000E12F0029F7D11B0501D5FFF7BDFF002494
:107F2000E2E700BFB800002060D70A0067D70A0068
:107F300054F8090007B5009313460A460146034862
:107F4000FFF7CEFE03B05DF804FB00BFD1F90A00D5
:107F50000A4601460148FFF70DBF00BFD1F90A00EC
:107F600030B50378012B11D0022B21D06BB90A4612
:107F7000144B03F1100453F8045BA34242F8045B72
:107F8000F9D143881A0A8A70CB7030BD0A460D4B6E
:107F900003F1100453F8045BA34242F8045BF9D1E7
:107FA00043681A0C180E4A700870C3F30722EAE7F8
:107FB00000F11003013913F80129984201F8012F4B
:107FC000F9D1E2E7573C0B0010B566F09BFD6BF072
:107FD0000AFD044608B927F043FB064BD3E8AF3F40
:107FE0000BB10A2098471CB9BDE8104027F04CBBE4
:107FF00010BD00BF1C3B002038B50446084865F0A2
:10800000A7FF054648B1631EDBB21F2B96BF054A8A
:108010000021D15C0C3066F033F8284638BD00BF33
:10802000AC170020673C0B000F2810B50CD80D28AA
:108030000CD90A4865F08CFF044618B104210C30B5
:1080400066F01EF8204610BD1328F2D009B104488E
:10805000F0E70220BDE81040FFF7CEBF0418002073
:1080600028170020C3681B780221024A024866F0E4
:10807000E7BD00BFA9D70A001CF80900F8B50646FD
:108080000F4604F0F5FA044690B9394630460AF036
:1080900061FF0546F0B93946304608F0A9FF164B96
:1080A0001B6823B153F80C4904B10C3CB3B9F8BDBB
:1080B00083781321012B4FF0000312BF1D46D0F827
:1080C000A450C0F8A43067F0E8F9204603F05CFE45
:1080D000002DDAD0284669F05EFADCE79B6813B120
:1080E0003946304698472CB1E26802B10C3A234633
:1080F0001446DBE72246FAE7E43B002010B50024F3
:1081000086B003AB00934FF480624FF0FF33054914
:108110000548CDE90344059426F080FE204606B0CC
:1081200010BD00BF68A70020A023002038B5C56897
:108130002B7893B9B5F801400F21204603F082FF58
:10814000EB78054650B90A4A118831B96FEA0450F4
:108150006FEA10501080074A137038BD0373012175
:1081600003F05EFE2846BDE8384003F00DBE00BFB8
:10817000A88500205C88002070B5C3681D787DBB91
:10818000B3F801600F21304603F05CFF044638B9B4
:1081900001213346BDE87040124A134866F050BDD5
:1081A000294603F03DFEA378012B04D02046BDE80C
:1081B000704003F0E9BD201D66F02BFDC307F5D527
:1081C0000321204603F02CFE032002F019FF034692
:1081D0000028EBD00221054A034866F031FDE5E7AF
:1081E00070BD00BFD1D70A001CF80900F7D70A00FC
:1081F00010B5C3680121B3F80140204603F022FF07
:1082000038B901212346BDE81040044A044866F00D
:1082100017BDBDE8104003F0B7BD00BF1DD80A0070
:108220001CF8090010B5C36801211C88204603F022
:1082300009FF38B901212346BDE81040034A04482C
:1082400066F0FEBCBDE8104003F09EBD1DD80A00DC
:108250001CF8090010B501210C3065F043FF0378CC
:108260000121BDE81040024A024866F0E9BC00BFA7
:1082700041D80A001CF80900014610B5084865F00D
:108280007EFE084908486BF028FB031E06DABDE8AD
:1082900010400121054A064866F0D2BC10BD00BF5F
:1082A00034010020A0040020A024002063D80A008C
:1082B0001CF809000121024A024866F0ADBC00BF6B
:1082C00080D80A001CF8090070B5C5680121B5F80E
:1082D0000160304603F0B6FE044638B9012133464A
:1082E000BDE870400B4A0C4866F0AABC2B783BB93D
:1082F000D5F80330C0F89930D5F80730C0F89D3074
:10830000201D4FF4003166F090FC2046BDE870401F
:1083100003F03ABD1DD80A001CF8090008B502F0A8
:1083200025FE064B184666F074FC00F00B00D3E8FF
:10833000EF2FC3E8E10F0029F9D108BDB8000020F4
:108340000B46B0B50D8A00AF04462946D868FFF742
:1083500095FB8AB06A460A4BCDE90750CDE9053452
:1083600040F20243ADF82430064B42F8103F0023A0
:108370004FF432510448FBF7A7FCBD46B0BD00BF27
:108380009AD80A00050000011CF809002DE9F84FF1
:10839000D0F80C90018A99F8004000AFA300013397
:1083A0008B4260D96D468AB06A46CDE90731052314
:1083B0002E48CDE9050442F8103F00234FF4215127
:1083C0002B48FBF781FCAD46BD46BDE8F88F012187
:1083D0002B46284A264866F033FC013699F80030CF
:1083E0009E42F1DA09EB8603B3F801500F212846CB
:1083F000B3F8038003F026FE04460028E7D000F11E
:10840000C00AB8F1000F06D0656945B901211A4AC2
:10841000174866F001FC204603F0B6FCDDE7A269D0
:108420002B6895422046636108BFA36103F0CCFB33
:1084300026F0C0FAC5F800B0236A8BB9C4E9075525
:10844000DAE8EF3F013BCAE8E23F002AF8D1002119
:10845000204608F1FF3803F0C1FB1FFA88F8D0E787
:108460001D602562ECE70026B346B7E7BCD80A00DA
:108470001CF80900E7D80A0003D90A0080B500AF4C
:108480008AB06A46094BCDE90530094B079340F2A3
:108490000133ADF82030074B42F8103F00234FF472
:1084A00012510548FBF710FCBD4680BD1AD90A00E1
:1084B000BC010B00040000011CF8090037B504469C
:1084C000084602EBC3039A4202D16FF05E0010E04F
:1084D000114611F8085BA54211D1038A51789942DF
:1084E00009D908480121084A009465F0B5F96FF0F0
:1084F000150003B030BD536898470020F9E70A46DD
:10850000E1E700BF1CF8090036D90A002DE9F04761
:108510000C4627F0A5F8E5682B78022B72D0042BC7
:1085200007D001213B4A3C4866F08AFB6FF01504F6
:108530000EE0B4F81080B8F1020F0ED84346374A67
:108540003548012166F07CFB2046FDF79DFA0024AA
:1085500027F09AF82046BDE8F08768783E280CD1CD
:10856000B8F1030F02D12E4A4346E9E7EB78012B1D
:1085700001D00A2B46D1032704E066F037FB0746FB
:10858000F8073FD504F10C0601213046D4F814A0B9
:1085900065F0A0FD0221304665F0A4FD814600781B
:1085A0003E2807D1E3681B78012B01D00A2B06D1A6
:1085B000032614E066F01AFBC10706460FD441F209
:1085C0008A13184A1849194864F0A4F8002383F361
:1085D0001188BFF36F8F0323184602DF0226144A67
:1085E0000623214699F8000066F04BFBB2070DD533
:1085F0006369A5EB0A0513FA85F5E560A4F8108018
:10860000BB07A4D52046FFF737FEA0E72046FDF7BD
:108610003BFAF5E7FED90A001CF8090058D90A0010
:1086200074D90A0094D90A00C8D90A00E1D90A000D
:10863000B0FF090010B5012104460C3065F052FD71
:108640002146BDE810400223014A007866F019BBBC
:10865000E0FF090073B53E4865F0A6FC044600281B
:1086600073D000F10C05284665F044FD022803464E
:1086700003D0042847D0374A03E0238A032B05D8C8
:10868000354A0121354866F0DBFA13E0042128461B
:1086900065F028FDFF23428806882376238AC6F3E7
:1086A0000B009A42608309D0012100922B482C4A8A
:1086B00065F0D2F82046FDF7E7F912E00F2103F04C
:1086C000C1FC054610B9638B264ADAE703F0E0FCEB
:1086D00021462076320B284603F0D2FA284603F0D2
:1086E00053FB214BD3F804317BB3204920486BF076
:1086F000F4F8031E29DA01211E4A184802B0BDE829
:10870000704066F09DBA2846022165F0EBFC0546F4
:1087100000783E2812D066F069FA10F002060DD1FA
:1087200040F6BC43144A1549154863F0F3FF86F33D
:108730001188BFF36F8F0323184602DF06232146FB
:10874000104A287866F09DFAB4E702B070BD00BF09
:1087500034010020A7DA0A0012DA0A001CF8090026
:1087600033DA0A0057DA0A0030000020A0040020A3
:10877000A024002063D80A0094D90A0079DA0A00FC
:10878000E1D90A00F0FF090010B5012104460C30C0
:1087900065F0A8FC2146BDE810400D23014A007891
:1087A00066F06FBA20000A00F8B50121044600AF58
:1087B0000C3065F097FC0678002321463046114ABC
:1087C000FFF77CFE5F301AD1258AE0682946FFF763
:1087D00055F96C468AB06A460B4BCDE90750CDE996
:1087E000053640F20243ADF82430084B42F8103F02
:1087F00000234FF432510648FBF766FAA546BD4602
:10880000F8BD00BF88000A00BBDA0A0005000001BD
:108810001CF809002DE9F74F0023804689461746CA
:10882000DFF810A1DAE8EF4FCAE8E23F002AF9D1F9
:10883000264644B9012143463A4A3B4803B0BDE8C5
:10884000F04F66F0FDB92046FDF77EF84FF00C0BB7
:10885000364D0BFB0050438843451BD02046FDF7A7
:1088600073F80BFB0050438801210093304A4346C4
:108870002D4864F0F1FFDAE8EF3FCAE8E26F002A22
:10888000F9D1002B4BD01E46304603B0BDE8F04F67
:10889000FDF7FAB8A74208D0204665F054FB3A8AA3
:1088A000F96804F10C0065F0E2FB2046FDF74CF896
:1088B0000C2707FB00504368ABB1B9F1000F12D190
:1088C0002046FDF741F8012107FB0050426853683C
:1088D00003F01F00814010685B0900EB8300137AEE
:1088E000CBB166F0A2F92046FDF72EF80C2707FB66
:1088F00000508368002BC7D02046FDF725F8784349
:1089000005F800902046FDF71FF807FB0055A86802
:1089100026F050F8B8E7C94366F099F9E3E703B0E9
:10892000BDE8F08FEDDA0A001CF80900203B0020BA
:1089300015DB0A003001002073B5C5680121B5F8C8
:108940000160304603F07EFB044640B90121334606
:108950003D4A3E4802B0BDE8704066F071B92B78E0
:10896000061D1A2B19D1C378012B50D14FF4804129
:10897000304666F05AF942040FD4D4F88C30694678
:108980000093D4F894302046019304F09FFB2046D6
:1089900002B0BDE8704003F0F7B92B78BBBB40F2E2
:1089A000E242B5F803302A495343C4F88830B5F899
:1089B0000520A4F89020B5F80720A4F89220A3F58C
:1089C000EA520C3A8A4204D90221224A1F4866F030
:1089D00037F9B4F89030B3F5FA7F04D302211E4A78
:1089E0001A4866F02DF940F67641B4F89230A3F1BA
:1089F0000A0292B28A4204D90221184A134866F048
:108A00001FF96FF48051304666F021F914E03046CA
:108A100066F0FFF8C304F4D52B78202BF1D194F83D
:108A20009830002BEDD0013B84F898300C4A00239D
:108A300004F1400026F05CFA2B78002BA7D12046E9
:108A400003F0FCFCA3E700BF1DD80A001CF80900D6
:108A500095F03C0048DB0A006FDB0A0096DB0A0059
:108A60005A62020010B5C1E900239DF808300C4697
:108A70000B72FCF769FF0C22024B02FB00335C60B7
:108A800010BD00BF203B0020F8B502460B46104841
:108A900065F05EFA0446C0B104210C3065F0D6FAE8
:108AA0002046FCF751FF0C2700260A4D07FB00501B
:108AB00046802046FCF748FF07FB005086602046B2
:108AC000FCF742FF07FB00556E602046F8BD00BF73
:108AD00080170020203B00200138C0B202289ABF36
:108AE000014B185C00207047B13C0B0037B50C46B9
:108AF0008DF8070000F0FF05A0B929B10722204634
:108B00000A4986F0E9F940B9002009490DF1070248
:108B10000AF08CF9002003B030BD21462846FFF74B
:108B2000ADFAF7E76FF01500F5E700BF333C0B0037
:108B300045EC070029289ABF014B185C09207047B3
:108B4000873C0B0070B5C3680F21B3F801601D7836
:108B5000304603F077FA044638B901213346BDE8C0
:108B60007040184A184866F06BB865B12846FFF7A0
:108B7000E1FF29460246204603F018FD2046BDE8E5
:108B8000704003F001B98378012B07D10AF03AF85D
:108B9000204666F013F8002808BF05252846FFF791
:108BA000C9FF29460246204603F000FD002DE5D00E
:108BB0000121064A044866F02FF80521204666F098
:108BC0006CFCDBE7D1D70A001CF80900C2DB0A0005
:108BD0002DE9F041C6680F21B6F8017035783846A6
:108BE00003F030FA044638B901213B46BDE8F041B4
:108BF0001E4A1F4866F024B865B12846FFF79AFF61
:108C000029460246204603F0D1FC2046BDE8F0414B
:108C100003F0BAB8F278C37A934205D10221154A1B
:108C2000134866F00DF8F0E78378C272012B08D183
:108C30000AB109F0E7FF204665F0C0FF002808BF31
:108C400005252846FFF776FF29460246204603F011
:108C5000ADFC002DD9D00121074A054865F0DCFFA5
:108C60000521204666F019FCCFE700BFD1D70A00E6
:108C70001CF80900E8DB0A00C2DB0A00034B0146CE
:108C8000D3F8240182689268104700BF30000020AA
:108C900008B50421034865F0C8FFBDE8084002F0AC
:108CA00065B900BFB800002008B5034865F0B1FF02
:108CB000C0F3800008BD00BFB800002038B50546ED
:108CC000F8F728F91C2804461BD829460E48F8F75F
:108CD0000FF9A0B1224629460B4886F0CFF80022B2
:108CE0000A482146031900F5947083F82821FFF7FC
:108CF000B7F820B10221064A064865F08DFF002032
:108D000038BD6FF00B00FBE7580100203000002059
:108D100017DC0A001CF809000048704758010020C1
:108D2000014BB3F8460170473000002037B50F4DB6
:108D3000ADF80600B5F84631834203D10024204641
:108D400003B030BD02210DF10600FFF797F804468D
:108D500030B101210346064A064865F071FFEEE78F
:108D6000BDF80630A5F84631E8E700BF3000002026
:108D70002CDC0A001CF80900014902486AF0ADBD6C
:108D800090040020A023002070B505460C4639B1A0
:108D9000CB684A699B1A032B0ED86FF0150509E0C2
:108DA0004FF0FF304FF0FF31FFF76EFE044618B969
:108DB0006FF06805284670BD2046FCF7C5FD0C2203
:108DC000164BA61802FB0033032130465D8065F088
:108DD00070F90580238A0121033B8370304665F0DA
:108DE00070F940F635439D420FD12046FFF746FF0C
:108DF00005460028DED001210346094A094865F0EE
:108E00001FFF2046FCF740FED4E7214606486AF0E3
:108E100056FC0025FFF7B0FFCCE700BF203B002049
:108E20005DDC0A001CF809003C0100202DE9F04738
:108E300086B0804691460C4600AF71B94FF0FF30C6
:108E40004FF0FF31FFF720FE044660B96FF0680570
:108E500028461837BD46BDE8F087887AFCF76CFDD8
:108E60003C4B83426FD10122002138466AF05EFC00
:108E70002046FCF769FD0C23DFF800A103FB00A0EE
:108E80008760204665F0A6F801464046FFF77CFF64
:108E9000054618B12046FCF7F7FDD9E70023384610
:108EA0002D4A25F0C3FD064690B140F2E3132B4A4C
:108EB0002B492C4863F02EFC324641462A4863F089
:108EC00029FC85F31188BFF36F8F0323184602DF57
:108ED0002046FCF739FD0C2358431AF8006066B3AE
:108EE0006D468AB06A46214B0796CDE90538204B7E
:108EF000089340F20243ADF824301E4B42F8103F75
:108F000000234FF432511C48FAF7DEFE2046AD46EE
:108F1000093EFCF7B9FD092E0CD8DFE806F0050B79
:108F20000B08170B0B0B0B146FF06E0590E76FF02F
:108F30000C058DE76FF004058AE7B9F1000FA9D0A1
:108F4000C9F8004084E76FF0150581E76FF00B0565
:108F50007EE700BF80170020B4C4040094D90A0043
:108F60007FDC0A00E1D90A0088DC0A00CDDC0A00B7
:108F7000BC010B00050000011CF80900203B00208B
:108F800073B506460D4642F22F00002101AAFFF7F5
:108F90004DFF044638B10121144A154865F03CFEE6
:108FA000204602B070BD0198C368B3F8012032803A
:108FB000B3F803302B80FCF767FD3388A3F11B0265
:108FC000E02A04D902210B4A094865F039FE44F22F
:108FD00048112B88A3F5A47292B28A42E0D90221EB
:108FE000054A034865F02CFEDAE700BFECDC0A0016
:108FF0001CF809000CDD0A0031DD0A002DE9F04300
:1090000085B004460DF10301002001F01DF805466E
:1090100000287CD14FF0FF304FF0FF31FFF734FDD7
:109020000746002877D000F10C080A21404665F079
:1090300018F80646056045600581384D023095F800
:10904000DA3095F8DB209A4294BF04F1700104F104
:109050007E0165F0E3FD9DF803307370AB6813F09B
:1090600002091DD1012310214046737264F0F9FFFB
:10907000AA890280EA894280B4F88C208280B4F800
:109080008E20C280B4F890200281B4F8922080F83B
:109090000C90428180F80D9080F80E9080F80F902F
:1090A000AB68DB071CD5737A102143F004034046FC
:1090B000737264F0D6FF2A8A02806A8A4280B4F80A
:1090C0008C208280B4F88E20C280B4F89020028177
:1090D000B4F8922042810022027342738273C273F9
:1090E0000F4B384601930723029301238DF80C3070
:1090F000FCF72AFC0C220B4B394602FB003301AA79
:109100005A6042F243000022FFF790FE05462846CF
:1091100005B0BDE8F0836FF06805F8E73000002087
:10912000B8000020203B00203C2870B5054644D004
:1091300002283ED100210246084603F01BFB0446EC
:1091400080B901211D4A1E4865F066FD032001F02B
:1091500057FF034688B3BDE870400221194A1848FA
:1091600065F06EBD043065F054FDC30707D50321DB
:10917000204602F055FE204602F006FEE6E704F126
:1091800040006AF0E8FB10F00C0607D10E4A2946B1
:109190000B4865F041FD31462573E9E72046FFF7AE
:1091A0002DFF0028E7D00121084A054865F034FD6D
:1091B000E1E7BDE87040FFF761B970BD54DD0A001A
:1091C0001CF80900F7D70A0072DD0A0098DD0A00D2
:1091D00030B54FF0FF304FF0FF3185B0FFF754FC52
:1091E0000446B0B10C4B0025019307238DF80C50B9
:1091F0000293FCF7A9FB0C22084B214602FB00332B
:1092000001AA5A6042F20E002A46FFF70FFE05B08F
:1092100030BD6FF06800FAE7B8000020203B002066
:109220002DE9F0478CB0002605466F4BB0F8019051
:10923000198849F47042914204BF1E806B4B00AF05
:1092400008BF1E7800F074FDEB7805F10408012BCF
:1092500008BF674B404614BF002493F8224065F0D6
:109260004DFC4146002841D007F1080065F03BFC69
:10927000D5F81130C7F80130B5F81530A7F805302A
:1092800001233B70E87800283DD1022207F1080154
:1092900003F070FA0446EB7823B96FF0800155486B
:1092A00065F0D5FC002C43D107F110054146284656
:1092B000FEF798FB6E4688B06A464F4BCDE9053500
:1092C0004FF40073ADF81C304C4B42F8103F4FF494
:1092D000E2514B482346FAF7F7FC1321B5464846BE
:1092E00065F00AFD3037BD46BDE8F087204665F0E1
:1092F0009FFE014607F1080065F090FC41463846A4
:1093000065F08CFCBEE7012810D1DFF8E4A006224E
:109310009AF8220007F1080103F02CFA044600280D
:10932000B9D1052237499AF82200B1E70024B2E703
:10933000204640F2E242B5F8013007F1080120F87A
:10934000703B65F06BFCB5F817305343C4F88830B8
:10935000B5F81930A4F89030B5F81B30A4F8923065
:109360000023EA782373012AE2702BD1394604F1F5
:10937000770065F053FCD5F80B30C4F87F30B5F8B2
:109380000F3084F87E20A4F883300721204602F0B5
:1093900047FD26B101212046267302F041FD2046FB
:1093A00002F0B2FEE3784BB9032001F029FE034638
:1093B00020B10221144A124865F042FC204602F016
:1093C000E3FC8FE7002AE0D1394604F17E0065F026
:1093D00025FC217A064BC1EBC101194404F1770049
:1093E00065F01CFCD1E700BFA88500205C88002048
:1093F00030000020B8000020B4DD0A0003000001A6
:109400001CF809002C3C0B00F7D70A0000B5C16816
:1094100089B0087820B109B05DF804EBFFF784BE8D
:10942000B1F801308DF80000ADF80130CB7801A81B
:109430008DF80330B1F80B300431ADF81730B1F8C6
:109440000930ADF81930B1F80B30ADF81B304B7B5B
:109450008DF81D3065F0E2FB084B68461A689B8862
:10946000CDF80B20ADF80F30CDF81120ADF8153048
:10947000FFF7D6FE09B05DF804FB00BF403C0B00CF
:1094800010B5F7F7ADFE034B1B6813B1BDE81040F4
:10949000184710BD443B00202DE9F341344D0646EA
:1094A000D5F8240169F00FFF50B90121314A324843
:1094B00065F0B2FB6FF01204204602B0BDE8F08107
:1094C0006FF0020105F1880065F0C1FB012165F034
:1094D000ACFBC30748D4FEF7F1FB04460028EBD1F0
:1094E000264B1E60012205F1E80011466AF01EF9C4
:1094F000234F05F586706AF0A4F838466AF018FA2A
:1095000038466FF007034FF400621E49009425F0BF
:1095100085FCD7F8E0001C496AF06BFAD5F8240105
:109520000769D7F80080B8F1000F15D1174B3B60E1
:1095300083681B689847044628B986B902B0BDE81D
:10954000F041F7F74DBEC7F8008001212346104ACD
:10955000094865F075FBAFE76FF07704F5E705F1B3
:10956000780025F055FCA7E76FF07704A4E700BF6B
:109570003000002030DF0A001CF80900443B0020C6
:10958000A024002068AB002048DF0A000D85010000
:1095900051DF0A00F0B5C56801212F8887B0BCB241
:1095A000204602F04FFD064640B901212346274AD6
:1095B000274807B0BDE8F04065F042BB02ACD5F8E3
:1095C0000220D5F8063001946989009167F02DFEDC
:1095D00048B34FF0FF304FF0FF31FFF755FA054623
:1095E00048B901211B4A1A4865F016FB304602F0C3
:1095F000CBFB07B0F0BD12210C3064F032FD034606
:10960000224623F8027B144603CC596006A98C42FB
:109610001860224603F10803F5D1294642F21A00E8
:10962000FFF7B2FBE2E74FF0FF304FF0FF31FFF7FB
:109630002BFA04460028D4D002210C3064F011FD2E
:109640002146078042F21B00EAE700BF1DD80A004E
:109650001CF809006DDF0A0073B5C368D9789A78E1
:109660001E8842EA0122ADF8002059791A79B4B275
:1096700042EA0122ADF80220D9799A79204642EADD
:109680000122ADF804201A7A5B7A012142EA032311
:10969000ADF8063002F0D6FC054658B901211D4848
:1096A00023461D4A65F0CCFA0221204665F0ABFB4B
:1096B00002B070BD694602F00DFF38B91E21204688
:1096C00065F0A1FB284602F05FFBF1E74FF0FF30A9
:1096D0004FF0FF31FFF7D8F904460028F2D00E21F1
:1096E0000C3064F0BEFC00230680C0F80A30BDF8E0
:1096F000003021464380BDF802308380BDF804303D
:10970000C380BDF80630038142F22000FFF73CFB26
:10971000D8E700BF1CF809001DD80A0038B504219D
:1097200004460C3064F0DEFC034640885D7818B1D6
:1097300022461978FFF76EF835B1044825F03AF95A
:10974000BDE83840FFF718BB38BD00BF1801002046
:10975000B0B50446032100AF0C3064F0C3FCE268EE
:109760000346117840F63542B0F80100904217D117
:109770006C468AB06A46114BCDE90531104B079310
:1097800040F20133ADF820300E4B42F8103F002379
:109790004FF412510C48FAF797FAA546BD46B0BDF2
:1097A0001D7810B12246FFF735F8002DF6D0074896
:1097B00025F000F9FFF7E0FAF0E700BF84DF0A00C8
:1097C000BC010B00040000011CF809001801002076
:1097D00038B525F045FF314DD5F80C31002B5AD066
:1097E0000022002305F1E80025F020F9002852D1DD
:1097F0000022002305F5867025F0A6F8044668B916
:1098000040F6CC43264A2749274862F083FF84F379
:109810001188BFF36F8F0323184602DFD5F800319C
:109820007BB1224A0121224865F0F6F90022214B42
:10983000D3E8EF0FC3E8E12F0029F9D108B1FCF715
:1098400023F9204664F0C6FBC5F800012046FFF767
:1098500015FA0346C8B10121174A154865F0F0F919
:10986000164825F0A7F82046FCF76EF80C22144B9A
:1098700002FB0033588818B122461F21FEF7CAFFA9
:109880002046FCF701F9FFF777FAFFF775FABDE814
:10989000384025F0F9BE02F047FCF8E73000002020
:1098A00094D90A009DD70A00E1D90A00BCDF0A005A
:1098B0001CF80900300100205DDC0A0018010020BE
:1098C000203B002070B54FF0FF320D464FF0FF33C4
:1098D00000210646FEF7A8FB044660B91A230A4A8F
:1098E0000A490B4862F016FF84F31188BFF36F8FAB
:1098F0000323184602DF022104F10C0064F0B1FBDF
:1099000006704570204670BD20E00A009DD70A0011
:10991000E1D90A00F8B506460024094DEF79E3B213
:109920009F4202D86FF0010007E02946304665F0FB
:10993000B4FA0735631C08B12046F8BD1C46EEE7B3
:109940003000002037B504460D46B9B12846164907
:1099500065F0A3FA90B929461448C4EBC404204426
:1099600065F094FA124865F08EFA430703D5FEF7C6
:1099700093FA65F05BF8002003B030BD684665F0EF
:10998000A4F80028F8D16846FFF7C4FF0028F5DAEC
:10999000064BC4EBC4006946184465F077FA002D05
:1099A000E0D001462846DBE7333C0B0030000020C6
:1099B000B800002070B5174E06223146054685F0E6
:1099C0008BFA10B34FF0FF304FF0FF31FFF75CF828
:1099D0000446E0B1062229460C3064F048FB2146DB
:1099E000002242F20500FFF721FA044648B110F1C7
:1099F0000D0F04D10221084A084865F056FA2046A6
:109A000070BD28683060AB88B3800024F7E76FF042
:109A10006804F4E74C00002056E00A002CF8090026
:109A2000064BD3E8EFCF4CF4806CC3E8E2CF002ABA
:109A3000F7D1037A19430172704700BFB8000020C4
:109A40002DE9F341002104460222084602F092FE6D
:109A5000054648B120460121FFF7E2FF284602B043
:109A6000BDE8F04102F090B98DF8000069464E481B
:109A700000F0ACFE9DF8003033B101212046FFF725
:109A8000CFFF02B0BDE8F081484865F0FCF98106DF
:109A9000C0F3401708D5454865F0F5F9420603D5EF
:109AA00001212046FFF7BCFF0021414800F08EFE57
:109AB00017B1002001F070FA3E4D95F8DB309BB1F4
:109AC000002065F031FA78B102213B4A3B4865F04D
:109AD000ECF917B1012001F05FFA0021384802B01B
:109AE000BDE8F04100F072BE95F8DB2095F8DA3061
:109AF0009A4218D10221334A304865F0D6F9002243
:109B000042F229001146FFF791F910B101212E4AC6
:109B1000DCE795F8DB30013385F8DB30237A43F05E
:109B200004032372D5E7224604F10108414612F8E6
:109B30002E0B65F0BCF9064610B1244A01210EE057
:109B400095F8DB30013385F8DB30237A43F00403EA
:109B5000237295F85B305B0708D402211C4A174832
:109B600065F0A3F9012065F0DFF9B2E741466846E8
:109B700065F08CF901234FF0FF304FF0FF318DF885
:109B80000730FEF781FF044660B1082269460C30B9
:109B900064F06DFA3246214642F24E00FFF746F974
:109BA0000028DFD00B4AC9E711F00700B8000020F9
:109BB000E1EF07003000002065E00A002CF8090002
:109BC0005BEF07008AE00A00BBE00A00DBE00A0066
:109BD000FBE00A0025E10A002DE9F74300210446D5
:109BE0000222084602F0C6FD054648B12046022181
:109BF000FFF716FF284603B0BDE8F04302F0C4B8F3
:109C00008DF807000DF10701404800F0DFFD9DF8D9
:109C1000073033B102212046FFF702FF03B0BDE851
:109C2000F0833B4865F02FF98206C0F3401808D551
:109C3000374865F028F9430603D502212046FFF78F
:109C4000EFFE0021334800F0C1FDB8F1000F02D053
:109C5000002001F0A1F9002065F066F92E4D0646BE
:109C6000C0B1012103462D4A2D4863F0EBFD95F864
:109C7000DB3013B1012065F057F9B8F1000F02D0C5
:109C8000012001F089F90021264803B0BDE8F04326
:109C900000F09CBD95F8DB3095F8DA209A420CD2A2
:109CA000013B85F8DB30237A024623F004030220CF
:109CB0001D49237209F0DCF8D9E74FF0FF304FF06F
:109CC000FF31FEF7E1FE04F10109074668B1072103
:109CD0000C3064F0C6F9494665F0D8F8324639468A
:109CE00042F22800FFF7A2F828B101210F4A0C48E0
:109CF00065F0DBF8BBE795F8DB30013B85F8DB303E
:109D0000237A23F004032372B1E700BF11F00700A8
:109D1000B8000020E1EF07003000002040E10A0019
:109D20002CF809005BEF070013EF07006DE10A0054
:109D3000084BD3E8EF2F22F48061C3E8E01F00282E
:109D4000F7D1530504D500220220034909F090B849
:109D5000704700BFB800002059F10700002307B585
:109D60000549CDE900036A46022009F081F801980F
:109D700003B05DF804FB00BF85EF0700034610B495
:109D800070B10B4991F8DA4091F8DB200CB19442A4
:109D900009D2013281F8DB201A7A42F004021A72E9
:109DA0005DF8044B70475DF8044BFFF749BE00BFF8
:109DB00030000020034610B4A0B10C4C94F8DA1027
:109DC00094F8DB2031B101318A4204DC5DF8044BA8
:109DD000FFF702BF12B1013A84F8DB201A7A22F0B1
:109DE00004021A725DF8044B704700BF3000002077
:109DF00038B50D460649CC7938B12B689C4228BF4E
:109E00001C46C4EBC40285F039F82C6038BD00BF95
:109E10003000002070B5044611BB20B3254965F021
:109E20003CF800BB2046FFF775FD00283BDA23789D
:109E300053B92148C279002A35D1214665F026F868
:109E40000123C371104670BD012B04D1A37903F027
:109E5000C003C02B07D00121184A194865F025F826
:109E60006FF01500EFE7144DEB79012B1ED005F1D3
:109E7000880065F008F8C30707D4002CF0D020460E
:109E80000C4965F00AF80028EAD1EE792146731CE6
:109E90003046EB71FFF756FD08B93046D3E7EB7952
:109EA000013BEB71CFE76FF07700CCE76FF00B0071
:109EB000C9E700BF333C0B003000002092E10A00EC
:109EC0002CF809002DE9F341044640B91A4A022151
:109ED0001A4864F0EAFF002002B0BDE8F0810021DA
:109EE00041F2090001AAFEF7A1FF054608B1144A94
:109EF000EDE7019E0622D6F80C80124908F1010711
:109F0000384684F0E9FF28B1062238460E4984F02D
:109F1000E3FF18B93046FBF7B7FDDCE7D8F80130AE
:109F20003046C4F80130BB882570A4F80530FBF733
:109F3000ABFD0120D0E700BFC0E10A002CF809000A
:109F4000D9E10A00403C0B003A3C0B0007B56846DB
:109F5000FFF7B8FF044BD87118B169460020FFF72E
:109F6000F1FC03B05DF804FB300000202DE9F04166
:109F7000304E88B0F179002954D196F8764014F02B
:109F8000010411D12C4A02212C4864F08EFF0024D8
:109F9000F471162500240127F379E0B283422BD80F
:109FA000002B3FD000203AE06A464FF60940FEF70A
:109FB0003DFF08B1224AE6E7DDF800C0DCF80C50AE
:109FC00095F80180B8F1000F0ED0AB1C02AA123533
:109FD000174618685968083303C7AB423A46F7D1A9
:109FE000186838609B88BB806046FBF74DFDB8F170
:109FF000000FCDD1134AC6E708AB05FB003353F879
:10A00000182C33F8143C6946CDF80120ADF8053022
:10A010008DF80070FFF796FC01340028BCD008B022
:10A02000BDE8F0810021084608B0BDE8F041FFF727
:10A03000F1BE00BF30000020F7E10A002CF8090053
:10A0400023E20A0043E20A0038B50C4661B1084831
:10A050000578012D05D10130FFF7ACFC00B9257062
:10A0600038BD00200870FBE76FF01500F8E700BF6F
:10A07000300000202DE9F0411D460E4617460346EC
:10A0800048B145B10A0311D54C0708D50121284A2A
:10A09000284864F00AFF6FF01500BDE8F08165F014
:10A0A00038F80028F9D101232B70F6E7B1070478BE
:10A0B00024D021492FB1B20603D591F89020500643
:10A0C00032D5C4EBC40411F80480B8F1010F09D1F2
:10A0D00001341846214464F0B7FF0028DDD185F82B
:10A0E000008002E0B8F1000FF9D02FB1B30642BFF3
:10A0F0002B7843F002032B700020CEE7720710D5B7
:10A100000D49C4EBC4040F5D012F07D10134214474
:10A1100064F09AFF0028C0D12F70E7E7002FE5D147
:10A12000FAE764F0F6FFBEE76FF08500B5E700BF21
:10A130006CE20A002CF809003000002070B500F134
:10A140000F0604460D46072230460C4984F0C4FE33
:10A150000346207873B90522094902F00BFB044637
:10A1600058B10573002101F05BFE2046BDE8704048
:10A1700001F00ABE06223146EFE770BD333C0B000A
:10A180002C3C0B00F8B504690646456844B140F222
:10A1900003432B4039D005F48263B3F5806F34D08C
:10A1A00015F4806302D115F4F84F2ED1184F307892
:10A1B000FB79834229D9C0EBC000072215493844F6
:10A1C00084F08AFEA8B115F0030306D197F8232086
:10A1D000082A02D8B2689F2A17D915F0300F09D083
:10A1E0009CB1EB0608D405F46035B5F5603018BFB6
:10A1F0000120F8BD002CF6D1D6E902239A4204D8FA
:10A200001F2A02D9B3F1807FEDD30020F1E700BF10
:10A2100030000020333C0B0038B50E4D284664F06A
:10A22000BAFF10F0010412D1A5F118031846582204
:10A23000214684F049FE0346D5E8EF2F42F00102A3
:10A24000C5E8E12F0029F7D118465C7038BD002021
:10A25000FCE700BFB8250020F8B5044614F80F7BD2
:10A26000154B06460D4607222046144983F82270F6
:10A2700084F032FE70B93846114902F0CDF9044637
:10A2800010B96FF00B00F8BD052101F0C9FD0020E9
:10A290002C60F8E72146384602F004FA40B921461E
:10A2A000307802F0B9F904460028EAD00621ECE73C
:10A2B0006FF01500E7E700BF30000020333C0B00D3
:10A2C0002C3C0B002DE9F04F91B0154603905068DF
:10A2D000002214460691824212D1FB2C18D89F4BC3
:10A2E000B3F8D8309C421ED99D48009302212346E2
:10A2F0009C4A63F0B1FA6FF0200011B0BDE8F08F16
:10A300002968023401EBC2014B7801321C44E2E7B8
:10A31000039B082103F1180064F040FF0028DED001
:10A320006FF00A00E9E7FB2C6ED8039B0B2103F1C9
:10A33000180064F033FF10B91F2C28BF1F244FF002
:10A34000FF304FF0FF31FEF79FFB04F10408074692
:10A35000002800F0FF8041460C3063F082FE4FF091
:10A36000000906464246002184F0AEFD4946D5F874
:10A37000008006F1040B6B6899450FD3039BF170C5
:10A380005B780022337003233946737001230698EB
:10A39000B37011B0BDE8F04FFEF748BD98F801204A
:10A3A000881C13189C4298F800C013D2BCF1090F06
:10A3B000A4EB000201D1002A0ADC694801216A4AA3
:10A3C00063F037FA3846FBF75FFB6FF0150094E750
:10A3D0004FF0080C5FFA82FA0AF101030BF8013022
:10A3E0000131C9B20BF801C0C3B2D8F80410584407
:10A3F000049384F043FD049B09F101099A445FFA38
:10A400008AF108F10808B6E7002110220CA884F0B0
:10A410005BFD0027012340F272600B933B466968A5
:10A420000A958B4207D100240123A046A346059339
:10A430005FB9384661E72A68023702EBC3025278F7
:10A4400017448742C1D80133EBE7FB2F4FF0FF30B1
:10A450004FF0FF31BA4628BF4FF0FB0AFEF714FB5E
:10A460000AF104060490002874D031460C3063F0E1
:10A47000F8FD039B81465B78002603704FF00003D4
:10A480005FFA8AF283700792031D55F83B2005EBB3
:10A49000CB0102EBC80252780232944209D14A68D9
:10A4A00008F10108904509BF00240024A0460BF1E3
:10A4B000010BBBF1010F12D055F83B204FEAC80148
:10A4C00012EBC80C0BD09819FCB901249CF80120A0
:10A4D00001329A550136F6B2079AB242D5D8059B99
:10A4E000BF1B002B31D0002F0CBF03230123002200
:10A4F0000499069889F8036089F80130FEF796FC04
:10A5000000287FF4FAAE059092E7012C05D1525C49
:10A51000013602240270F6B2DEE79CF80120AAEBB5
:10A520000601121B02328A4228BF0A46DCF804C028
:10A53000A11E61440993089284F0A0FC089A099B2B
:10A5400014443244A4B2D6B2C6E7B7FA87F35B0923
:10A550005B00CCE76FF06800CFE600BF3000002062
:10A56000B4F7090091E20A00BFE20A002DE9F347BF
:10A570000F690D46496890463A1E18BF01224C02E9
:10A580000646016505D5EB787F33DBB2932B00F2ED
:10A59000048130460DF10303FFF76CFD04460028EB
:10A5A00040F0E88006F10F03002F00F0E7802A69F1
:10A5B00011684FF0FF30C6F80F109188998092799A
:10A5C0004FF0FF319A71FEF75FFA8146002800F0E4
:10A5D000E78019210C3063F044FD04460021192264
:10A5E00084F072FC73782370AB68E370C3F30722C6
:10A5F0001B0C22716371EB68A371C3F307221B0C60
:10A600002372E2716A6812F4004F14BF0623072315
:10A61000D00348BF03F00503910348BF03F0FB03D9
:10A6200063729DF80330A3726B685A0254BF7F2394
:10A6300095F90330E374012323756B6803F44063D9
:10A64000B3F5806F14BF01230223A3756B68DB048D
:10A6500042BF03232375A3756A68C2F3802383F086
:10A6600001031B0150049BB248BF43F04003910417
:10A6700048BF43F02003D20544BF012222766A6816
:10A6800090077DD043F0010A1FB9510501D443F072
:10A69000030A900502D4B8F1000F03D04AF0020A71
:10A6A0001FFA8AFA002F6DD0D1062A6948BF4AF0F6
:10A6B0000403116858BF4AF00C03C4F80B109188CA
:10A6C0009BB2A4F80F10927962746A7801AFE275B8
:10A6D000AA7849466275A4F801303A4642F236003B
:10A6E000FEF7A4FB0446002844D1019BDB6893F9E4
:10A6F0000130B370D7E8EF0FC7E8E34F002BF9D173
:10A7000008B1FBF7C1F906F11807D7E8EF3F43F0AE
:10A710000203C7E8E23F002AF7D16FF01001384684
:10A7200064F043FDC2062FD46A68092112F00302C7
:10A7300018BF0122384664F043FD0A213846CAF3A7
:10A74000400264F03DFD2A790C213846C2F38002B4
:10A7500064F036FD6A790B213846C2F3800264F05A
:10A760002FFD9DF803200321531E5A4238465A41BB
:10A7700064F026FD204602B0BDE8F0870A4A17E7DC
:10A780009A4686E75346A0E7304606F1090164F091
:10A790005BFC0028C8D00446ECE76FF01504E9E73D
:10A7A0006FF06804E6E700BF333C0B0008B520B942
:10A7B000044864F0F0FCC30701D4002008BD02483F
:10A7C000FCE700BFB8250020A0250020034610B5F7
:10A7D000044864F0E0FCC20703D5BDE8104002481D
:10A7E000184710BDB8250020A025002010B5054C45
:10A7F000A06930B16FF00101183064F0D6FC00237D
:10A80000A36110BD3000002010B5164B9C693CB907
:10A810000121154A154863F00CF80024204610BDAC
:10A82000204664F053FD04F118020821104664F03C
:10A83000B5FC10B9FFF7DAFFEFE70921104664F025
:10A84000ADFC18B100212046FFF778FC002220461D
:10A85000114664F0F6FC04460028DFD1FFF7C6FF7E
:10A86000DCE700BF30000020D8E20A00B4F709009E
:10A8700010B50A4B20389B6983420AD1FFF7C4FF09
:10A88000034648B1BDE810400221054A054862F080
:10A89000D9BF64F01EFDF3E710BD00BF30000020FB
:10A8A0000FE30A00B4F709002DE9F04FDFF888B193
:10A8B0000646DBF818400F469046994685B0002CB6
:10A8C00040F09E80FFF7A8FC0546CBF81800002852
:10A8D00000F099800BF18800D6F810A0ADF8084080
:10A8E0008DF80A40039464F056FC410774D57368F0
:10A8F0005A0574D432690AB19B0770D03046FFF70D
:10A9000041FC00286BD005F1180B0821584664F073
:10A9100045FC002866D1434864F03DFC440501D560
:10A92000FFF706FA3378B9F1000218BF0122314669
:10A9300028462B70FFF71AFE044660B9BAF1000FE3
:10A940000CD10E9B4246009339464B46284664F094
:10A95000EBFC044680B1FFF749FF33E07368D8068B
:10A960000AD48023ADF80830DBE8EF3F43F08003E2
:10A97000CBE8E23F002AF7D17368990716D101218D
:10A98000284602AA64F05DFC0446B8B10121264ABB
:10A99000264862F04EFF039E002EDCD03046002198
:10A9A00001F03EFA304601F0EFF9D4E7284603A95A
:10A9B000FFF752FC04460028E1D0CCE7039808B129
:10A9C00001F0E2F93946002340F2011098450CD11C
:10A9D000204605B0BDE8F08F6FF00A04BBE76FF0CA
:10A9E0001504B8E76FF07704B5E70A88824204D10E
:10A9F0004A6812B11278D20708D401330831E5E76A
:10AA00006FF07704E4E76FF00B04E1E720352846A8
:10AA1000074968F094FF00232846064A24F0A0FA6C
:10AA2000D6E700BFB8000020F4E20A00B4F709003E
:10AA300071A801001C4E0E00300000202DE9F341EA
:10AA4000C6687078FFF7B2FE044638B90121364A6D
:10AA5000364802B0BDE8F04162F0EBBE04F11808E0
:10AA6000758864F033FC6FF48071404664F09DFBA0
:10AA700033782F4F1BBB2846012101F0E3FA05462E
:10AA800050BB6FF08001404664F08FFB03060ED58B
:10AA9000204664F057FBFFF74BF963683BB11B6836
:10AAA0002BB1327920468DF8042001A99847BB6963
:10AAB0009C4235D102B0BDE8F041FFF797BE0921B5
:10AAC000404664F06BFB18B120463178FFF736FB47
:10AAD0003378002BD5D1CEE7236D00F17E0213F43D
:10AAE000002F12D0A368C0F87E30A3899380A37B87
:10AAF000937163682BB15B681BB12046019501A976
:10AB00009847284601F040F9BBE7037AC3EBC3033B
:10AB1000F918FB58C0F87E308B8893808B79E7E773
:10AB200002B0BDE8F08100BF2EE30A00B4F70900CF
:10AB3000300000207FB5C5682878FFF737FE04464F
:10AB400038B90121134A144804B0BDE8704062F0DE
:10AB500070BE43688BB19B687BB10135284663F0BA
:10AB6000CDFF02AE294650B1304663F0BCFF6368AA
:10AB700020469B68019601A9984704B070BD2078D3
:10AB800064F056FA0346006802909A889B79B28076
:10AB9000B371ECE72EE30A00B4F70900034B1A7A0D
:10ABA000012A04BF02221A72704700BF5D8800208C
:10ABB00008B5094868F0D1FE031E04DA0121074AEE
:10ABC000074862F03FFE0022064B99689A801960A0
:10ABD000054B1A7208BD00BF7801002042E30A004D
:10ABE0004CF80900B00400205D880020F0B505464F
:10ABF0000F464FF0FF304FF0FF3187B01646FDF79C
:10AC000043FF0446C0B106210C3063F02AFA4680A7
:10AC100000264770057006714671094A204603A94F
:10AC200005230095FDF71EFF3246214642F2420001
:10AC3000FEF7FCF807B0F0BD6FF06800FAE700BF60
:10AC4000B800002038B50546407A0C46FDF744FFB1
:10AC50002073A87AFDF740FF607395F90C30A3715B
:10AC600095F90D306371EB7A2371EB8963812B8841
:10AC7000103BDBB20B2B8EBF0523054AD35CE3717F
:10AC80002B8883F0100303F01F03238138BD00BF1E
:10AC9000B43C0B0008B50C4B0246400903EB8000A6
:10ACA00064F06EFB02F01F0340FA03F313F001009F
:10ACB00006D122B9054864F063FB40F3C01008BD1B
:10ACC0006FF07700FBE700BF483B0020B800002092
:10ACD0002DE9F04788B0002200238E4823F072FD52
:10ACE0000646002840F0CB808B4864F049FB10F00A
:10ACF000010F894D7ED02B1D93E8070008AB03E9B7
:10AD00000700864864F03CFBC0F34013824864F0BF
:10AD100037FB0446002800F0A3808BB10C22804949
:10AD200005A884F0D9F80446002800F0A480002289
:10AD300011461046FFF75AFF0446002840F09B805A
:10AD4000764864F01DFB410501D5FEF7F1FF9DF843
:10AD500015502A0757BF9DF8143000278DF804308E
:10AD6000BDF816305FBF01AFADF80530BDF8183043
:10AD7000ADF8073015F0040500F0C880BDF81C20C0
:10AD80000AB9BDF81620BDF81E300BB9BDF8183051
:10AD90009DF81410ADF80D208DF80C10ADF80F30A3
:10ADA00003AD002F6FD03B78012B71D0002D6AD1FD
:10ADB0000025BDF81A3006F0010043B1574BD3E827
:10ADC000EF1F41F04001C3E8E21F002AF7D10DF167
:10ADD000030164F0D1F9044600284CD14FF0FF3054
:10ADE0004FF0FF31FDF750FE8046002852D16FF042
:10ADF000680440E0494864F0C3FA10F0800F494A03
:10AE00000ED09089D18913694FF48072ADF8160085
:10AE1000ADF81420ADF81810ADF81A60079370E77C
:10AE2000414C05AB2068616803C3A068186092F8C4
:10AE3000913039481F0744BF05238DF8153064F061
:10AE40009FFA840706D53023ADF818306023ADF89B
:10AE5000163056E7304864F093FA4007F3D450E7D1
:10AE60004BB102460146FFF7C1FE044618B92C4B10
:10AE70002861C3E90100274823F016FD2646304625
:10AE800008B0BDE8F0872E78731E5E425E4190E701
:10AE90001E468EE700F10C090321484663F0E1F8F5
:10AEA0009DF803309DF815A00370CAF340030646D1
:10AEB0008470437037B101230522837039464846B8
:10AEC00063F0D5F845B1B378052243F00403294671
:10AED0004846B37063F0CBF80022414642F241008D
:10AEE000FDF7A4FF04460028C5D10120BDF81A20B3
:10AEF0000AF00101FFF77AFE04460028BBD1084B97
:10AF000008AA12E9070083E80700B4E7002F7FF4DE
:10AF10004AAF4DE7643B0020483B0020B8000020CA
:10AF2000583B0020300000206CFA0900002347F64F
:10AF3000122210B5064824F013F8031E06DABDE805
:10AF400010400121034A044862F07CBC10BD00BFE0
:10AF5000780100206FE30A004CF809000022024B40
:10AF60001A60FFF725BE00BF943B002010B54422B5
:10AF70000021084883F0A8FF064B03F11C001C4683
:10AF800068F0E0FA04F1300068F0DCFABDE8104047
:10AF9000FFF7E4BF483B00200022044B801A597C95
:10AFA00018BF012001F00101FFF720BE483B00203F
:10AFB000032870B5054603D1BDE87040FFF788BE91
:10AFC000FFF768FE0446B0B9012605F01F039E4056
:10AFD0000A4B6D0903EB8505D5E8EF3F3343C5E820
:10AFE000E23F002AF8D1FFF773FE044618B1F1439F
:10AFF000284664F0C8F9204670BD00BF483B0020D9
:10B00000032808B50AD0012100F01F039940054B21
:10B010004009C94303EB800064F0B5F9BDE808407E
:10B02000FFF756BE483B00202DE9F74F05465E4826
:10B0300064F0A6F900F001085B4864F0A1F90E463F
:10B04000144699468246B8F1000F03D00B895A077F
:10B0500000F1A680284663F051FD6F46002868D0B5
:10B060002946684663F03FFDB8F1000F02D11AF09F
:10B07000040F28D14D4BD3F800B0BBF1000F13D013
:10B080002268A368B4F804A0A4F80490A2EB030813
:10B0900038462346F27996F90510D847A368A4F8F4
:10B0A00004A013FA88F32360414B37601A6842B159
:10B0B00052F80889B8F1000F01D0A8F10808002A59
:10B0C00047D1002333603848338964F059F910F0D0
:10B0D000010665D1DB0763D503223946304601F00E
:10B0E00049FB044600285BD00220FFF789FF2B684C
:10B0F0002046C4F87E30AB88A4F88230AB7984F85F
:10B10000843063F0F7FD002843D01F2331462373BA
:10B11000204600F085FE204600F036FEFFF7D8FD01
:10B12000034600283CD00221224A234862F08AFBD1
:10B1300036E02B78FF2B07D1204B186800909A88B7
:10B140009B79BA80BB718FE7294663F071FF034694
:10B15000F3E713688BB12168A368B4F804B0A4F8CE
:10B160000490A1EB030A3046136821469847A36870
:10B17000A4F804B013FA8AF32360B8F1000F06D0E4
:10B18000D8F8083003B1083B4246984697E7434653
:10B19000FAE72046022100F043FE204600F0F4FDCD
:10B1A00003B0BDE8F08F00BF483B0020943B002077
:10B1B0008C3B0020F7D70A004CF80900333C0B0009
:10B1C00010B50020FFF71CFF58B168F036FC0020D6
:10B1D000FFF716FF034620B10221124A124862F01F
:10B1E00031FB6FF04001114864F0CDF86FF48071CD
:10B1F0000E4864F0C8F8FEF79BFD0D4B1B6823B1A9
:10B2000053F8084904B1083C03B910BD5B6803B1A9
:10B2100098472CB1A26802B1083A23461446F3E7D6
:10B220002246FAE7A0E30A004CF80900B800002023
:10B230008C3B00202DE9F04F00F10C0989B0074646
:10B24000484662F057FF06465D4864F099F800F002
:10B2500001035B48039364F093F85A4DC0F38003F5
:10B26000DFF874A102939EB1039B53B13B8A172B65
:10B2700011D80121544A554809B0BDE8F04F62F099
:10B28000D8BA2B7A0BB1FFF793FC029B002BEDD1C0
:10B2900009B0BDE8F08F1821484662F023FF3A8AD2
:10B2A000C37DB0F800B09342CBF3411804460BF0D5
:10B2B000100B0FD9454800920221454A62F0CCFAA2
:10B2C000384662F040FEBBF1000FE1D102223D4B57
:10B2D0001A72DDE7BBF1000F0DD004A9FFF7B2FC35
:10B2E0004A46E37D04A9A01CFFF79EFE4846E17D87
:10B2F00062F0F0FE29E095F808B0BBF1000F37D0FE
:10B30000C27AEB799A4205D1811C0722284683F044
:10B31000E3FD48B3B8F1000F02D1204604A9DDE7F0
:10B32000BBF1010F27D102212A4A284862F081FA95
:10B33000DCE72B7A022B3DD05046F96862F097FE8D
:10B34000B8F1010F04D1FFF7F1FD013EF6B28AE733
:10B35000204604A9FFF776FC5246BAF8043004A947
:10B36000A01CFFF761FE28E0B8F1020F18D124E01D
:10B37000B8F1000FD1D0B8F1020F1ED0BBF1020F0F
:10B3800001D1FFF715FCD4F80220E37A2A60E288A5
:10B39000EB710123AA80227A2B72AA71FFF7C6FDF6
:10B3A000E27DBAF80430BAF8061013448B42C0DDCF
:10B3B00002232B72B8F1010F98D0FFF7F9FB95E744
:10B3C000483B00205D880020C9E30A004CF80900D2
:10B3D000E2E30A000CE40A00B00400202DE9F04F7B
:10B3E00000F10C0785B00646384662F083FE05463C
:10B3F0002A4863F0C5FF00F00109284863F0C0FF48
:10B400004FF0010ADFF8A0B0C0F3800815B905B00D
:10B41000BDE8F08FB9F1000F02D1B8F1000FF6D0FE
:10B42000338A082B07D801211D4A1E4805B0BDE804
:10B43000F04F62F0FEB90921384662F053FE037AFC
:10B44000328A01339A420446EDD37F23ADF80CA033
:10B450008DF80630037A694603445B7A01308DF833
:10B460000530FF238DF804300023ADF80A3010F8C2
:10B47000012C013D042A98BF1BF802308DF80720EB
:10B48000ADF80830C3793A46FFF7CEFD217A384649
:10B49000013162F01FFEEDB2B8E700BF483B00206B
:10B4A000C9E30A004CF80900C03C0B00F8B505469A
:10B4B000224863F065FF43070F463CD52A78012AEE
:10B4C00003D96FF015042046F8BD6B780F2BF8D820
:10B4D00043F6FC746888031F9BB2A342F1D8A98885
:10B4E0000B1F9BB2A342ECD88842EAD37AB9002260
:10B4F0000023134823F066F904460028E3D1FFF740
:10B50000C9FB044640B10E4823F0CEF9DBE763F0F7
:10B5100017FE0028EBD1D4E728686968094E0A4B6A
:10B5200003C6A8681F6030602046FFF741FD04464F
:10B5300006F12400E8E76FF00A04C4E7B800002031
:10B54000783B00204C3B0020943B002008B5FFF7DF
:10B5500005FD00220A4B6FF040010A481A6063F0B3
:10B5600012FF430606D56FF48071064863F00BFFA7
:10B57000FEF7DEFBBDE808400020FFF741BD00BF3D
:10B58000943B0020B80000200A4A00F1080311682B
:10B5900031B98160516839B9C2E900330020704780
:10B5A0008B4204D00968F3E70B605360F6E76FF055
:10B5B000100070478C3B002008B5034863F0E0FEA4
:10B5C00000F0010008BD00BF483B002070B59AB0F4
:10B5D0001422002104A883F077FC47F21213ADF87F
:10B5E0000C304FF4807344F20102ADF80E30364B4C
:10B5F00001A903A8CDE905235AF0ACFA034618B314
:10B60000324A0121324862F01DF91F25314BD3E83F
:10B61000EF1F21F00101C3E8E21F002AF7D12E4EEF
:10B6200024F01EF8346804B1043C002D2B4D18BFE3
:10B630000025002C41D023680BB128469847646848
:10B64000002C3AD0043CF6E702AB4122019809A94C
:10B6500082F0D0FA034608B1214AD2E7214A0DF11F
:10B6600025030DF1650153F8040B8B4242F8040BDE
:10B67000F9D102AB20221C49019882F063FA0346FB
:10B6800008B11A4ABDE7019882F014FA054610B1D4
:10B69000174A0346B5E71349104863F07FFE154883
:10B6A000203163F07BFE144BD3E8EF1F41F0100113
:10B6B000C3E8E21F002AA9D0F6E70023C6E9003359
:10B6C00023F0E2FF1AB070BD0000020931E50A0064
:10B6D0000CF80900983B0020A03B0020AB8900201B
:10B6E0004FE50A006B8900204B89002072E50A00B3
:10B6F00096E50A00CB890020B800002030B5A7B03D
:10B700001422002108A883F0DFFB04233D2200213E
:10B7100016A8159383F0D8FB47F21213ADF81C302E
:10B720004FF4807344F20102ADF81E30284B2949D2
:10B73000CDE9092307A805AB202282F085FA03464C
:10B74000E0B1254A0121254862F07CF86FF004043D
:10B7500023F086FF224B1D6865B100201860214B45
:10B76000D3E8EF1F21F00201C3E8E21F002AF7D15E
:10B7700044B3A84723F088FF27B030BD1A4B0DF122
:10B780005502194603F1400053F8044B834242F836
:10B79000044BF9D106AB029320230D48CDE90013E9
:10B7A00015AA4123059982F022FC034608B10F4AED
:10B7B000C8E7059882F07EF904460028C8D00C4AF4
:10B7C0000346BFE70DA8084963F0E8FD0DA8D0E7E0
:10B7D000000002094B890020B6E50A000CF80900B8
:10B7E0009C3B0020983B00206B890020ECE50A0080
:10B7F00008E60A00402208B5034983F06DFBB0FA61
:10B8000080F0400908BD00BFC53C0B0010B598B0E2
:10B8100004461422002102A883F056FB44F21213BE
:10B82000ADF804304FF480734FF48042ADF8063029
:10B83000144B2146CDE9032304230DF11D008DF89F
:10B840001C3063F0ABFD04F120010DF13D0063F00D
:10B85000A5FD6B46412207A901A882F0F5F904462F
:10B8600001A882F0EAFC2CB9009882F023F90120AB
:10B8700018B010BD044823460121044A61F0E2FFDC
:10B880000020F5E7000002090CF8090025E60A008F
:10B8900010B5002834D01D4A136823B1043B9842E8
:10B8A00031D05B68F9E71A4BD3E8AF1F890707D59A
:10B8B00018480221184A61F0BCFF6FF00F0010BD5C
:10B8C0001468011D44605068116000B95160D3E8EC
:10B8D000EF2F42F00101C3E8E01F0028F7D1D307A2
:10B8E00001D50020EBE70D4BD3E8EF1F21F010014D
:10B8F000C3E8E21F002AF7D10948FCF709F9F0E78D
:10B900006FF01500DBE76FF07700D8E7A03B002071
:10B91000983B00200CF8090049E60A00B800002016
:10B92000CC040020044BD3E8AF3F13F0100F0348C2
:10B9300008BF0020704700BFB8000020AB8900207E
:10B9400070B50546194803688B4228D0184BD3E8D8
:10B95000AF3FDA0626D5036813B16FF00F0070BD54
:10B96000144AD2E8AF3FDB07F7D4D2E8EF3F43F009
:10B970000204C2E8E64F002EF7D113F00204ECD126
:10B98000016029460C4863F009FD0C4805F12001CF
:10B9900063F004FD0A48FCF7BBF82046DFE76FF0D0
:10B9A0007700DCE76FF07C00D9E700BF9C3B00200C
:10B9B000B8000020983B00206B8900208B89002074
:10B9C000BC04002070B505460B4B1C6844B154F80C
:10B9D0001C3C1C3C13B12846297B9847E469F5E7D9
:10B9E000064C074EB44200D370BD236813B12846FD
:10B9F000297B98472034F5E7DC3B002064F70900F9
:10BA0000A4F7090010B50446F9F79EFF044901EBBD
:10BA10000011204663F0B3F8BDE81040FDF7ACB963
:10BA2000A83B0020002270B50446D1E90156074822
:10BA3000C1E9012267F043FE3DB1314620462B4665
:10BA4000BDE870406FF06D02184770BDB816002059
:10BA500030B5051D04464FF48061284685B063F07B
:10BA6000C7FC400533D4284663F0BDFC810321D5D3
:10BA7000E17871B3637B072B29D1224B93F8903087
:10BA80009B0624D563F00BF908B30DF10E0103A852
:10BA9000FDF776FAD8B92046BDF80E20BDF80C1097
:10BAA00063F069F9034690B10121174A174863F022
:10BAB0009DFC0CE0204663F043F9034620B10121D0
:10BAC000134A124863F092FC637B072BD0D005B079
:10BAD00030BD0C4B93F89130DA0706D40223194697
:10BAE0000C4A0A4863F082FCC4E7022320461A4647
:10BAF000009163F05FF903460028BBD00121064A9C
:10BB0000EFE700BF30000020C8E60A00CCF70900CC
:10BB100077E60A0098E60A00B1E60A0070B5054625
:10BB2000002200230E4822F081FFB8B90D4B1C689B
:10BB300034B154F8143C1C3C03B19847E469F7E76E
:10BB4000094C0A4EB44204D32846BDE8704023F0A5
:10BB50005FB9A36803B198472034F3E770BD00BF15
:10BB600094160020DC3B002064F70900A4F70900CC
:10BB70002DE9F041044620270025EFF3118287F3D9
:10BB80001288BFF36F8FE16929B1206A0B68814287
:10BB9000E36108BF236282F31188BFF36F8F71B135
:10BBA000D1E901680748C1E9015567F088FD1EB178
:10BBB000002241462046B047FDF7DEF8DDE7BDE84C
:10BBC000F08100BFB81600200348B0F8BC30C03088
:10BBD000002B08BF002070473000002030B504461D
:10BBE000F9F79CFB0D460D4A0D498BB00858D2F869
:10BBF000E010884205D120460BB0BDE83040FFF789
:10BC0000B7BF24342146104667F067FE1DB1694670
:10BC1000204667F072FE0BB030BD00BF40310020FF
:10BC20000800000038B5002204468A4202D10024F0
:10BC3000204638BD012004F1C803D3E8EF5F002D92
:10BC400004D1C3E8EC0FBCF1000FF6D102D0D03420
:10BC50000244EAE7002CEAD0C8220021204683F003
:10BC600033F904F14000044967F069FE034904F127
:10BC7000240067F007FEDBE7B1CA010013F40700F8
:10BC8000F7B516460D4601210446FFF7A7FF012E22
:10BC900023D0022E52D123693BB135480121354AC8
:10BCA00061F0C7FD204663F0D2FB25612269138A4B
:10BCB000012B5AD9D2681288043292B2934254D3DB
:10BCC00043D9012100922A482B4A61F0C5FD204644
:10BCD00003B0BDE8F04063F0BABB206940B9274A21
:10BCE0003146234861F0A5FD204663F0B0FB01E03A
:10BCF0002A8A2AB9284603B0BDE8F040F9F7C4BE45
:10BD0000018A438A47695B1AC168C91B5B1A9A4258
:10BD10000CD91B4A3146164861F08BFD00222046A3
:10BD2000216901F0A7F900232361E3E7E9680C30FA
:10BD300062F09DF92846F9F7A7FEB7E701213346DF
:10BD4000104A0B4863F052FBCEE7002204F11003C7
:10BD5000D3E8EF1FC3E8E02F0028F9D101222046E5
:10BD600003B0BDE8F04001F085B903B0F0BD00BFFD
:10BD7000CCF70900E4E60A0064E70A0001E70A00DC
:10BD80001FE70A0046E70A0008B500F1C803D3E838
:10BD9000EF2F013AC3E8E12F0029F8D1AAB90B4BE4
:10BDA000984212D303F1D00290420ED2C01AD0238F
:10BDB000B0FBF3F203FB120038B9054822F0FAFD9C
:10BDC000BDE80840034823F023B808BDF82500204B
:10BDD00094160020EC04002010B5044663F046FBE6
:10BDE00023F03EFC0C4B04F1BC01D3F8DC3043B92A
:10BDF0000A4863F0DDFA23F047FCBDE81040FCF789
:10BE0000BBBF994201D01B68F1E723F03DFC2046FF
:10BE1000FFF7BAFFF1E700BF300000200C0100205F
:10BE2000F8B5457B04468D420E4600AF1CD1082D67
:10BE300098BF694B6C4688B094BF53F82530674B68
:10BE40006A466749CDE905134FF40073ADF81C301D
:10BE5000644B42F8103F00234FF4E4516248F7F777
:10BE600033FFA546BD46F8BD4173DDB1022D1CD0A0
:10BE7000637B082B00F2AD8001A252F823F000BFD3
:10BE8000DFBE010079BF010049BF010065BE0100AE
:10BE900065BE010065BE010065BE0100B9BE0100BE
:10BEA00065BE010063F0E2FAE2E78378012BDFD19F
:10BEB000403067F052FDDBE70023C4E90D33E3783F
:10BEC000012BCFD1A378494A012B04BF032384F867
:10BED0009830002304F1400023F00AF8C2E7082D4F
:10BEE000C0D8DFE805F02A0521172626212A2A00D6
:10BEF00004F14005284667F030FD01212046FFF798
:10BF00006DFE204663F0A3FA00220023284623F0AA
:10BF100027F8A7E70220FFF773F8034620B10221B4
:10BF2000334A314863F062FA237B13B12046FFF7AE
:10BF300049FD2046FFF728FF94E733462D4A0221AA
:10BF4000294863F053FA8DE7A378012B8AD12A4B55
:10BF50009D8A002D86D00A2340F2E730002147F663
:10BF600012265D434FF47A720023E5FB0601F4F7D5
:10BF7000A5FF02460B46ADE7237B3E2B0FD16D4656
:10BF800088B06A461D4BCDE90534032342F8103FC3
:10BF900000234FF4C4511448F7F796FEAD46164DF2
:10BFA00005F1C006616911B9FCF7E6FE5AE7A2691E
:10BFB0000B68914208BFA36120466361FFF732FD21
:10BFC000B5F8BC30002B14BF3046002022F0F2FC44
:10BFD000E8E70B4A3346B2E79C000A007FE70A0015
:10BFE00089E70A0003000001CCF709005A62020049
:10BFF0009AE70A00CBE70A0030000020E2E70A00D7
:10C0000009E80A00F8B5074609480D46164663F0E8
:10C010002DFA044650B183781F4203D1BDE8F840A1
:10C02000FFF7B2BE3146A8472046F7E7F8BD00BF8C
:10C03000F8250020002201200149FFF7E3BF00BFDF
:10C0400007F4070070B505460E480E4663F00EFA79
:10C050000446A0B1437B012B02D0073B012B0CD837
:10C060002388AB4208D1A3781E4209D102212B4676
:10C07000054A064863F0BAF92046FFF785FE00241A
:10C08000204670BDF825002025E80A00CCF70900FD
:10C09000034BC01A034B00115843C0B2704700BF96
:10C0A000F8250020C54EECC470B51C461443054667
:10C0B0000E460DD0F9F732F90E49D1F8E0400E499D
:10C0C00009588C4206D102210C4A0D4861F0B1FB9F
:10C0D000002213460B49002D14BF2846084661F084
:10C0E00037FF044618B1711D0C3061F0AFFF2046D8
:10C0F00070BD00BF40310020080000003CE80A008D
:10C10000CCF70900D016002010B50446054822F0EF
:10C110007FFE204600F0A8FE2046BDE81040FFF755
:10C1200051BC00BFDC0400202DE9F04F002387B094
:10C1300000AFFB607B61B94B5A8B3AB1B84DD5F873
:10C14000DC403CB91C37BD46BDE8F08F1B68002BB6
:10C15000F4D1F7E754F8BC3903B1BC3B0026B14930
:10C1600001E01C461346B5F8BC20002A00F05481BB
:10C17000D5F8C8204AB904F1BC06002BE2D0D3F8A8
:10C18000BC20002AEDD0BC3AEBE70A68002AF2D0C6
:10C19000D4F8A820002AEED0D4F8AC20002AEAD0A7
:10C1A000D4F8B020002AE6D0637B072B6AD1204662
:10C1B0009047002866D004F1C00063F014F902280B
:10C1C00060DC204663F052F904460028BAD0637B55
:10C1D000072B40F01E812046D4F8A830B5F8BC10DB
:10C1E00007F1100298478146002800F00581B5F854
:10C1F000BC203B699A4208D30146D4F8AC60204683
:10C2000007F1140307F10C02B0477B69D7F80C80E3
:10C210003B60B9F81030002B00F0F5804846D7F8A5
:10C2200010A062F0C2FC7860002840F0EF80B5F802
:10C23000BC30DFF800B2002B14BF584600200022AB
:10C24000002322F0F3FB78B900220023754822F086
:10C250007BFB064600283BD1B5F8BC30002B18BF4D
:10C260005E46304622F0A6FB6FF00B054846F9F714
:10C270000BFCB8F1000F00F0AA802A46204639686E
:10C28000C047A4E0D4F8BC3004F1BC02C6B9D5F86C
:10C29000E010C5F8DC308A4201D1C5F8E030002357
:10C2A0002046C4F8BC30D4F8B030984700288ED06F
:10C2B000637B072B40F0AD802046FFF78DFD86E7BE
:10C2C0003360D5F8E0309A4208BFC5F8E060E6E791
:10C2D0003B68C0F804808360B5F8BCB00022DA4542
:10C2E0004FF000034FF000014C4898BF1FFA8AFB43
:10C2F000F9F74CFB804650B1F9F726FB4A4B5A46FA
:10C3000003EB00134946404662F014FC8046B5F842
:10C31000BC3094F8C4909A4584BF01237B607B684D
:10C320009CBF09F102095FFA89F984F8C43004F16D
:10C33000C00ADAE8EF3F0133CAE8E23F002AF8D149
:10C3400004F1140B3146584663F032F8A378012B00
:10C3500056D108F10C03042118467B6061F0A9FE58
:10C36000228809F0FD0942EA09320280B8F810205B
:10C370007B68043A42800221184661F0A2FE4046E2
:10C38000FCF77CFC8146002843D0DAE8EF3F013B14
:10C39000CAE8E23F002AF8D13146584663F03CF83B
:10C3A000224A4B460121224863F020F84046F9F723
:10C3B0006BFB20463146FFF735FBB5F8BC301D4816
:10C3C000002B08BF002022F0F5FA6FF004056E463E
:10C3D00088B0194A0423CDE905256A46079442F836
:10C3E000103F4FF4015112480023F7F76DFC132161
:10C3F000B546204663F051F82046FFF7C5FCA1E69C
:10C400006FF01509C1E76FF079052FE76FF00405AC
:10C410002CE7FCF7B1FCEFE79368FFDE5417002030
:10C4200030000020B8160020A83B00205DDC0A0088
:10C43000CCF70900F000002065E80A0040F2E24372
:10C440002DE9F041D0F888600446B6FBF3F6031DF1
:10C45000184662F0C8FF8204B6B213D5B4F88C2037
:10C46000B2420FD8B4F88E20B2420BD3D4E92412D2
:10C47000914207D1D3E8EF1F21F40051C3E8E21F36
:10C48000002AF7D1104B1D6865B155F80C7C1C3D96
:10C4900037B131462046B4F89230B4F89020B8470E
:10C4A000ED69F1E7094DDFF82880454501D3BDE886
:10C4B000F0812F6937B131462046B4F89230B4F894
:10C4C0009020B8472035F0E7DC3B002064F70900F6
:10C4D000A4F709002DE9F041074608460D4662F031
:10C4E000E0FB064618B900263046BDE8F081144B43
:10C4F0001C6884B154F8103C1C3C0BB9E469F8E7A3
:10C500002946384698470028EDD0284662F0C9FBF6
:10C510000028F3D1E7E70B4CDFF82C804445E3D249
:10C52000E3680BB92034F9E72946384698470028D4
:10C53000D9D0284662F0B5FB0028F3D1D3E700BF7D
:10C54000DC3B002064F70900A4F709002DE9F04165
:10C55000C37804468BB900F17E06114B1D687DB18E
:10C560001C3D04F170076B691BB13A463146204609
:10C570009847ED6925B11C3DF5E700F17706ECE73A
:10C58000084D094F04F17008BD4201D3BDE8F081A8
:10C590006B691BB142463146204698472035F3E788
:10C5A000DC3B002064F70900A4F70900F8B5437AE2
:10C5B00004468372164663F042F9144B1D684DB170
:10C5C00055F8043C1C3D1BB132462046617A984721
:10C5D000ED69F4E70E4D0F4FBD420DD3A6B9637A56
:10C5E000012B11D9A378012B0ED1207A04F170010F
:10C5F000BDE8F84006F0ACBEAB691BB13246204640
:10C60000617A98472035E7E7F8BD00BFDC3B0020A2
:10C6100064F70900A4F7090038B505460C460F4831
:10C620000121FFF7FFFAC0B1057223680367A388F1
:10C63000A0F87430A37980F87630012343728372B6
:10C640008370074BC0F8A830064BC0F8AC30064BDF
:10C65000C0F8B030054BC0F88C3038BDF82500204C
:10C6600069CD0100D1F30700C5F3070018002800C9
:10C6700070B505460A480E4662F0F8FE044620B141
:10C680008378012B04D0FFF77FFB0024204670BD88
:10C690003246294662F0F5FF0028F7D12046F2E73E
:10C6A000F8250020F0B589B000AF0D46FFF7E0FF98
:10C6B000044618B329463846FBF794F9637B6D4668
:10C6C000082B98BF0F4A8AB094BF52F823300E4B04
:10C6D0006A46CDE907730D4B0D4909930D4BCDE922
:10C6E000051442F8103F00234FF442510A48F7F76F
:10C6F000EBFA2046AD46FFF747FB01202437BD4645
:10C70000F0BD00BF9C000A007FE70A00010302049D
:10C7100088E80A0005000002CCF7090038B5044695
:10C72000134862F060FE420702D46FF00A0038BD81
:10C73000084662F0B6FA10B96FF01500F7E7FEF799
:10C740003BFF0028F1D10A4862F04DFE0306C0F31A
:10C75000C0150AD462F0F4FC0028EDD0214628462A
:10C76000FFF7A0FF0028E2D0E6E76FF07700DEE7F2
:10C77000B8000020F8B505460E480E46174662F090
:10C7800075FE044620B18378012B03D0FFF7FCFA35
:10C7900000240DE036B13246294662F072FF08B936
:10C7A0002046F3E7637BBB42FAD1237AAB42F7D151
:10C7B0002046F8BDF825002070B58B780646012B81
:10C7C0000C4692B042D191F8703007AD032B37D8A8
:10C7D000DFE803F0023032341E492846F4F792FBBA
:10C7E000059594F871301E21049394F872301A4A1A
:10C7F000039394F873300AA8029394F87430019369
:10C8000094F87530009394F876305BF06FFC324604
:10C810000AAB10AD1C4603CCAC42106051602346FD
:10C8200002F10802F6D1206810603046A388938098
:10C8300012B070BD0949D0E70949CEE70949CCE7F4
:10C840000A212846084A5BF051FCC9E700238DF80D
:10C850002830DCE7A9D50A00C4D50A00A62B0B00B6
:10C86000B0D50A00BAD50A0061F70A00002210B557
:10C87000837804460B70C3784B70037A8B70437BCC
:10C8800081F82320023BDBB2062B8EBF13462848DB
:10C89000C35C204681F82030A378012B14BF00230D
:10C8A000637A81F8213062F07EFE81F82200A3785D
:10C8B000012B3AD104F170038B60237A1D4AC3EB3C
:10C8C000C30313444B60E27804F1770304F17E0064
:10C8D00012BB1A460346C1E9032340F2E242D4F8F0
:10C8E00088304B61B3FBF2F30B83B4F890304B8389
:10C8F000B4F892308B83D4F8A4302BB15B7CDA0689
:10C9000044BF012381F82330D4F8A43013B15B7CF9
:10C910009B0603D4002010BD0246DCE791F82330CB
:10C9200043F0020381F82330F4E76FF01500F2E7DB
:10C93000053D0B00300000202DE9F04104460F4674
:10C9400015469846002B6ED01B6823B10221394A48
:10C95000394860F06EFF29462046FFF7DFFE0646A5
:10C9600000283FD12046294662F061FE0446002897
:10C970005CD097E80F00314D05F1080C8CE80F00F2
:10C98000AB8A002B08BF4FF49673AB822B8A03B996
:10C99000AB892B826B8A03B9EB8929486B8262F0E1
:10C9A00022FD430501D5FDF7C3F995F8DB2095F885
:10C9B000DA309A4219D903212046FFF731FA0220D2
:10C9C000FEF7F6FA054658B10220FEF719FB20469D
:10C9D0000021FFF725FA2046FFF7D6F92E4601E0A1
:10C9E000C8F800403046BDE8F08102212046FFF73C
:10C9F00017FA204662F07EF905460028F0D00021A3
:10CA000020462173FFF70CFA2046FFF7BDF90320FB
:10CA1000FEF7CEFA03460028E0D00221094A064874
:10CA200062F0E4FCDAE76FF01506DBE76FF00B0667
:10CA3000D8E700BFC1E80A00CCF7090030000020A9
:10CA4000B8000020F7D70A0038B5044608460D465E
:10CA500062F027F938B3154B93F89030990707D453
:10CA6000E37873B129462046BDE8384000F02EBB7C
:10CA700094F899309A07F3D5201D62F0B4FC430472
:10CA8000EED42946204662F022FE58B92B88A4F83D
:10CA90008C306B88A4F88E30AB88A4F89430EB8887
:10CAA000A4F8963038BD6FF01500FBE73000002089
:10CAB000F7B510F8333C0446A0F140060BBB3046F6
:10CAC00062F060FE3C4B1D684DB155F8183C1C3DB2
:10CAD0001BB1304614F8341C9847ED69F4E7374D24
:10CAE000374FBD4205D3304603B0BDE8F040FFF7F5
:10CAF0004BB96B681BB1304614F8341C984720358D
:10CB0000EFE710F83E3C012B53D110F83D3C8BB9B8
:10CB1000FCF75EFB69304CD102212A4A2A4860F0BA
:10CB200088FE40F239120023204603B0BDE8F040F1
:10CB300022F016BAA0F13C05D5E8EF3F23F40052ED
:10CB4000C5E8E12F0029F7D199041FD5E36C6946A8
:10CB50000093636D30460193FFF776FF034678B983
:10CB6000D5E8EF3F23F48053C5E8E23F002AF7D130
:10CB70004FF40061284603B0BDE8F04062F038BCD5
:10CB8000124A0221104862F031FCF1E74FF42813F9
:10CB90000F4A69463046CDE90023FFF755FF0346AB
:10CBA00028B94FF48051284662F022FCE0E7094A98
:10CBB000E7E703B0F0BD00BFDC3B002064F70900ED
:10CBC000A4F70900F6E80A00CCF7090029E90A00F1
:10CBD000180028004EE90A0008B568B1094B00F1B9
:10CBE0000C011A6822B9074862F0E2FB104605E022
:10CBF000914204D01268F5E76FF0150008BD6FF0A0
:10CC00007700FBE7E43B002038B5174866F019FDD4
:10CC10001649154866F053FD1549134866F04FFD57
:10CC20001449114866F04BFD63F015FA04F0C4FA9C
:10CC30000446B8B906F094F8044698B962F061FE6B
:10CC40000D4862F013FC054660B1043062F0CBFB86
:10CC5000C30704D5032128462C72FFF7E1F82846C4
:10CC6000FFF792F8204638BDB8160020B83B0020E8
:10CC7000C43B0020D03B0020F825002003460121C2
:10CC8000014A024860F0DEBD01EA0A003CF80900F2
:10CC900080B500AF88B06A46074BCDE90530032365
:10CCA00042F8103F00234FF4C2510448F7F70CF844
:10CCB0006FF00B00BD4680BD29EA0A003CF8090070
:10CCC00008B5064A136823B90548506018460A603B
:10CCD00008BDFFF7DDFF6FF00B00F9E7F03B002028
:10CCE000E8000A0070B5044652EA030008D0F8F7DD
:10CCF00015FB074D074ED5F8E0503058854201D15D
:10CD0000002213462046BDE870400431FFF7CCB93D
:10CD1000403100200800000038B5054618462B6851
:10CD2000DBB15B7B072B18D10B7A012B07D00121DC
:10CD30000B4A0C4860F086FD6FF0150038BDCB7AC9
:10CD4000072BF9D9C8618A6105F1300066F0B7FC9C
:10CD5000284662F0EEFC0020F0E76FF07F00EDE780
:10CD600050EA0A003CF809002DE9F84F8846914640
:10CD7000D0F8B44000AF44B1483C236B63B920689D
:10CD8000B43062F0F5FCA46CF5E7FBF7F5FF002684
:10CD90003046BD46BDE8F88F04F1300A504666F0D3
:10CDA000B3FC05460028F0D061F0FFFE80B16C4670
:10CDB00088B06A46294BCDE90535032342F8103F78
:10CDC00000234FF4C2512648F6F77EFFA546DEE762
:10CDD000284661F0FFF8E56C06469DB9A38C058AEC
:10CDE000403B9BB23F2B03D8238D9D4228BF1D465D
:10CDF000042106F10C0061F05CF90580A38C043578
:10CE00004380E56445451FD8B6F810B0AB4506D160
:10CE100000220023504621F097FDF8F735FEA38C41
:10CE2000A3F140023F2A06D8AB451ABF00221346A1
:10CE30000C4AF361B2612068B43062F099FC236B54
:10CE400013B1204662F075FCE36C98452CBF0021BD
:10CE5000A3EB0801C9F80030E16499E768EA0A0029
:10CE60003CF80900B5F80700F7B504460026234D45
:10CE7000234FBD4201D303B0F0BD2988204662F0A4
:10CE800010FD6B68019001A920469847002830DB0F
:10CE9000019B2A889A829A8403F11002D2E8EF1F3C
:10CEA000C2E8E06F0028F9D19E64DE649E60A16B49
:10CEB00003F10802F9B9C4E90D221C60DE6003F138
:10CEC000300066F0BEFB019843681B6803B19847C9
:10CED000019B1033D3E8EF1F41F00101C3E8E21FCB
:10CEE000002AF7D101984368DB6913B100F1100102
:10CEF00098470835BDE70A60A263DEE74CF70900F2
:10CF000064F709007FB50D460646042105F10C00C3
:10CF100061F0E8F82A8A43880446934208D00093D7
:10CF20001346444A0121444860F096FC04B070BDA9
:10CF3000417839B90121414A3F4804B0BDE8704009
:10CF400060F077BC0278122A22D0132A1AD0012A64
:10CF5000ECD0022113463848394A60F073FC6178FE
:10CF600002220120356862F082FC04460028DDD0F0
:10CF700002210C3061F075F80023214603704370E4
:10CF8000284624E0022BD1D0022200922D4AC9E784
:10CF9000082B03D0082200922B4AC3E73468637B36
:10CFA000072B02D00221294AC6E7E378A3B1022267
:10CFB000012062F05CFC05460028B7D002210C304D
:10CFC00061F04FF80023294603704370204604B0F7
:10CFD000BDE8704062F07BBCEB6813201A88ADF8A6
:10CFE00008205A88ADF80A209A88ADF80C20DB8812
:10CFF0000222ADF80E3062F03AFC0546002895D0CA
:10D0000002A92046FFF766FA0646022105F10C0048
:10D0100061F027F886F00103DBB203802946204641
:10D0200062F055FC002E81D0204602A962F04FFB31
:10D030007CE700BF80EA0A003CF80900A1EA0A0088
:10D040002DEB0A00C2EA0A00EDEA0A001FEB0A0013
:10D0500008B50B8A032B06D80121044A044860F066
:10D06000E8FB002008BDFFF74DFFFAE755EB0A008B
:10D070003CF8090038B50B8A0546032B0C4609D845
:10D0800001210F4A0F4860F0D4FB2046BDE838402C
:10D09000F8F7FABC042104F10C0061F023F8418890
:10D0A000284662F025FC30B9074A0B4605480221A4
:10D0B00060F0C8FBE9E7436821465B699847E4E70D
:10D0C00073EB0A003CF8090090EB0A0070B5134AB4
:10D0D0000C4613780646013313F0FF010ABF012303
:10D0E0000B46194613701220082262F0C0FB054659
:10D0F00088B108210C3060F0B4FF228829460280F4
:10D1000062884280A2888280E288C2803046BDE880
:10D11000704062F0DCBB6FF00B0070BDEB8900204B
:10D1200023281FD81A2804D8431E182B0ED90620EE
:10D130007047A0F11B03082B1ED8DFE803F0051D84
:10D140001B231D19251D05000320704701230F4ACD
:10D1500083401A40C2B90E4A1A40002A0CBF06206A
:10D160000120704700F07F03522B05D1002070474B
:10D17000012070470520704710F0400F14BF0020B9
:10D18000062070470420704702207047AAAA8A022E
:10D19000545545012DE9F74F064608460C46F8F769
:10D1A000D3FB182343432D4F0546FA18916801918C
:10D1B000E16806F15400D0E8AF0FC0070AD401219E
:10D1C000274A284862F0C0FB6FF01509484603B0B3
:10D1D000BDE8F08FE068007810710022FA500B78FB
:10D1E000D22B0FD133682146186864F08BF8814642
:10D1F00040B101211C4A1B4862F0A6FB2046F8F70B
:10D2000043FCE3E7182303FB0573D4F80C80D4F840
:10D2100014B0B4F810A09E60002321461A46301DB9
:10D22000FFF77AFD81460028D0D010F1690F04D1B4
:10D2300001210E4A0B4862F087FB6269A8EB0B08DC
:10D2400012FA88F2E26018225543019B7A19A4F879
:10D2500010A0936047F80590B8E700BF483C002055
:10D26000CCEB0A00BCF70900E6EB0A00F9EB0A0078
:10D2700008B5EFF31181202383F31288BFF36F8F7A
:10D28000002303600F4B5A68C2B9C3E9000081F361
:10D290001188BFF36F8F0C4821F0BAFD031E0CDA22
:10D2A00001210A4A0A4860F0CDFA002383F311886D
:10D2B000BFF36F8F0323184602DF08BD106058606C
:10D2C000E5E700BF403C0020240500201CEC0A00DC
:10D2D000BCF70900094B011F9A680948914204BF35
:10D2E00000229A601A6A914204BF00221A629A6B65
:10D2F000914204BF00229A6366F081B8483C002046
:10D30000741500200121024A024862F01DBB00BFD3
:10D3100045EC0A00BCF7090010B5044600F15003C3
:10D32000D3E8EF1F41F00101C3E8E21F002AF7D163
:10D33000201F62F032FB04F17400044966F0FFFA2A
:10D340002068BDE8104003F08DBD00BF55E301002B
:10D3500073B50E46438D418B01328B4228BF0B467D
:10D360009A42054609D9022100921D481D4A60F0E3
:10D3700073FA0024204602B070BD3046FFF7D0FE9D
:10D380006FF01403034113F0010310D0F7F7C6FF49
:10D39000154B1958154BD3F8E03099421DD0144B5A
:10D3A0001B685A1A18BF4FF0FF32134600E0114AAB
:10D3B00000211148FFF796FC04460028DAD0F8F760
:10D3C000C3FA18220D4B012102FB003304F10C00BB
:10D3D0009D6060F046FE0670CCE70022E5E700BFE6
:10D3E000BCF7090062EC0A00080000004031002090
:10D3F000903C00201C4E0E00FC160020483C0020F3
:10D4000070B5044601F10C000D4660F07BFE266805
:10D4100001462B8AEA68306863F00DFD1E21002268
:10D420002046FFF795FF014630B90121044A05481F
:10D4300062F08AFA002070BD204662F0A0FAF9E797
:10D4400087EC0A00BCF70900F0B51D4603680E46DC
:10D450000039044618BF012187B01868174663F0E9
:10D46000FBFC40B904F1540062F0C8FB002846D030
:10D47000002007B0F0BD002D43D0182200216846DF
:10D4800081F022FD6FB1002213212046FFF760FFDB
:10D49000019030B91C4801211C4A62F055FA112054
:10D4A000E7E7236829461B68284600930023ADF868
:10D4B00012300C9B164A0393BDF834308DF8086087
:10D4C000ADF8103001238DF814306B4662F03EFB4E
:10D4D0009DF8143063B1002FCAD00198F8F7D4FA40
:10D4E0002A46314620469DF8143062F092FBBFE791
:10D4F00001990029BCD0204662F041FAB8E7122019
:10D50000B7E70120B5E700BFBCF70900A4EC0A00AB
:10D5100003FA07002DE9F3410B8A04460D4643B98F
:10D520000121294A294862F00FFA002002B0BDE823
:10D53000F0810768012105F10C0060F0D3FD7B7BD1
:10D540000646072BF1D154F8043C002BEDD0002205
:10D5500003781F4F043C17F832004FEAC208984284
:10D5600007EBC20114D12A8A4878904226D90121BA
:10D57000009316481346174A60F06EF90423474497
:10D58000BA78012AD1D1002BCFD00022317811E016
:10D5900001321C2ADFD1104A02210C4860F052F9F6
:10D5A00031780846FFF7BCFD2122C24012F001028B
:10D5B000BBD10623204662F02CFBB6E74B68204621
:10D5C000294698470346DAE7BDEC0A00BCF7090094
:10D5D00010010A00F2EC0A00D8EC0A00F8B5124A71
:10D5E0000746002311480D4660F0B2FC044638B9E6
:10D5F00001212B460E4A0F4860F024F92046F8BD61
:10D6000000F10C060921304660F020FD2046F8F7B5
:10D610009BF91822084B012102FB003330469F6022
:10D6200060F01FFD0570E9E71C4E0E00FC1600209F
:10D6300001EA0A00BCF70900483C00202DE9F0414E
:10D640000E8A0446043EF6B2022E08468CB001D083
:10D65000102E64D104210C3060F044FD0DF1080857
:10D6600005884788011D3246404661F00EFA0028C1
:10D6700057D0A5B300268FB3AF4230D34FF4205319
:10D68000404601A98DF80460ADF8063061F0D0F98C
:10D6900048BB1422002107A881F016FC1121204666
:10D6A000FFF79CFF0990002837D001210C30CDE90D
:10D6B000074860F0D6FC00230A90394603701A4AE6
:10D6C0000B93284607AB62F041FADDE909131B789A
:10D6D000FBB90846F8F7D8F90A2301E03D460123D3
:10D6E0002A4610210EE042F60103404607A98DF8B4
:10D6F0001C60ADF81E3061F09BF90028C9D01023E2
:10D700002A461946204662F084FA00200CB0BDE893
:10D71000F081204662F033F9F7E71120F6E70420A4
:10D72000F4E70E20F2E700BF81DC01002DE9FF41A4
:10D73000036804460D461868012163F08DFB40B96B
:10D7400004F1540062F05AFAA0BB122004B0BDE804
:10D75000F08110220021684681F0B6FB212120468D
:10D76000FFF73CFF029038B34FF00108009405F139
:10D770000C072B8A012B04D82046029962F0FFF88F
:10D7800018E0384660F0BEFC6B4601460B4A064680
:10D790008DF80C8062F0DAF99DF80C30002BE8D09F
:10D7A0000298F8F771F93246202120469DF80C3096
:10D7B00062F02FFA0020C9E71120C7E775FE0700C5
:10D7C0002DE9FF41036804460D461868012163F006
:10D7D00043FB40B904F1540062F010FAA0BB1220E0
:10D7E00004B0BDE8F08110220021684681F06CFB96
:10D7F0000F212046FFF7F2FE029038B34FF00108E8
:10D80000009405F10C072B8A012B04D820460299BD
:10D8100062F0B5F818E0384660F074FC6B460146DB
:10D820000B4A06468DF80C8062F090F99DF80C309A
:10D83000002BE8D00298F8F727F932460E2120464F
:10D840009DF80C3062F0E5F90020C9E71120C7E728
:10D85000F9FE0700F0B51D46036804460E4685B084
:10D8600001211868174663F0F7FA38B904F154003B
:10D8700062F0C4F950BB122005B0F0BD65B31022B0
:10D880000021684681F020FB39462046FFF7A6FEBE
:10D89000029018B3BDF828302946ADF804300123B2
:10D8A00028468DF80C300E4A6B46009462F04EF913
:10D8B0009DF80C3002995BB10846F8F7E5F82A4666
:10D8C000314620469DF80C3062F0A3F90020D3E7E2
:10D8D000204662F054F8F9E70120CDE71120CBE7AC
:10D8E000F9FE07002DE9F0410E8A0446043EF6B227
:10D8F000022E08468CB001D0102E76D104210C30B7
:10D9000060F0F0FB0DF1040805884788011D3246E0
:10D91000404661F0BAF8002869D085B377B3BD42BC
:10D920002DD80121606863F097FA064678BB42F66D
:10D9300002038DF8000069464046ADF8023061F000
:10D9400077F820B342F60303404606A98DF8186025
:10D95000ADF81A3061F06CF8C8B1012D03D14FF663
:10D96000FF739F4213D004F1540062F047F900287E
:10D9700014BF002012200CB0BDE8F0813D46012309
:10D980002A460821204662F044F90020F3E71822D5
:10D9900000210DEB020081F097FA09212046FFF7E4
:10D9A0001DFE0890F8B101210C30CDE9064860F069
:10D9B00058FB0023099003700A2339468DF82C3058
:10D9C000284606AB0B4A62F0C1F89DF82C30089946
:10D9D0002BB10846F8F758F89DF82C30D0E72046D0
:10D9E00061F0CDFFD1E71120C5E70420C3E70E2089
:10D9F000C1E700BF39DD01002DE9F0430F460446C1
:10DA0000062187B007F10C0060F06CFB0588EDB1D2
:10DA1000B0F80280B8F1000F17D0454516D80023A2
:10DA200082888DF800308DF804304FF4205368461A
:10DA300001A9D7F80C90ADF80220ADF8063060F0DF
:10DA4000F7FF064660B10A2301E0454601232A4656
:10DA50000621204662F0DDF8002007B0BDE8F08323
:10DA60000146142201A83F7C81F02EFA07212046AE
:10DA7000FFF7B4FD0290D8B10A2341468DF8153066
:10DA8000284601AB0B4ACDE9036901948DF8147067
:10DA900062F05CF89DF8153002992BB10846F7F753
:10DAA000F3FF9DF81530D2E7204661F068FFD3E719
:10DAB0001120D2E725DB01007FB5CB6804461D8825
:10DAC0008DB15E8876B1B5420DD81022002168462E
:10DAD00081F0FAF905212046FFF780FD019058B941
:10DAE000112007E0354601232A460421204662F032
:10DAF00090F8002004B070BD6B4631462846084AB5
:10DB0000009462F023F8DDE9011323B90846F7F722
:10DB1000BBFF0A23E8E7204661F031FFE9E700BFD9
:10DB200075FA07002DE9F04342F60103002591B094
:10DB3000D2F8008006460F4600680BA9D8F804907A
:10DB400014468DF82C50ADF82E3060F071FF00288F
:10DB50006DD04FF4205330680BA98DF82C50ADF8E0
:10DB60002E3060F065FF38B1A3681BB15A88BA4205
:10DB700000D25F80012010E06168084661F0CCFEB1
:10DB8000B8F82A20B8F81A309A4294BFC0EB0200C5
:10DB9000C0EB0300032803D8002011B0BDE8F083D8
:10DBA000084660F01EFA05466168084661F0B4FE5A
:10DBB0006B8A2A8AA3EB020C6B69EA68D21AACEB77
:10DBC0000203B8F82AC0B8F81A20944594BFC0EBF5
:10DBD0000C00C0EB0200834228BF03466BB9887A71
:10DBE000F7F7AAFE0022002360F0B2F905460028EC
:10DBF000D2D00146606860F005FA002300933146F8
:10DC0000D6F804801023484602AAC047061E0EDB41
:10DC1000227CE068964227D001460BA860F035FFD1
:10DC200040B9237C134A022113485FF00BFE002306
:10DC3000A3609FE7F2B202A906A860F026FF10B920
:10DC40000E4A3346EFE706A90BA860F0F1FE002864
:10DC5000EDD100230421637405F10C0060F001FA9A
:10DC6000A0600780A36884E7324602A981F034F9F6
:10DC7000EDE700BF11ED0A00BCF7090030ED0A0026
:10DC80002DE9FF414FF000084FF4205305460E46A2
:10DC9000006802A9144617688DF80880ADF80A30AC
:10DCA00060F0C6FEA0B142F60103286803A98DF812
:10DCB0000C80ADF80E3060F0BBFE48B123691BB19B
:10DCC0005A88B24200D25E80012004B0BDE8F081E3
:10DCD0006168286860F0ACFE10B100232361F3E7AF
:10DCE000E368A0681A786AB1B7F81AC0798D038A18
:10DCF0008C4594BFC3EB0C03C3EB0103934201DAE1
:10DD00000020E2E704210C3060F0ABF920610680CE
:10DD1000236929465E80074B01940093384600230F
:10DD2000A26862F01EF80028EADB2069003818BFFC
:10DD30000120CAE72DFB07002DE9F34717680546C8
:10DD40008946006851681446D7F804A060F070FE58
:10DD5000804600284BD195222946504662F0DDFED0
:10DD60000646207540B1E3681B780BB184F8148037
:10DD7000002002B0BDE8F0872946504663F0A5F8C0
:10DD800010B908232375F3E7A068267560F029F918
:10DD900002210C3060F065F9164B2061A0F800906C
:10DDA00000930194334629463846A26861F0D9FFB2
:10DDB000002807DA10F1FF0F32BF0E204042C0B238
:10DDC0002075D5E72369002BD2D0A06861F0A4FDAF
:10DDD0007B8D7A8B9A4294BFC0EB0200C0EB0300AC
:10DDE000E3681B78984294BF00200120C1E701201E
:10DDF000BFE700BF29F907002DE9F04182B000AF6D
:10DE0000044688460022002339463B4820F0DCFBCC
:10DE10000546B0B16D4688B06A46384BCDE9053449
:10DE2000032342F8103F00234FF4C2513448F5F762
:10DE30004BFFAD466FF00B0630460837BD46BDE8D8
:10DE4000F081F7F76BFA2F4B29461A582E4B38689A
:10DE50001A602C2281F038F83B6800221C603C6874
:10DE60000023C4E90155C4E909552848391D7D60DE
:10DE700020F0AAFB064688B123686C4688B06A4643
:10DE80002349CDE90513032342F8103F4FF4C45151
:10DE90002B461B48F5F718FFA546CBE70146B022F5
:10DEA000786881F011F878681A4B83605C3065F00F
:10DEB000C8FB7B685433D3E8EF2FC3E8E16F002938
:10DEC000F9D17B681C60636A7D681BB904F10C00A2
:10DED00065F0B7FB626A05F1A803C5F8A820A26A3D
:10DEE000636202B9A36217227B685A855A8304339E
:10DEF000C8F80030A0E700BF581500204FED0A0019
:10DF0000BCF7090008000000903C002074150020B8
:10DF100074ED0A00FC04002008B5437B072B06D0F3
:10DF200002210C4A0C4861F00FFD002008BD0421BD
:10DF300061F0DEFC10B9094A0121F3E700F150035A
:10DF4000D3E8AF3FDB0701D4054AF5E750F8040CEE
:10DF5000ECE700BF1FEB0A00BCF7090099ED0A00CF
:10DF6000CCEB0A002DE9F04F85B000AFB860EFF3BD
:10DF70001188202383F31288BFF36F8F584C2046FB
:10DF800061F0C0FC2668054688F31188BFF36F8FE7
:10DF900000285FD0F7F7D8FC182202FB00F35149A4
:10DFA000C81851F803A003690021D0E90248FB60BA
:10DFB00090F80490B0F806B080F086FFA87AF7F7E2
:10DFC000BBFC6969034659B16A7AD00706D45A6A1C
:10DFD000284612687B60926890477B6800226A61DD
:10DFE0002946184665F07EFBB9F1000F0DD064B1EB
:10DFF000236853B11B6843B1BAF1000F2ED0012141
:10E000005346394A39485FF01DFC1EB30020B968F9
:10E0100065F063FC00281DDA6C468AB06A46344B12
:10E020000593344BCDE906304FF40073ADF8203042
:10E03000314B42F8103F00234FF411512B48F5F7B4
:10E0400043FE0023A54683F31188BFF36F8F03239C
:10E05000184602DF1437BD46BDE8F08F201D61F081
:10E060007BFF4846FFF75CF80528CED801A353F89C
:10E0700020F000BFB9E001008DE001000BE00100DD
:10E08000B9E001000BE001008DE0010004F1540350
:10E09000D3E8AF3FDA0705D40121184A134861F0ED
:10E0A00053FCB2E7A36D002BAFD00023144A04F158
:10E0B000780020F055FFA8E754F8543B1D68D4E8D9
:10E0C000AF3FDB07E8D5B8F1000F9ED0002403E096
:10E0D0002846F968C0470134A3B29B45F8D894E7B5
:10E0E000403C0020483C0020B4ED0A00BCF7090089
:10E0F000D3ED0A00103D0B0004000001CCEB0A0038
:10E100001C4E0E00F8B50F461646FFF705FFB0B1DE
:10E11000446A20461CB150F8A84904B1A83C731CBD
:10E12000194638B1428B458DAA4228BF2A469A42E9
:10E1300007D264B902210A4A0A485FF083FB002033
:10E14000F8BD32463946BDE8F840FFF701B9D4F8CA
:10E15000A85005B1A83D20460B462C46E2E700BF7B
:10E16000EEED0A00BCF7090007B50B460021024698
:10E17000F7F7D4F801910E4909580E480068884213
:10E1800004D00D48D0F8E000884201D100221346A7
:10E1900001A90A4820F018FA014638B91C22019852
:10E1A00080F092FE019803B05DF804FB0020FAE7CE
:10E1B00008000000903C0020403100209015002015
:10E1C00010B50022044600F10803D3E8EF0FC3E8BE
:10E1D000E12F0029F9D108B1F7F756FC2146BDE837
:10E1E0001040014865F00BB9901500202DE9F74368
:10E1F000044678300F4690461E4665F0AEFBA06D93
:10E2000050B90221144A154861F09EFB204603B024
:10E21000BDE8F04300F086B8114B98424FF0000380
:10E2200017D045684360A06DD0F81890FFF7C8FF7D
:10E2300000232068A36561F0C0FE3DB12068CDF8E1
:10E24000009043463A4631460068A84703B0BDE80F
:10E25000F0831D46ECE700BF09EE0A00BCF7090099
:10E26000943C0020F7B550F8044C0546002C55D0DE
:10E2700000F1A40104F1240061F0A7FC2E1F05F1B8
:10E28000580700220023384620F05EFB024658BBA8
:10E290006B6D2BB101466FF067033046FFF7A6FFA9
:10E2A000002345F8043C05F15003D3E8EF1F21F0AB
:10E2B0000101C3E8E21F002AF7D1636A73BB04F1CE
:10E2C0000C0600220023304620F03EFB78B9666839
:10E2D00086B921461248266065F091F8286803B097
:10E2E000BDE8F04002F0DEBEF7F7CEFBC9E7F7F776
:10E2F000CBFBE6E7A26833689642636008BFA36081
:10E3000077683FB1B3696FF067010093002320681D
:10E310001A46B8473046FFF753FFD8E703B0F0BDC1
:10E320005815002010B504460430FFF79BFF132159
:10E33000606861F0B2F8034630B1BDE810400121D9
:10E34000024A03485FF07EBA10BD00BF20EE0A000B
:10E35000BCF70900F0B589B0044654F8783D00AF29
:10E3600038461968FEF728FA6E4688B06A460B4BA5
:10E37000CDE905374FF40073ADF81C30084B42F877
:10E38000103F00234FF4E2510648F5F79DFC20466C
:10E39000B546FFF7C7FF2437BD46F0BD3EEE0A0085
:10E3A00003000001BCF7090070B550F8043C0446B6
:10E3B000061F002B3BD039B1436D002B37D01B7C9F
:10E3C000DA0734D505231CE00568284602F0B2FDC3
:10E3D0006B7A012B2BD0646D4CB3237CDB0726D5E5
:10E3E000E368002BEED030466269617CFEF7B0FF37
:10E3F000054668B9637C01210D4A0E485FF022FA98
:10E400000E2300223046BDE870401146FFF7EEBEF5
:10E41000E368D4E90512984718B12846F7F734FBAA
:10E42000EEE729463046FEF7B5FE0028F5D170BD6F
:10E430006AEE0A00BCF7090038B5836D044623B3C1
:10E44000164A934221D0CB68DD78F5B1052D40689E
:10E4500015D00F2D1AD1437A012B17D8022161F064
:10E46000AFF808B1103011D104F1780065F075FAF9
:10E47000A26D137C43F001031374002038BD437A6E
:10E48000032B03D8064AD15CE9E70E2500222B4670
:10E4900011462046FFF7AAFEEFE700BF943C00209C
:10E4A0000C3D0B0010B50C4608B301B3FFF734FD6B
:10E4B000E8B1436A3BB153F8A82902B1A83A996D73
:10E4C0008C4206D062B90430214661F07EFB2046C2
:10E4D00002E02046064A9A65BDE81040FFF770BE8C
:10E4E000D2F8A81001B1A83913460A46E7E710BDD3
:10E4F000943C0020F8B51D460F461646F7F724FA5F
:10E500001823044C03FB00400123C0E90376C380B9
:10E510000575F8BD483C002008B57FF006FD38B110
:10E5200001210346034A044861F0A8FE6FF004008D
:10E5300008BD00BF91EE0A0014F8090010B5184696
:10E54000144607491022A047041E07DA012123467A
:10E55000044A054861F092FE204610BD0024FBE706
:10E5600020270020A7EE0A0014F8090070B50D4C12
:10E57000064623780D46834204D12846611C61F08B
:10E58000D3FE58B9237CB3420AD12846064961F02C
:10E59000CBFE10B1012004EB001070BD0020FAE7A3
:10E5A0000020FAE7C83C0020D93C002070B50D4C93
:10E5B000064623780D46834204D12846611C61F04B
:10E5C000B3FE58B9237BB3420AD12846064961F00D
:10E5D000ABFE0028054808BF002070BD2046FCE7C0
:10E5E0000020FAE7C8260020D5260020D4260020E7
:10E5F00070B50E4C054623780E46834203D1601C4D
:10E6000061F092FE68B9237BAB420CD131460848D9
:10E6100061F08AFE20B10120404200F00C0020444D
:10E6200070BD0020F8E70020FAE700BFAE850020AB
:10E63000BB85002038B50C4619466BB103F11405B3
:10E640005B698AB9E268A360954200D1E360002368
:10E650000D681A464B61A847A3685BB9601C064960
:10E66000BDE8384061F08DBE1360E3689D4208BF8D
:10E67000E260ECE738BD00BF333C0B0070B5204BC7
:10E68000144682689A420FD1A568C66875B9227986
:10E690003046216861F050FE024628B11949013028
:10E6A00061F06FFE15701581012070BDE0680028D3
:10E6B000FBD02B888B420AD0F6D2E068A3680138E1
:10E6C0000433E060003818BF0120A360EDE725683F
:10E6D00022792946304661F02FFE024660B9304665
:10E6E000084961F029FE02460028E6D0294601309B
:10E6F00061F047FE23791370A3685B881381DCE720
:10E70000D1EB0100333C0B00102110B50648F9F79E
:10E7100099FB034630B1BDE810400121034A04488B
:10E7200061F0ACBD10BD00BF10270020C8EE0A008C
:10E7300014F8090038B5054648B1154B1A4613F8C8
:10E74000011C5C1E60F09DFF58B1204606E0114997
:10E750000F4861F0E9FD78B10D4B581E38BD00201F
:10E76000FCE72846217C04F1110260F08AFF0028B2
:10E77000F5D004F11000F1E7054B064903F1100054
:10E7800061F0D2FD0028EAD0014B03F10F00E5E76C
:10E79000C93C0020333C0B0010B54A1C0C4628B184
:10E7A000097860F06EFF30B1204610BD1046034975
:10E7B00061F0BAFDF7E70020F7E700BF333C0B003C
:10E7C00038B5054648B1154B1A4613F8011C5C1EB6
:10E7D00060F057FF58B1204606E011490F4861F03C
:10E7E000A3FD78B10D4B581E38BD0020FCE728462C
:10E7F000217C04F1110260F044FF0028F5D004F1FF
:10E800001000F1E7054B064903F1100061F08CFDA3
:10E810000028EAD0014B03F10F00E5E7FD3C0020A2
:10E82000333C0B002DE9F04106468846174660F060
:10E8300058FA60B341463046FFF7B8FE0546B0B916
:10E84000144861F018FD0446F8B1134861F013FD57
:10E8500068B90124114D6342114A03F00C030133DE
:10E86000D018414661F08DFD0C235C431655012103
:10E8700005F10800B94061F06EFDBDE8F04147F6D2
:10E8800012220023074820F06BBB054DE3E7BDE8EB
:10E89000F08100BFD0260020DC260020D4260020F6
:10E8A000C8260020E02600200246014610B50423B9
:10E8B00011F8010B0832F9F783FA034630B1BDE8CD
:10E8C00010400121024A034861F0D8BC10BD00BFCE
:10E8D000EEEE0A0014F80900022110B5094861F0B3
:10E8E0003AFD084007D10849084A0B88084CA24263
:10E8F00002D300B10B8010BD5068083203449BB2B4
:10E900000120F4E7E83C0020C6850020A4F70900B8
:10E91000B4F7090008B50121024A034861F084FDFB
:10E92000002008BD0AEF0A0014F8090038B51446A3
:10E930000E4B82680D469A4215D122792168C06833
:10E9400061F0FAFC78B1D4F8C8302F2B03D9FFF767
:10E95000E1FF002038BD04EB8302158101890133FA
:10E960005181C4F8C8300120F4E700BFD1EB0100A9
:10E9700008B50121034A044861F056FD6FF0150007
:10E9800008BD00BF5EEF0A0014F8090038B515464F
:10E99000084B82689A420AD1C4682968013420462B
:10E9A00061F0C2FC18B12046696861F0EAFC012000
:10E9B00038BD00BFD1EB010008B513468168074A96
:10E9C000914209D11A791968C06861F0B5FC18B193
:10E9D0000023036043600381012008BDD1EB0100E7
:10E9E00040F239120023014820F0BABAA8270020CB
:10E9F00008B50421084861F0AEFC6FF0020106483A
:10EA000061F0B4FC044861F036FCC30701D5FFF7A0
:10EA1000E7FF002008BD00BFD8270020024608B548
:10EA20000749013061F0ADFC00230C3202F8043CD0
:10EA3000D2E8EF1FC2E8E03F0028F9D108BD00BFCF
:10EA4000333C0B002DE9F04385B00E4690469946C5
:10EA5000044600AF58B90121344A354861F0E4FC5E
:10EA60006FF0150528461437BD46BDE8F08307F161
:10EA700008015FF0B7FF0546A0B16D4688B06A4651
:10EA80002C4BCDE905344FF40073ADF81C302A4B04
:10EA900042F8103F00234FF4E2512548F5F714F9EE
:10EAA000AD46DDE72046391D5FF0E7F8786858B1DC
:10EAB0000A22294659F0B8FB034628B101211F4A12
:10EAC0001B4861F0DBFBCBE7002007F10801FFF7F3
:10EAD0008FFD044620BB002EC4D01949FFF788FDE6
:10EAE000044638B90121174A114861F09DFC6FF0C6
:10EAF0000B05B7E7002307F1080100F8013B61F0BF
:10EB000040FC04F1080104224846C047041EA9DA6B
:10EB1000012123460C4A064861F0B0FB2546A1E7D7
:10EB2000002EEED10660466086609BE7F7D50A00AE
:10EB300014F809006AEF0A000300000186EF0A00DA
:10EB4000333C0B00A1EF0A00A7EE0A002DE9F047C5
:10EB500006460D461D48002190461F469DF820A000
:10EB6000DDF82490FFF700FB044688B1456080F88B
:10EB700011A0C0F81490C760C0F818804A465146EA
:10EB80003046FFF7BFFA054638B92046FFF718FBB5
:10EB90006FF00B052846BDE8F087002201231146DF
:10EBA000FFF7A8FC2846A56042464946B8470546F7
:10EBB00018B12046FFF704FBECE72146304661F030
:10EBC000D2FA05460028E5D0F3E700BF1C4E0E0040
:10EBD0002DE9F0471F46BDF8203006468846D1F89B
:10EBE0000C90002B4ED17B1E012B4ED8012F494695
:10EBF0000CBF15781588FFF7CFFD0446B8B915B9D5
:10EC00003846BDE8F0874946FFF7C6FD044638B9E7
:10EC10001F4802211F4A61F007FC6FF01000F0E767
:10EC200006F17001013061F0ACFB337A2370D9F842
:10EC30001030DBB9B4F808A02581B9F80A30AB422E
:10EC400003D04946404661F0F1FBAA4505D00022B9
:10EC5000307A06F17001FFF7E5FD002DD0D10E49A5
:10EC6000601C61F08EFB25702581C9E72A4641466C
:10EC7000304698470028C4DB01380128DAD96FF004
:10EC80000D00BEE76FF00600BBE76FF00C00B8E7C1
:10EC900014F80900C3EF0A00333C0B002DE9F041E2
:10ECA00080460F4616461D46FFF7A2FC044680B973
:10ECB0001749FFF79DFC044630B9BDE8F04101213A
:10ECC000144A154861F0B0BB394600F8018B61F079
:10ECD00058FB238973B9628972B9268165812146FF
:10ECE00011F8010B5FF0FDFF80B12046BDE8F04157
:10ECF000FFF7DABD9E4204D36289AA4206D29E4241
:10ED0000ECD263892681AB42E9D2E7E7BDE8F08126
:10ED1000333C0B00DDEF0A0014F8090010B5FFF7D3
:10ED200067FC044678B1014611F8010BF9F756F873
:10ED3000034620B10121044A044861F09FFA0023F0
:10ED400023606360A36010BDFCEF0A0014F80900A3
:10ED50002DE9F041214B1546826807469A4202D1BF
:10ED6000C4686389E3B90120BDE8F08105F170084A
:10ED70004146287A5FF0B5FF68B9194B9C4202D131
:10ED8000284661F063FD3046164961F0FAFA002327
:10ED90002370238119E04146304661F0F2FA14E015
:10EDA000238993B1264616F8011B2846324660F0A7
:10EDB00068FC0028DAD131462078FDF759FC20B1F3
:10EDC000457BFCF7E1FF072DCDD00021E368618191
:10EDD000002BC8D038469847C5E700BFD1EB0100EB
:10EDE0005C050020333C0B0073B50C46054608213A
:10EDF00004F11000164661F0AEFA122304223146E7
:10EE0000CDE9003228462246024BFFF79FFE02B0B2
:10EE100070BD00BF9908080038B505460C460F487C
:10EE2000012161F098FA10F0010F0D4B0AD11D83FA
:10EE30005C830A4861F01FFA830709D4BDE83840B3
:10EE4000FFF7CEBD198B5A8BA94202D89442EFD856
:10EE500038BD94421D83ECD9EAE700BFD8270020D3
:10EE6000882700202DE9F0419846BDF81830064665
:10EE7000012B174636D84344012B454635DCFFF7B6
:10EE800059FC044668B9FFF755FC044648B902210D
:10EE9000194A1A4861F0C8FA6FF010052846BDE813
:10EEA000F081B8F1000F11D00023217A21FA03F28A
:10EEB000D00703D53A78DA40D20719D50133032BAE
:10EEC000F4D13B7803F007031943217206F1700176
:10EED000601C61F056FA337A01212046237061F0FC
:10EEE00000FDDBE76FF00605D8E76FF00C05D5E70E
:10EEF0006FF01205D2E700BF19F00A0014F80900FC
:10EF000010B56FF0020104460E4861F02FFA0D486B
:10EF100061F0B1F9C20704D5002200230A4820F0AD
:10EF20001FF8204661F055F958B12046FFF702FC62
:10EF300038B1037ADB0704D5BDE81040012161F048
:10EF4000D0BC10BDD8270020A827002070B56FF0D6
:10EF50000801184861F00AFA40F2391200231648F5
:10EF6000F8F7D0FD0026154C651C2846144961F0C1
:10EF7000DBF9B0B9237ADB0713D52946FDF778FB17
:10EF8000054620B161F027F92846FCF7FDFE6FF039
:10EF9000020104F10C0061F0E9F90021204661F062
:10EFA000A0FC731C022B4FF0010604F11004DBD10E
:10EFB00070BD00BFD827002030270020C83C0020AB
:10EFC000333C0B002DE9F04385B089461646984640
:10EFD000044600AF58B90121414A424861F024FA81
:10EFE0006FF0150528461437BD46BDE8F08307F1DC
:10EFF00008015FF0F7FC0546A0B16D4688B06A468F
:10F00000394BCDE905344FF40073ADF81C30374B64
:10F0100042F8103F00234FF4E2513248F4F754FE17
:10F02000AD46DDE72046391D5EF027FE786858B111
:10F030000A22294659F0F8F8034628B101212C4A42
:10F04000284861F01BF9CBE7002007F10801FFF722
:10F050008DFA044690B9FFF76DFB044638B90121DB
:10F06000244A204861F0E0F96FF00B05BAE700236D
:10F0700007F1080100F8013B61F083F9B9F1000FD5
:10F080002AD0022239464046B047061E07DA01213F
:10F090003346194A134861F0F1F83546A2E73B7848
:10F0A000022E237209D00221144A0E4861F0BCF9E5
:10F0B0000021204661F015FC94E77B78012B05D9EF
:10F0C0000F4A3146074861F0D9F8F1E7204603F0CE
:10F0D000010161F0F6FB85E72046FFF79FFC81E721
:10F0E000F7D50A0014F809006AEF0A0003000001CE
:10F0F00086EF0A0045F00A00A7EE0A0067F00A0052
:10F10000BBF00A0037B504460D46FFF72FFA02465A
:10F11000D0B1037A0C308DF8043061F0ACF810F007
:10F12000010318BF01238DF80530022301AA2946E7
:10F130002046F8F75BFE034620B10121034A04484C
:10F1400061F09CF803B030BD0346F0E70CF10A0013
:10F1500014F80900104908B5104861F0E5F80146B7
:10F1600040B90E4B581E61F0ACFB0C4911F8010C74
:10F17000FFF7C8FF08490A4861F0D6F8014650B9C0
:10F18000084861F09EFB084B187C03F11101BDE8B3
:10F190000840FFF7B7BF08BD333C0B00C93C002057
:10F1A000D93C0020D83C0020C83C002008B50121F3
:10F1B000114861F0D0F8C3071CD4FFF78DFB0F494D
:10F1C0000F4864F0BCFB002340F239120C48F8F7FA
:10F1D00093FC0C490C4864F0B2FB02210B4861F02F
:10F1E000BAF80B480B4964F0AAFBBDE808400A488E
:10F1F000FDF7F2BC08BD00BFE83C0020150A08007E
:10F2000030270020CDFD0100A8270020D8270020AE
:10F21000E0260020A50A08003405002003462DE959
:10F22000F04148B1008A38B901244FF0140C11495B
:10F23000DFF844E0714501D3BDE8F081D1E9007603
:10F24000BB4204D30CFB0672143A93420ED93444E9
:10F25000A2B214460831EDE70CFB0578434507D010
:10F2600001356219AE4292B2F6D1F2E70025F8E715
:10F270001046E1E7A4F70900B4F709002DE9F74FBC
:10F2800099464FF6FF73BDF830400746002C08BF83
:10F290001C46444B90461B880091834252D2424BFD
:10F2A0001D68002D43D04FF0140B083DAE682EB101
:10F2B00056F8083C1B8ABB4203D900266B689E4265
:10F2C00043D3AD68002D32D0083DEFE773682B447F
:10F2D000BB4234D29DB20836344B9E42F6D3DEE7B1
:10F2E0004046D1585FF0A4FBA0B101350AF1010AF4
:10F2F000ADB273685345EED9009B9D4217D8BD420D
:10F30000F3D3142303FB0AF3326802EB030BB8F1C7
:10F31000000FE5D1B9F1000F0CD1013CA4B2294690
:10F3200058460E9A0D9B98470CB10028DDD103B0CA
:10F33000BDE8F08FDBF80C309945D6D1EDE74FF002
:10F34000000AD6E701251A4EC6E70BFB06F229682C
:10F35000009801EB020ABAF810309842E7D39F42B6
:10F3600018D8B8F1000F0DD1B9F1000F14D1013C3C
:10F370001946A4B250460E9A0D9B9847002CD6D041
:10F3800040B9D4E74046895801935FF051FB019B97
:10F390000028E9D0013691E7DAF80C209145F9D13F
:10F3A000E5E700BFC6850020EC3C0020B4F709006B
:10F3B000A4F7090010B59EB01022002168467FF026
:10F3C00083FD142200210DEB02007FF07DFD4FF440
:10F3D0001053ADF8103080231022ADF812304FF4E6
:10F3E0008063284C6946CDE906340DEB02001CAB66
:10F3F0007EF02AFC034630B1234A0121234860F005
:10F400003DFF1EB010BD014648220AA87FF05CFDFA
:10F4100022461C990AA87EF085FD034660B10121B1
:10F420001B4A1A4860F02AFF1C987EF043FB0346F3
:10F430000028E6D0174AE0E74FF6FF710120164A90
:10F440000AAB61F0DCFA1022144904AB0AA87EF082
:10F4500087FD04461C987EF02DFB14B1104A23460C
:10F46000CBE708220D4B03F11001187811F8014D7C
:10F47000013A03F8014B0870F7D10821094860F000
:10F480006AFFBEE70002C00335F10A0014F8090064
:10F490005EF10A007CF10A008102080010270020BA
:10F4A00092F10A00D82700202DE9F04118490446BE
:10F4B000A1F1300015461E46BDF8187064F064FADC
:10F4C000144860F0D8FE010705D4FFF773FFFFF77B
:10F4D00041FEFFF719F92046FFF72CF968B1037ACE
:10F4E000DA070AD500F10C04204660F0C4FEC30719
:10F4F00003D40221204660F02EFF10233A460693E3
:10F5000031462846BDE8F041034B61F0DCB800BF4E
:10F5100060270020D82700201027002010B51B48A6
:10F5200060F0A9FEC0F3C00080F0010408B9FFF745
:10F5300041FF164860F09FFE0346144860F09BFEB2
:10F54000DA0622D5830606D5FCB1FFF703FEBDE837
:10F550001040FFF7D9B820210C4860F0FCFE1022C3
:10F560000B4988187FF0B8FC48B90A4864F0F5F9EF
:10F57000BDE810406FF00101044860F0F7BE4FF69F
:10F58000FF710120FFF748FCDFE710BDD8270020FE
:10F5900010270020A827002008B51021034860F09C
:10F5A000DAFEFFF7BBFF002008BD00BFD827002010
:10F5B0002DE9F3470446624860F05DFEC10713D4AD
:10F5C000FFF78AF92368002518684FF4C05369468D
:10F5D0008DF80050ADF802305FF02AFA60B96FF094
:10F5E000770002B0BDE8F087564860F044FE42075D
:10F5F000E6D46FF01500F4E7236801A9186841F616
:10F6000001038DF80450ADF806305FF011FA0028C0
:10F61000E5D04D4D20F024F82B6826689BB9002ECC
:10F6200065D1002204F10803A2606A68002A68D14B
:10F63000C5E90033424860F01EFEC30771D420F0D4
:10F6400023F80020CDE76B68002B77D053E9023216
:10F65000142101FB023333F8047C002E4FD1002F1C
:10F66000DFD023681E8ABE42DBD829680029E1D09A
:10F670000022A1F108031868008AB0424AD904F1B7
:10F680000803002A40D09168A1600029CDD0936082
:10F69000D0E7F37C318A23F08003F37489B9791CB5
:10F6A000DBB289B243F080033182F3740F4609F173
:10F6B000FF3914361FFA89F9B9F1000FE9D147462D
:10F6C000CDE78F42F2D301AB0846204ACDF804A023
:10F6D00061F095F9019B43B1338A01211C4A1D4811
:10F6E00060F0CCFD1FF0D0FF83E73946DEE7984697
:10F6F000194A17884FF0000AB4F80490DCE7B846BE
:10F70000F8E713606B6095E76A68A1602B60002AD8
:10F7100090D1F7E7986800288CD01A46A0F108032A
:10F72000A9E71421D4E9002301FB0323108A33F84D
:10F73000041CFFF771FBFFF709FC80E71B68FFDE85
:10F74000E83C0020D8270020EC3C002017020800ED
:10F75000A8F10A0014F80900C68500202DE9F04F31
:10F76000B9B000AF0C46904638493A46D7F8080180
:10F7700099465EF05EFA40B9FFF7FAF86FF01505AA
:10F780002846E437BD46BDE8F08F3E68391D304657
:10F790005EF073FA3EB901212D4A2E4860F044FE16
:10F7A0006FF015043FE0786800BB4FF0000B07F1E5
:10F7B000080A5146304687F814B05FF013F9054641
:10F7C00008B36C4688B06A46234BCDE905364FF442
:10F7D0000073ADF81C30214B42F8103F4FF4E2515A
:10F7E0005B461C48F4F770FAA546D9E70A220021C7
:10F7F00058F01AFD03460028D7D00121184A1548B1
:10F8000060F03CFDCCE7C7F810A0E4B1C022484648
:10F8100007F12001C047041E07DA01212346114ADF
:10F820000C4860F02BFD2546AAE7A40807F1200349
:10F83000C7E906344FF6FF7101200B4A07F11003A8
:10F8400061F0DDF89CE72346F2E700BFC9F10A004A
:10F85000F7D50A0014F809006AEF0A000300000156
:10F8600086EF0A00A7EE0A007DE60100002330B50E
:10F87000B5B001918DF808003393044601AB0D46F5
:10F8800001204FF6FF710B4A61F0B9F8339B73B159
:10F890009B0003AA29462046F8F7BEFA034620B18A
:10F8A0000121054A054860F0E9FC35B030BD1A4633
:10F8B000F0E700BF2DE90100D0F10A0014F80900BB
:10F8C0002DE9F34100F17008CDE9001204460F461E
:10F8D000007A414615465FF004FA06466B464FF63D
:10F8E000FF710120214A61F08AF81EB14146207A59
:10F8F000FFF7BCFF3946207AFEF738FE40B12946B3
:10F90000013060F03EFD1EB14146207AFFF7FAFB60
:10F9100094F8088039464046FEF76AFE0446C8B1AE
:10F9200029464046FEF764FEC8B1844217D02289BA
:10F93000638952EA030106D00589418995420CD8B2
:10F94000994200D24381002323606360A3600EB11B
:10F95000FEF7AAFF02B0BDE8F0810281F0E7601C6B
:10F96000294660F00EFD2046F1E700BF8DE9010059
:10F970002DE9F74F1421054603681A8A0092426860
:10F9800001FB023333F804BC1FF06AFE384805F16E
:10F99000080160F040FF814600285ED11FF074FE30
:10F9A0006FF0010003B0BDE8F08F14222B6802FB5A
:10F9B0000434304AA368934219D094F91330002BD1
:10F9C00005DA236923F000431B0C1B0423610AF1B1
:10F9D000010A6B681FFA8AF4A342E6D8264860F051
:10F9E0004AFCC3073CD41FF04FFE0020DAE7002397
:10F9F000E668224906F101084046738160F094FCF4
:10FA000007460028D9D141463078FCF731FE03463D
:10FA100048B9414630785FF064F9A0B1414630788A
:10FA2000FFF724FF0FE0427B072A14D100F1700199
:10FA30003A46007A0193FEF7F5FE019B1846FCF763
:10FA4000A3F9002FE5D140460C4960F09AFC002351
:10FA500033703381B1E74F46F0E74FF0000AB8E763
:10FA600059460098FFF7D8F9FFF770FABBE700BFD7
:10FA7000EC3C0020D1EB0100E83C0020333C0B00C3
:10FA8000002307B50193FFF7C9FB411C89B2084663
:10FA9000034A01AB60F0B3FF019803B05DF804FBCB
:10FAA000DB0708002DE9F04387B0437B8046072B36
:10FAB0000C46154602AF40F0A68000233B7342F689
:10FAC0000303206807F10C01FB815EF0B1FF0646DD
:10FAD000002834D1D4F80490B9F1000F05D10121E8
:10FAE0004B4A4C4860F0A0FC8DE001232146009079
:10FAF00007F10802C847031E11DA6D4688B002AA52
:10FB0000D36104234449C2E9051442F8103F4FF47D
:10FB1000015133463F48F4F7D7F8AD4673E0012B67
:10FB200005D001213D4A3B4860F0A8FB6BE03B7AE1
:10FB300013F0300F67D02046FFF7A2FF04460023E2
:10FB400020683B7342F6021307F10C01FB815EF063
:10FB50006FFF18B12046FFF793FF0446002642F6D8
:10FB60000219206839463E70A7F802905EF060FFE7
:10FB700018BB002320683B7342F6021307F10C0107
:10FB8000FB815EF055FF064600283CD1D4F8049076
:10FB9000B9F1000FA3D0022300902146404607F19F
:10FBA0000C02C847031EA8DB022BBAD1BB8905EAA9
:10FBB0000300003818BF012026E042F60303206846
:10FBC000391D3E71FB805EF033FF0028D1D04FF429
:10FBD0002053206807F108013E727B815EF028FF08
:10FBE0000028C6D042F60103206807F10C013E73DD
:10FBF000FB815EF01DFF0028BBD02046FFF740FFD1
:10FC000004460028ADD100201437BD46BDE8F0837E
:10FC1000EEF10A0014F8090002F20A0028F20A00C4
:10FC20002DE9F8431546894694226968064660F036
:10FC300074FF8046002841D1022230466968FFF7F0
:10FC400031FF00283DD000211F48AF8AFEF78CFA13
:10FC50000237044680B11D211C4B47613A4641746E
:10FC6000C0F80C80436085613046FEF74BFA0746CA
:10FC700038B92046FEF7A4FA6FF00B052846BDE818
:10FC8000F883012342464146FEF734FCA98A07F176
:10FC90000C0002315EF0E5F920F8029BAA8A29697E
:10FCA0007FF0ECF821463046A76060F05CFA05462C
:10FCB0000028E3D02046FEF783FADFE74FF0FF3558
:10FCC000DCE76FF01505D9E71C4E0E001D02080099
:10FCD00070B505468AB03A4860F0CDFA42070C4646
:10FCE00067D515B16B7B072B66D1666830460596E4
:10FCF000FFF794FA2268ADF81800002A2FD005A962
:10FD00000291304900230191012100914FF6FF71CA
:10FD10000593FFF7B3FA059E1EB96FF001000AB014
:10FD200070BD6660002330688DF8103042F6030322
:10FD300004A9ADF812305EF07BFE40B90598C368A7
:10FD40009B799B0608D560F013FEADF81800059866
:10FD500060F0B8FE606028B96FF01500DFE700289A
:10FD6000E0D1DAE7BDF818003DB101230146224693
:10FD70002846A375FFF754FFD1E76FF07F03079381
:10FD80000223ADF8203042F60213ADF8123005AB75
:10FD9000A57502930C4B4FF6FF710193012304AA42
:10FDA00000932B4609948DF81050FFF767FA0798D7
:10FDB000B5E76FF00A00B2E76FF07F00AFE700BF72
:10FDC000B80000204B0208003100020073B5044661
:10FDD00050F8083C00F130056FF00101A0F1200659
:10FDE0002846019360F0C2FA0D4B002044F81C3CF9
:10FDF0000C4B314644F8183C01AB44F8103C04234A
:10FE000024F8080C24F8060C24F80C3CFFF760FFDB
:10FE100018B90221284660F09EFA02B070BD00BFFA
:10FE20002C020A0001EF01002DE9F84316463A4B77
:10FE3000826805469A4200AF24D1D0F80C8034681D
:10FE4000B8F80830F3B14246204612F8011B5FF0C3
:10FE500018FCB8B14FF495722946204660F05DFE5B
:10FE600028B3032812D16C4688B06A462B4BCDE9E3
:10FE7000053542F8100F00234FF4C4512848F3F71A
:10FE800023FFA5460120BD46BDE8F883052820468E
:10FE90000CBF4FF003094FF002095FF0C2FB814530
:10FEA00005D933794B45EDD286F80490EAE741460F
:10FEB000284660F0BBFA1B4B9845E3D1207A04F149
:10FEC0007001FEF795FB05460028DBD0038913B9C6
:10FED0004389002BD6D02046FCF7DAF82A89124B4A
:10FEE000124923F820206A8903EB80035A801822E4
:10FEF00002FB00110B6104230D4A20464A600D4AA3
:10FF00008B828A60FFF7E4FE0028BBD001210A4AF9
:10FF1000034860F089FAB5E7D1EB010041F20A002D
:10FF200014F809005C050020AA850020B03C0020E0
:10FF30002C020A00FF08080055F20A0070B50446BA
:10FF40008AB0384860F097F942070D4663D514B17E
:10FF5000637B072B62D16E6830460596FFF75EF92A
:10FF60002A68ADF81800002A2FD005A902912E4961
:10FF700000230191012100914FF6FF710593FFF7D6
:10FF80007DF9059E1EB96FF001000AB070BD6E606C
:10FF9000002330688DF8103042F6030304A9ADF851
:10FFA00012305EF045FD40B90598C3689B79DB06C9
:10FFB00008D560F0DDFCADF81800059860F082FD12
:10FFC000686028B96FF01500DFE70028E0D1DAE7B4
:10FFD000BDF818002CB101462A46204660F0D8FD35
:10FFE000D3E76FF07F0342F6021207930123ADF8C7
:10FFF000122005AA02920D4AADF82030CDE9003258
:020000022000DC
:100000004FF6FF71234604AA09958DF81040FFF7BB
:1000100035F90798B9E76FF00A00B6E76FF07F008F
:10002000B3E700BFB80000204B0208003100020017
:100030002DE9F0413D4B1546826807469A4203D0B0
:1000400001273846BDE8F081D0F80C80384B984540
:1000500012D0B8F80820AB899A42F1D1414611F884
:10006000010BFCF705FB06460028E9D0437B072B74
:1000700024D0FBF789FEE3E700262E4C20462E49CC
:1000800060F052F978B90722214614F8010CFCF708
:1000900071FB80B92B6921461A6914F8010C538849
:1000A0001288FEF7FBFD731C022B4FF0010604F1D2
:1000B0000C04E3D1CDE7FBF767FEF4E7D8F8143082
:1000C00023B13946984708B93046D2E739469422D9
:1000D000304660F022FD07460028F5D1AB89022B9F
:1000E00015D1B8F808309A071ED530462A69A98874
:1000F000FFF796FD044618B92A69937D013393757D
:100100003046FBF741FE002CAC609ADB98E7012BF0
:100110000AD1B8F80830DB0706D530462A69A98825
:1001200060F036FD0446EBE73C46E9E7D1EB010021
:100130005C050020AF850020333C0B0073B5437B8A
:100140000446072B0D461AD1061D4FF48031304668
:1001500060F001F9C30315D402232046CDE9003332
:100160002A460A4B0A49FEF7F1FC044620B16FF417
:100170008031304660F0FAF8204602B070BD6FF072
:100180007F04F9E76FF07704F6E700BF5D0408002D
:100190005302080070B5437B0546072B0C4686B01A
:1001A00040F0A1800B7C062B10D8DFE803F004049C
:1001B0005A5A629528000B68CBB11B784BB1022BC1
:1001C00013D00121494A4A4860F058F86FF01500F1
:1001D00009E0082301930623224600934549464B34
:1001E0002846FEF7B3FC06B070BD1623F2E71023D5
:1001F00004212246CDE90031404B4149F0E708682F
:100200000028E3D00678002EE0D14FF4245302A951
:100210008DF80860ADF80A305EF00AFC08B342F6CB
:100220000213206803A98DF80C60ADF80E305EF063
:10023000FFFBB0B142F60313206804A98DF81060EB
:10024000ADF812305EF0F4FB58B142F604132068AA
:1002500005A98DF81460ADF816305EF0E9FB0028B2
:10026000B4D1082304222749CDE900322246264B87
:10027000B6E7086880B300264FF4205302A98DF832
:100280000860ADF80A305EF0D3FB00289ED042F63D
:100290000103206803A98DF80C60ADF80E305EF004
:1002A000C7FB002892D042F60203206804A98DF80B
:1002B0001060ADF812305EF0BBFB002886D042F62D
:1002C0000303206805A98DF81460ADF816305EF0C0
:1002D000AFFB00283FF47AAF04232246CDE9003378
:1002E0000A490B4B7CE76FF07F007CE772F20A0053
:1002F00014F809003B0C08008F070800F1040800FF
:10030000150302003904020021050800B1070200AC
:10031000890408002DE9F0478EB0064617461C46B2
:10032000169D31B12A4600216B680EB0BDE8F0473A
:10033000184763B902213D4A3D4860F075F82A46E6
:10034000002130466B6898470EB0BDE8F0871378FF
:10035000062B08D0142B05D00121364A34485FF013
:100360008DFFECE702214FF00008C146013C8DF8FB
:100370001010A4B207F1010A9C420CD2002CDED16D
:10038000B8F1000FDBD02A46414630460EB0BDE83A
:10039000F04760F034BC1422002109A87EF094FDDF
:1003A000BAF8002093B2002BC9D0BAF802101FFA95
:1003B00081F8B8F1000FC2D04345C0D89DF8103085
:1003C00013B3022B25D02B7CADF80C10002B42F67A
:1003D000010308BF4FF42053ADF8063004AB02937D
:1003E00001AB099302ABADF834200C932A4630469A
:1003F0006B688DF8049009A998470028A4D03B7831
:10040000E41AA4B29A44B7E7BAF80430ADF812304F
:10041000D9E70AF104030DF111000AF1140C53F8A5
:1004200004EB634540F804EBF9D1CCE787F20A000E
:1004300014F8090091F20A002DE9F04F93B0174625
:1004400080461C460A461C9D31B12A4600216B6835
:1004500013B0BDE8F04F1847297C022940F0838093
:100460004BB99B4A9B485FF0DFFF2A46002140467C
:100470006B6898475BE03B78062B08D0082B05D0CB
:100480000121954A93485FF0F9FEEEE711460026F8
:1004900042F6020A013C8DF82010A4B207F1010BCC
:1004A0009C420BD2002CE0D1002EDED02A463146F1
:1004B000404613B0BDE8F04F60F0A1BBBBF8009020
:1004C0001FFA89F6002ED0D0BBF802009DF820203C
:1004D000ADF81C00BBF80410ADF81E1062B1022A82
:1004E00015D0296831B308A85EF0A2FA10B33B78A2
:1004F000E41AA4B29B44D3E708AA06929BF806200C
:100500009BF8071042EA0122ADF82220E9E70A230E
:100510006881A981A5F808904046019200932A4677
:100520006E4B6F49FEF712FB86B2002EBED113B0A0
:10053000BDE8F08F4FF00003102200210EA88DF8C7
:100540001430ADF816A07EF0BFFC05AA0D9206AAE5
:10055000109240462A466B68ADF844900DA9984722
:100560000028C4D1E3E7032966D113B90221584A10
:1005700078E73B78072B02D0152B81D10222002689
:10058000013C8DF82020A4B207F101090DF1200AE9
:100590009C4287D3B9F800B01FFA8BF6002E3FF4C7
:1005A00064AF9DF8203063B1022B13D02968F1B1FC
:1005B00050465EF03DFAD0B13B78E41AA4B29944BB
:1005C000E6E799F8053099F8062043EA0223ADF8EA
:1005D0002230EBE709F105030DF1210209F11501C4
:1005E00053F8040B8B4242F8040BF9D1DEE799F87B
:1005F0000230B9F803208DF81E304FF000038DF85B
:10060000143042F603030021ADF81C200EA810227E
:10061000ADF81630CDF818A07EF056FC05AB0D9362
:1006200006AB10932A4640466B68ADF844B00DA95E
:1006300098470028C0D17AE72A68167876B92BB98E
:10064000234A022123485FF0EFFE07E03B78012BAD
:1006500009D80221204A1F485FF010FE2A460021D7
:1006600040466B68F4E6B2F802A0013CA4B207F180
:100670000109AAF5245A9C4204D2002CEED1002E86
:10068000ECD013E7012C01D8164ADAE7B9F800B02C
:100690001FFA8BF6002EE1D0BAF1040FDED801A3C9
:1006A00053F82AF0B90602005D060200C1060200F6
:1006B000C906020031070200032C1BD80A4AC0E712
:1006C000032C17D8094ABCE7032C13D8084AB8E70B
:1006D00087F20A0014F8090091F20A007504080074
:1006E00079070200A5F20A00B3F20A00C1F20A007B
:1006F000CFF20A00B9F80230ADF820302B68102292
:1007000000210EA803937EF0DFFB039B2A460D9386
:1007100008AB109340466B68ADF844B00DA99847FC
:1007200000283FF404AF3B78E41AA4B29944A2E74E
:10073000082C01D80F4A84E799F802308DF8203050
:1007400099F803308DF8213099F8052099F8043094
:1007500043EA0223ADF8223099F806308DF82430B0
:1007600099F8073099F8082043EA0223ADF82630BB
:10077000C4E700BFDDF20A0070B5102B0546114634
:10078000049C0BD00121084A08485FF077FD2246FF
:10079000284663680021BDE8704018472246BDE83E
:1007A000704060F096BA00BF91F20A0014F8090098
:1007B0002DE9F04F8FB00746189D184629B953B957
:1007C0000221544A54485FF02FFE2A460021384641
:1007D0006B6898479BE01378012B07D0022B20D041
:1007E00001214E4A4C485FF049FDEEE70B464FF0C1
:1007F0000409013880B248458DF81030E5D34FF038
:100800000008B0FBF9FBC246541CCDF8008004AED2
:10081000BBF1000F08D12A463846009960F0EFF985
:1008200075E04FF01209E4E723880193BDF8043026
:100830000093B8F1000F53D19DF81030002B37D042
:10084000022B3CD02968002945D12B7C042B4DD1AB
:100850004FF42053304602A98DF808A0ADF80A30B5
:100860005EF0E6F800283BD042F60103304603A9CB
:100870008DF80CA0ADF80E305EF0DAF880B342F6D9
:100880000203304609A98DF824A0ADF826305EF0A9
:10089000CFF828B342F60303304609A98DF824A007
:1008A000ADF826305EF0C4F800BB4FF0010819E047
:1008B000A378E27843EA0223ADF81230C2E7A31C22
:1008C0000DF1110204F1120153F8040B8B4242F8AE
:1008D000040BF9D1B6E730465EF0AAF80028B4D090
:1008E0004FF000080BF1FF3B4C4491E71022002130
:1008F0000AA87EF0E9FABDF804302A46ADF8343093
:1009000038466B68099609A998470028EAD10FB0C4
:10091000BDE8F08F87F20A0014F80900EBF20A0034
:1009200007B5437B0A46072B2CD14B683BB90823FC
:100930004FF0040ECDE9003E144B154909E0012BA0
:1009400011D0097B5B00019341B120231149009331
:10095000114BFEF7FBF803B05DF804FB0E230F49C3
:1009600000930F4BF5E74B8933B10C234FF0040C88
:10097000CDE9003C0B4BE0E70A230221CDE9003131
:10098000094BDAE76FF07F00E5E700BFE1070800F9
:10099000AD090200450608008505080005060800A7
:1009A0005D050800B5040800A10408002DE9F04F1A
:1009B00085B002AF804691469A460E463C6B41B9DF
:1009C0006BB92568002322460093F1B24046A84740
:1009D00030E0B1F5807F28BF0E262568F2E7636816
:1009E000002B71D123890AF1FF35B4F80AB07B607E
:1009F000ADB202F1010A002D4DD099F80030AB42A2
:100A000028BF2B46012B0AD802213E4A3E485FF000
:100A100035FC00230093224604212568D6E7BAF866
:100A20000020023B91B29BB241B90121374A3648BE
:100A30005FF0FAFC0C37BD46BDE8F08F786888425D
:100A400001D88B4518D26D468AB002AA304BC2E954
:100A500005317B68C2E9073B052342F8103F0023BC
:100A60004FF422512848F3F72FF9AD4600230093A5
:100A7000256822460E21A9E7228100932246002103
:100A8000404626680AF10203B0470028D2D099F800
:100A90000030AB4206D921464046FFF741FF00280F
:100AA000C8DAE3E7238962899A4205D100230093DB
:100AB00025682246194689E70133238199F80030D9
:100AC000ED1AADB29A4496E7CDF800A0134625681A
:100AD0002246A8470028ADD0238A013B9A4503DA75
:100AE000009633462568E4E7638921460AEB03054F
:100AF00040466581FFF714FF00289BDA00963346D5
:100B00002568B6E7FDF20A0014F8090035F30A007B
:100B100044F30A0073B5437B0546072B0C4603D00C
:100B20006FF07F0002B070BDCB88B3B128465FF094
:100B300094FA0028F4D0A289431F9BB2934228BFA5
:100B4000134604339BB201931623224600930A49AD
:100B50000A4B2846FDF7FAFFE4E78E895FF07DFA3D
:100B600002360138B042E1D31223224600930449F1
:100B7000044B0196EDE700BFD30D0800C505080042
:100B80006302080089050800032A2DE9F743064699
:100B90001C460CD80221244A24485FF045FC22461A
:100BA0000E213046236803B0BDE8F0431847B3F880
:100BB0000C90151F4D4513D91D4A01211B485FF0AC
:100BC00033FC18230121CDE900311A4B224630466F
:100BD0001949FDF7BBFF0028E1D103B0BDE8F08360
:100BE000DB88B1F80280984506D1A7682A463846C6
:100BF00004317EF071F908B1104ADEE7A9EB050374
:100C000018FA85F82F449BB2A4F80680A760A38148
:100C10002BB918230122CDE90032094BD6E7214632
:100C20003046FFF777FFD6E787F20A0014F809008D
:100C3000ABF30A00CD04080063020800CDF30A00FC
:100C4000DF04080070B5437B0646072B0D463DD1F7
:100C5000FDF7B6FD044658B9FDF7B2FD044600287D
:100C600037D006F1700101305FF08BFB337A2370CF
:100C7000A36893B10022143B9D422DD01889298985
:100C8000884205D19889A989884228BF42F001028B
:100C90005B690BB1143BEFE772B9114A2946304644
:100CA000FEF7A2F8024638B1A3681BB90D49601CD3
:100CB0005FF067FB104670BDA26805F114036A611E
:100CC000E268A36002B9E3600022F3E76FF07F02FD
:100CD000F0E76FF00B02EDE76FF07702EAE700BF95
:100CE00091030800333C0B00F8B5437B0646072B05
:100CF0000C4643D1FDF764FD0546002841D08368CA
:100D0000002B3ED000221746143B9C4209D0188984
:100D10002189884208BF47F001075B691BB1143B7A
:100D2000F3E70122F9E762B304F110005FF0A3FAE0
:100D3000430703D52146304660F05EF877B104F1F1
:100D4000140105F108005FF066FDAB681BB90E49A0
:100D5000681C5FF016FB57B9002007E021463046BB
:100D60000A4AA781FEF740F80028E8D0F8BD002322
:100D700021461A4630462568A847EDE76FF07F0008
:100D8000F4E76FF01500F1E7333C0B009103080026
:100D90002DE9F0478C68064690469946BDF820A09C
:100DA00024B154F8145905B1143D0CB9BDE8F087CD
:100DB0002389434515D1727AA37B9A4211D35346B6
:100DC0004A46214630462768B84750B92146304642
:100DD000FFF78AFF034620B10221064A06485FF06A
:100DE0004DFA2DB1696901B114392C460D46DCE785
:100DF0002946FAE703F40A0014F80900F0B587B0B1
:100E000007460E461546FDF7DBFC0446C8B12A46E8
:100E1000314603A85DF014F9BDF81030042B10D949
:100E2000042103A85DF05EF9BDF810104688028821
:100E3000B14208D201213346084A094800955CF0C6
:100E40000BFD07B0F0BD2146031D00963846FFF7A5
:100E50009FFF314603A85DF045F9DDE722F40A0063
:100E600014F80900012370B500F170058EB0044636
:100E700003902946007A8DF810305DF032FF90B172
:100E8000227A52B302AE042130465BF0BCFE0096DB
:100E90002421134A2B4605A8F6F7D4FE05AA1046CE
:100EA0001049F3F7F7FA4FF6FF7101200E4A03AB32
:100EB0005FF0A5FD20465EF0B4FB9DF8101088425F
:100EC00009D220465EF07CFB034620B10221074A8E
:100ED00007485FF0D3F90EB070BD0092D8E700BFAD
:100EE000CBF20A005DF7010029FE01003BF40A0085
:100EF00014F809002DE9F0410D4B06461B680F461A
:100F0000904623B153F8044904B1043C0BB9BDE841
:100F1000F0811B681BB142463946304698472CB1D8
:100F2000656805B1043D23462C46EFE72546FAE700
:100F3000F43C00202DE9F04182B0012300AF0546CA
:100F4000386000F17001007A3B715DF0CAFEA0B913
:100F50004FF6FF7101203B46214A5FF050FD002112
:100F600028465FF079FF20B94FF6FF710120FDF7A9
:100F700053FF0837BD46BDE8F0812846FDF720FC49
:100F80000028E5D08468002CE2D0143C04F1100362
:100F900018465FF070F902071FD418465FF06BF92E
:100FA0008307C0F3400618D4214628460D4AFDF7B2
:100FB0001BFF002811DAE8468AB06A460A4BCDE9E1
:100FC0000740CDE90535052342F8103F4FF4225183
:100FD00033460648F2F778FEC5466469D3E700BF9A
:100FE00029FE01001D04080067F40A0014F8090036
:100FF00073B505460C466B46264A00918DF80400F1
:101000004FF6FF7101205FF0FAFC21462846F6F703
:1010100011FF00281DDB21462846FDF77FFE2146F3
:101020002846FDF7A3FA08B1FDF7F8FC214628464B
:10103000F6F7EAFE00280CDB174E3378AB4204D1FA
:101040002046711C5FF070F960B9337CAB4202D06E
:10105000002002B070BD204610495FF065F90028FD
:10106000F6D00F4EB368002BF2D053F8144904B1F8
:10107000143C002501E02346144600223146104668
:101080009D81FDF7D7FA002CE2D06269002AF2D0E8
:10109000143AF0E7B9E90100FC3C00200D3D0020C6
:1010A0000C3D00202DE9F74F044603464FF6FF7133
:1010B00001203A4A04F170065FF0A1FC3146207A23
:1010C0005FF0BAFC3146207A5DF00BFE50B1237A16
:1010D0004FF6FF718DF8043001206B46304A0096C0
:1010E0005FF08DFC2046FDF76BFB074640B92046BC
:1010F000FDF720FB054600283DD103B0BDE8F08F89
:101100008568002DF3D055F81489B8F1000F01D08F
:10111000A8F114084FF00009CA4601E04546984678
:1011200005F1100B6FF0080158465FF01FF93146CA
:10113000207A5DF0D6FD80B92B464A4639462046D6
:10114000A5F80CA0FDF776FAB8F1000FCFD0D8F8CB
:101150001430002BE2D0143BE0E758465FF08BF8E8
:10116000C307E9D47B781BB13146781C5FF009F9DD
:1011700005F11409E8E73146207A5DF0B2FD28B99F
:10118000284603B0BDE8F04FFDF748BC3146681C67
:1011900003B0BDE8F04F5FF0F4B800BF51ED0100BF
:1011A000B9E90100034B42689A4204BF836919827E
:1011B000704700BFAD0902007FB54FF420520023F5
:1011C000ADF8162004AA02920A4A0120CDE90032A5
:1011D0004FF6FF7105AA04938DF81430FEF74EF810
:1011E000049B012B14BF6FF01500002007B05DF8C1
:1011F00004FB00BFD30E0800014608B505485FF0A8
:10120000A1FE044B0028A3F1040314BF18460020DC
:1012100008BD00BFE4270020084B00F5B8701A682D
:10122000074BD0E8EF1F994204D1C0E8EC2FBCF186
:10123000000FF6D1D0E8AF0F704700BFEC3B0020A5
:10124000E027002008B5FFF7E7FFB8B1036843B116
:10125000426832B1826812B90B4A12783AB9042056
:101260000BE0094A127812B10BB1826842B94268A8
:1012700042B9002B14BF0020032008BD0320FCE767
:101280000120FAE70220F8E7EC89002038B50C4687
:10129000037BC17C03EA0102150704D5C27A857C71
:1012A0002A43D2070ED4042C0ED80B4313F00403A8
:1012B00006D0FFF7C7FF054B04EB840423441B5CF7
:1012C000184638BD0523FBE70023F9E74C3D0B002A
:1012D00038B50546FFF7A0FFD5F8EC3004469B7AF9
:1012E000032B0AD005D8013B012B8CBF0020012025
:1012F00038BD042B0FD00020FAE72846FFF7A2FFE5
:10130000032806D1002CF6D0E068003818BF012071
:10131000EEE70120ECE72846FFF794FF032802D10F
:101320001CB1E4680CB1024B1C7804F00100DFE74B
:10133000EC89002030B5037A044687B0052B1ED80F
:10134000DFE803F0250303251D3290F8DC20D0F8F8
:10135000D830D34003F0010343F08003134902ADBA
:101360000095096804F1370204F1570060F03EF976
:1013700078B101210E4A0F485FF0E2FD04E001213F
:101380000D4A0C485FF08BFE082007B030BD0023EB
:10139000E4E71022294604F117007DF09DFD003896
:1013A00018BF01208000F0E70020EEE71C3D002080
:1013B000C7F40A005CF80900ABF40A0008B5012183
:1013C000024A03485FF0BCFD002008BDE0F40A00BB
:1013D0005CF809000023024A00F5A0701DF0C0BDB2
:1013E0001C4E0E0038B5002304461A46EC300D465C
:1013F000FBF792FC58B1693004D10121064A074835
:101400005FF09EFD2846BDE83840F4F73DBB20461E
:10141000BDE83840FFF7DEBFF9EB0A005CF80900D1
:1014200073B50446D0F8EC60FFF7F6FE04214FF0E8
:10143000FF3305460DEB0100019313F0C9FBC8B95A
:10144000019B0D4A84F8DC00B3FBF2F102FB11337F
:101450000193C4F8D83055B12B6843B10B21201D3E
:101460005FF043FE30462B68D4F8D8109847002030
:1014700002B070BD0820FBE740420F0038B50446BB
:10148000051D082128465FF030FE084904F1570089
:10149000FAF756FA48B1082128465FF0F5FD0448EE
:1014A0000121044A5FF04CFD082038BD57140800A4
:1014B0005CF80900FBF40A0038B50546EC2200216F
:1014C0007DF002FD102105F1270013F081FB044699
:1014D00048B9052128465FF008FEFAF723FA034BC6
:1014E0001860204638BD0824FBE700BF1C3D0020E3
:1014F00070B5051D0E46284604215FF023FD68B136
:101500000022002100230846FBF7ECFB044638B913
:10151000042128465FF0E9FD204670BD034AF0E74C
:1015200001210C305CF09DFD0670F5E71C4E0E00AD
:1015300070B50C210546FFF7DBFF0446F0B14021F2
:101540000C305CF08EFD0E4B02461B68014603F129
:10155000200053F8046B834241F8046BF9D1203228
:1015600003F1200153F8040B8B4242F8040BF9D12C
:1015700028462146FFF736FF002070BD0820FCE713
:101580001C3D002070B5CD680446EB78102B70D15F
:101590002A7990F8E830D0F8EC60134080F8E83011
:1015A0006A7990F8E930134080F8E9300223037437
:1015B0002B68C0F81130AB88A0F81530AB781A074B
:1015C00006D5037B1B0703D5052104305FF08DFD95
:1015D000AB78980606D5237B990603D51421201DE8
:1015E0005FF083FDAB78DA0714D5237BDB0711D5D9
:1015F0000D21201D5FF079FD29782046FFF746FE7A
:101600002072D6F8A41020465FF0D7FC30B903252D
:10161000284670BD0023A4F8E830EDE720465FF0CF
:1016200001FD05460028F3D1261D052130465FF057
:1016300089FC0028EBD02046FFF7EEFD94F8E93056
:1016400084F8E85003F0020384F8E9300A4B1B6881
:1016500023B9062130465FF048FDD9E720460C212A
:101660005FF043FD0B215FF00FFDBDE87040FFF719
:101670005FBF0625CCE700BF1C3D00202DE9F041EF
:1016800004468CB01022002108A87DF01DFC237AAE
:10169000052B34D8DFE803F0060303063323D4F820
:1016A000D8300893D4F8EC3004F1470204F1C706AF
:1016B000CDE9016204F1270703F17E0204F1370846
:1016C000009239464246773304F1970001F054FE08
:1016D000F0B11E4A01211E485FF032FC14E0D4F83C
:1016E000E430002BDED008AD03F110062A4618685E
:1016F0005968083303C2B3421546F7D1D2E7012136
:10170000144A13485FF0CBFC08200CB0BDE8F08110
:10171000D4F8EC3004AD03F17E027733019304F189
:101720000A0302920093424639463046039508ABBD
:101730005FF081FF08B1084ACCE70D2120465FF039
:10174000D4FC29465FF00FFDDFE700BF14F50A0067
:101750005CF80900ABF40A0029F50A002DE9F04312
:10176000044691B0102200210CA87DF0ADFB237A35
:10177000052B34D8DFE803F0060303063323D4F83F
:10178000D8300C93D4F8EC3004F1470204F1C705CB
:10179000CDE9015204F1370603F17E0204F1270777
:1017A000009231463A46773304F1970001F0E4FDA8
:1017B000F8B13D4A01213D485FF0C2FB14E0D4F886
:1017C000E430002BDED00CAD03F110062A46186879
:1017D0005968083303C2B3421546F7D1D2E7012155
:1017E000334A32485FF05BFC0825284611B0BDE85B
:1017F000F083D4F8EC300DF1200803F177027E334A
:10180000019304F1110302920093324639462846AF
:10181000CDF80C800CAB5FF00EFF08B1254AC9E78C
:10182000237A052B0FD1D4F8E01019B30B460DF134
:10183000300C01F1100E624618685968083303C273
:1018400073459446F7D1D4F8EC300DF1100903F14B
:101850007E027733019304F10A03029200933A4621
:1018600031462846CDF80C900CAB5FF0E4FE30B169
:10187000114A9FE710220CA87DF026FBE3E7102217
:10188000494604F1B7007DF027FB58B94146204690
:101890005FF069FC05460028A6D10121201D5FF0FC
:1018A00024FCA2E70B25A0E714F50A005CF8090068
:1018B000ABF40A0029F50A004CF50A002DE9F041C5
:1018C000D0F8EC700446FD78CE6890B0002D69D158
:1018D000102229460CA87DF0F7FA237A052B50D860
:1018E000DFE803F0060303064F3ED4F8D8300C932C
:1018F00007F177030DF1200802937E3704F11103FD
:101900000093CDF80C8001970CAB04F1270204F191
:10191000370104F1C7005FF08EFE002836D1102297
:10192000314640467DF0D8FA002839D1627B237DCC
:1019300006A9069048609A4294BF00920093ADF8C1
:10194000140004F14703D4F8EC0005AA5DF0EBFDA8
:10195000002820DA0121284A28485FF0F1FA15E032
:10196000D4F8E030002BC3D00DF1300C03F1100E91
:10197000624618685968083303C273459446F7D124
:10198000B6E701211E4A1D485FF089FB082528465D
:1019900010B0BDE8F0810121201D5FF0A6FBF6E745
:1019A0000B25F4E7012D18D1051D102128465FF005
:1019B0006BFB314604F1B70306F1100251F8040B3A
:1019C000914243F8040BF9D1072128465FF0BAFA97
:1019D00028B1092128465FF088FB0025D7E70A21B6
:1019E00028465FF0AFFA0028F3D1204610B0BDE8DA
:1019F000F041FFF7B3BE00BF70F50A005CF80900C4
:101A0000ABF40A0073B5047A0546022C23D844B11E
:101A100090F8DC30D0F8D840DC4004F0010444F009
:101A2000800403212846FFF763FD0646D8B1102144
:101A30000C305CF016FB009012482346006805F15C
:101A4000270205F157015FF0D1FD044680B1304611
:101A5000F4F71AF807E0032C08D0012123460A4ABC
:101A60000A485FF01CFB082002B070BD0024D8E7D4
:101A700031462846FFF7B6FC281D21465FF004FBDF
:101A80002046F1E71C3D0020ABF40A005CF8090099
:101A900070B5061DCD6804460B2130465FF0F4FAA0
:101AA0002B4604F1170205F1100153F8040B8B4289
:101AB00042F8040BF9D1D4F8EC30DB783BB920467E
:101AC00004215FF012FBBDE870405FF02FBB237A6A
:101AD000012B09D0022B13D1204604215FF005FB16
:101AE000BDE87040FFF78EBF0A2130465FF02AFA4A
:101AF0000028F1D0304600215FF0F7FA002070BDD9
:101B000003480121034A5FF0CAFA0820F7E700BF43
:101B10005CF80900ABF40A0070B50446FFF77CFBE3
:101B2000261D05460E2130465FF00CFA70B9274B92
:101B30002022196804F157007DF0CEF930B9022156
:101B4000234A24485FF0FCF9082070BD2046FFF7C7
:101B5000EFFC0028F8D1237A052B31D8DFE803F019
:101B6000031D1003302D042120465FF0BEFAFFF75D
:101B700049FF0028E8D12046BDE870405FF0C5BAB3
:101B80002046FFF74DFC0028DED1032120465FF000
:101B9000ACFA0E215FF0A9FAEDE7204603215FF0D1
:101BA000A4FA0E215FF0A1FA30460A215FF09DFAF7
:101BB0006B68D4F8EC009847DDE704212046E9E79C
:101BC0000121054A03485FF06AFABDE71C3D002089
:101BD0008BF50A005CF80900ABF40A00F7B504467F
:101BE0000F46FFF719FB04F1570605463246FB681E
:101BF00003F1200153F8040B8B4242F8040BF9D196
:101C000004F1770203F1200153F8040B8B4242F8F0
:101C1000040BF9D13046F9F7EDFDD0B1201D0E21AE
:101C20005FF063FAD4F8EC70D7F8A40038B9387ACA
:101C300007F1700101F0A2F8C7F8A400A0B1438A2F
:101C400003F0240383B1437C9B070DD4032003B02E
:101C5000F0BD3046F9F7DAFD30B942480221424A78
:101C60005FF06EF90B20F2E7D4F8EC30DB78002B54
:101C700065D1271D0E2138465FF064F968B93B4BEA
:101C80002022304619687DF027F930B90221384A00
:101C900034485FF055F90820D9E7237A052B48D856
:101CA000DFE803F0031E08034728032120465FF006
:101CB0001CFA0FE02046FFF7B3FB0028EBD103210D
:101CC00020465FF012FA0E215FF00FFAFFF79AFE3E
:101CD0000028E0D1204603B0BDE8F0405FF015BA1F
:101CE0000A2138465FF001FA6B68D4F8EC00984797
:101CF0000E21DBE7102104F1270012F069FF0646F0
:101D00000028C8D165B3EB6853B31A4B20461B8833
:101D100001A9ADF804305FF0F3F838460C21C4E9AE
:101D200038665FF0E2F9EB68D4F8EC0001A9984757
:101D3000D0E70121104A0B485FF0B1F9ABE70B4B3C
:101D40001D682DB9201D06215FF0CFF928467EE7DA
:101D50002046FFF7E1FE003818BF0120C00076E7FB
:101D6000022074E75CF80900A6F50A001C3D00207B
:101D70008BF50A0078FA0900ABF40A00F0B50446C6
:101D800085B00F46FFF748FA04F13706054632469C
:101D9000FB6803F1100153F8040B8B4242F8040B6B
:101DA000F9D1D4F8EC30DB78002B56D12046FFF780
:101DB000C1FA00283DD1237A052B34D8DFE803F09F
:101DC0003B1C1C03333B03AB604800930068334665
:101DD00004F1270204F1570101F036FB40BB0A2150
:101DE000201D5FF082F909215FF07FF9AB6803994C
:101DF000D4F8EC00984728E094F8DC300133DBB2EB
:101E0000142B84F8DC3016D0102104F1270012F0D6
:101E1000DFFE68B9032120465FF067F905B0BDE831
:101E2000F040FFF7EFBD0121494A4A485FF037F91A
:101E3000082005B0F0BD231D072118465FF082F889
:101E400028B1092118465FF050F90020F1E720463B
:101E500005B0BDE8F040FFF711BC237A052BE2D8AE
:101E600001A252F823F000BFAD1E0200C51E020001
:101E7000C51E0200811E0200271E0200111F020063
:101E800003AB324900933246096804F1270304F199
:101E9000570001F0D9FA0028CAD10A21201D5FF0AD
:101EA00024F9AB680399D4F8EC00984720460D213B
:101EB0005FF01BF9201D10215FF017F920465FF03D
:101EC00035F9B6E72046FFF735FA0028B1D10321EE
:101ED00020465FF00AF95FF029F90028A8D194F8AC
:101EE000DC300133DBB2142B84F8DC3006D10D2159
:101EF00020465FF0FAF81021201DA4E7102104F11C
:101F0000270012F065FE003818BF0120C00090E7DE
:101F1000102104F1270012F05BFE0646002887D14D
:101F200095B1EB6883B10C4B20461B8803A9ADF833
:101F30000C305EF0E5FF0C21C4E93866201D5FF02F
:101F4000D4F8EB6803A953E7022072E71C3D002098
:101F5000ABF40A005CF8090078FA090038B50446C9
:101F60000D49A0F1EC05543061F0E9FC28465FF022
:101F700017F90A4A04F18403D3E8EF1FC3E8E02FFE
:101F80000028F9D14FF0FF338834D4E8EF2FC4E8AC
:101F9000E13F0029F9D138BDC92B0200E02700201C
:101FA000F0B589B0D0F8A44000AFE4B900F17001F9
